:020000040800F2
:10000000F0FF001071BE0508BD49050875E501083F
:1000100011BF050811BF050811BF05080000000049
:10002000000000000000000000000000C1490508B9
:10003000C549050800000000C949050851AD01087F
:1000400011BF050811BF050811BF050811BF05083C
:1000500011BF050811BF050871AF000879AF00088E
:1000600081AF000889AF000891AF00088DAC00088F
:10007000A1AC0008B5AC0008C9AC0008DDAC0008B4
:10008000F1AC000805AD000811BF050811BF050857
:1000900011BF050811BF050811BF050899AF000879
:1000A00099C50008F9C40008A9C50008E9C40008FA
:1000B00021C5000831C5000841C50008ADA30008EE
:1000C00039BA0008B5A300083DBA000811BF0508F9
:1000D00011BF050885A6010889A701088DA8010898
:1000E000A1AF000811BF0508F97E0508B9C50008D1
:1000F00071C50008C9C5000861C5000819AD000830
:1001000011BF050811BF050851C5000811BF05083A
:1001100091A9010895AA0108C1DA0008F9DA0008D6
:100120002DAD000841AD000855AD000869AD0008CF
:100130007DAD000811BF050811BF050811BF0508F6
:1001400011BF050811BF050811BF0508CD490508F5
:1001500091AD0008A5AD0008B9AD000899AB010844
:10016000BDA3000841BA000811BF050811BF05086A
:1001700011BF050811BF050811BF050811BF05080B
:0801800011BF050811BF0508BD
:10800000074BD0F8E4105B68D0F8F0205B1A9A4276
:10801000B8BFC0F8F030012380F81C310020704751
:10802000001000E0B94B00EB8002F0B503EBC20595
:1080300053F832205268918ACC074FEA800C74D4EE
:10804000CCB2A70743D5BFF35F8F297F0129CCB2FC
:1080500000F0E5804100148BBFF35F8F0CEB000450
:1080600003EBC404257F022D00F005810CEB000416
:1080700003EBC404257F032D08D1A47F34B10C1871
:108080001C4494F87850002D40F05F819488A4B28D
:1080900044F4806494800C181C4494F97AE00CEB4E
:1080A000000403EBC404247F013474450ED1014461
:1080B0001944002481F8784091F87910002940F0A3
:1080C000D380604403EBC00300225A76F0BD6607FC
:1080D00062D414F0400400F0E28000EB4001194447
:1080E000148A91F97AE06E6AE4B206F80E405FFAFB
:1080F0008EF6741C64B22F7F81F87A40E51CAF4283
:108100004FEA4001A64600F046810CEB000503EB68
:10811000C5052D7FAC42C2D10C1806F1020E1C44DD
:108120004FFA8EFE84F87AE0B9E7118821F40061F5
:108130000904090C1180118889B241F48061118011
:1081400000EB40041C44AE7F002184F87A1041000B
:10815000002E53D094F87840002C4CD00CEB000447
:1081600003EBC4040144247F19440125022C81F847
:10817000785004D1118889B241F4006111800CEB70
:10818000000103EBC101897E41F0010111826044CD
:1081900003EBC0031B7FF0BD00EB400E9E44AC7FA1
:1081A00001218EF8791000FA01F1002C00F0838093
:1081B0009EF87840002C40F084800CEB000403EB28
:1081C000C404647F002C00F0C3800D181D44148883
:1081D00095F87AE0A4B244F400740EF1010E148014
:1081E0004FFA8EF485F87A40B2F800E01EF4807FF2
:1081F000FAD1A64653E7EC7EFF2CAFD00CEB00047F
:1082000003EBC404A57E05F0FE051582E27EFF2A7D
:10821000BDD001441944FF2281F87A20B7E7A97F35
:1082200000293FF417AF00EB40051D44410095F8CD
:108230007860002E3FF40FAF168826F4806636046F
:10824000360C1680BFF35F8F85F87940148B148845
:1082500095F97AE0A4B244F4007414809488A4B22E
:1082600044F4806494801AE7918821F440710904F1
:10827000090C918025E7A47F002C3FF4F7AE0C1881
:108280001C4494F87850002D3FF4F0AE94F97AE055
:10829000148824F480642404240C14804EE01FFA13
:1082A00081FE1EF0800F33D100EB40041C444100DE
:1082B00094F97AE0F3E69EF87840002C3FF47DAF25
:1082C00083E72C7F022C14884FD924F48064240483
:1082D000240C1480178A6E6A9EF97A40FFB23755D3
:1082E0006F6A1588ADB245F400751580E4B2168A40
:1082F000651C6DB2F6B27E5595880234ADB264B29B
:1083000045F480658EF87A4095806DE76819002005
:1083100000EB40071F44410097F97A60B6F1FF3F38
:1083200040D02C6AA45D14822C7F06F1010E4FFA16
:108330008EFE744587F87AE07FF4B1AE948824F419
:1083400080642404240C9480A9E694F97AE0F5E78B
:108350001488A4B244F4807414800C181C440125C1
:1083600084F8785094F97A403EE7A4B244F400745B
:108370001480168A6F6A9EF97A40F6B23E55E4B2CE
:108380006F6A168A651C6DB20334F6B264B27E550C
:108390008EF87A4028E7958825F480652D042D0C09
:1083A0009580B2E6E97E1182A97F87F87A4019B9F3
:1083B000297F00297FF4EBAE918821F480610904C4
:1083C000090C9180E3E600BF1B4B01681B4A03F5D3
:1083D000727C03E063452CD053F82C2F9142F9D1E5
:1083E00070B593F804E0427996450AD0634505D00C
:1083F00053F82C2F9142F4D06345F9D14FF0FF3060
:1084000070BD9E468468DEF80C50A5424FF0000215
:1084100008D00132032A0EF10C0EE7D0DEF80C5022
:10842000A542F6D1DEF81050C668B542F1D150B27F
:1084300070BD4FF0FF30704718D7050800000140AD
:1084400030B5EAB18E464FEA014C034600F1C00553
:10845000002419689A6841EA0C0142EA0E029A6007
:10846000C3E900140C33AB42F3D1D0F8C030C0F8EC
:10847000C44043EA0E03C0F8C030C0F8C84030BD65
:108480004FEA014E8C46E0E783691969B3F80CC0E6
:108490000A6830B49C6822F0010224680A60A2894C
:1084A00092B222EA0C02A281027D04681F2A06D938
:1084B0006568203A08209040284245D0FEE72568AC
:1084C000082090402842F9D1202000FA02F2A26050
:1084D000264A1278002A35D01A7E012A39D0D3F8DC
:1084E000F4200132C3F8F420EFF31181502282F31B
:1084F000128858685C6C026822EA04029C6C224371
:10850000C9B2026081F31188D3E90C401A699968F5
:108510001D6C096814605061D3E90E40546090608E
:108520000024B3F8A800D5604C62C862106801242A
:10853000204310601C7683F8F1408A899B8913439D
:108540009BB28B8130BC7047202000FA02F2E260BF
:10855000BEE7002283F8F120D3F8F8000A68013062
:1085600022F00102C3F8F8000A60EBE704000010F3
:1085700010B40C4C6368002B11DD002004F1080CD2
:108580000146DCF8A03003F1C00259600C3393427D
:10859000FBD16368013083420CF5807CF1DC5DF82F
:1085A000044B704704000010F0B5494C04EB401C2C
:1085B0009CF8242402B9F0BD464B4FF08C0E0EFB04
:1085C000003E93F8E46493F8E5249EF886708CF8F6
:1085D0000A7496424FF0000C4FEA40158EF886C0A0
:1085E0000ED002EB420C03EBCC0C57009CF8E8C415
:1085F0000CF1FF3EBEF1010F5CD9BCF1030F53D06B
:108600006019A0F80814EFF31182902383F3128805
:1086100090F80A34B0F8081443EA41030021D2B2BA
:108620009BB280F80A1482F311881A09217882EA31
:1086300013225A40D9B1D0F82044D0F80C14D4F801
:10864000A040D2431B019BB202F00F0201208840E0
:10865000134304F1C0015A0013F4004F93B202D146
:108660006268024362600C348C42F4D1F0BDD0F8F1
:108670002014D0F80C04D1F8A0401B0100F1100127
:108680009BB202F00F0201208840134304F1C001A5
:108690005A0013F4004F93B202D162680243626041
:1086A0000C34A142F4D1F0BD02F1010C0CF0030C2A
:1086B000B445A5D03A4403EBC202131893F8F5145D
:1086C00000299DD06319012283F80A2498E700BF8E
:1086D0000400001068190020704700BF024B03EB34
:1086E000401090F825047047040000104368B0F86B
:1086F000502010B41A83EFF31182502383F31288B1
:108700004168446C0B6823EA0403C46C2343D2B26F
:108710000B6082F31188D0E907418268036912680F
:108720001C605961D0E909415C60C46A9960B0F885
:108730006010DC600023D1625DF8044B0376704763
:1087400010B4037D01681F2B09D94C68203B2022FF
:1087500002FA03F31C4215D15DF8044B70470C6814
:10876000202202FA03F31C42F6D00D4A406800248E
:1087700082F8484502685DF8044B22F0010202606D
:108780008B607047064A4068002482F848450268BA
:108790005DF8044B22F001020260CB60704700BF1D
:1087A00068190020704700BF0B4890F83C1589B14C
:1087B00001EB4101002310B4490000F244501C4673
:1087C00050F82320063302B114608B42F8D15DF8D3
:1087D000044B7047704700BF040000100B4890F82E
:1087E0003C1589B101EB4101002310B4490000F2AE
:1087F00044501C4650F82320063302B114609942BD
:10880000F8D15DF8044B7047704700BF04000010BA
:1088100001207047034B00EB400003EBC00090F8D1
:1088200055057047040000101F4890F83C35002B98
:1088300039D000222DE9F04300F244531B4E1C4D69
:108840004FF0500E4FF02C0C144607E053F8181B55
:108850000C6090F83C150132914222DD197C002910
:10886000F4D05F68B90AA1F5801105EB010952291E
:108870004FF0FE0898BF99F8F483EFF311898EF357
:108880001288796A0CFB08680131C8F87415B98A36
:1088900089B241F001015FFA89F8B98288F3118841
:1088A000D4E7BDE8F0837047040000106819002089
:1088B00018D7050807EE900AB8EE670A704700BFA0
:1088C000BCEEC00A10EE103A98B2704708B51D20F1
:1088D00011F080FB08B183794BB11E2011F07AFBB7
:1088E00008B1837903B108BD5523C38008BD552362
:1088F000C380F2E70D4B0E49DB68DB43C3F3022371
:10890000C3F104030122DBB202FA03F301EB000C12
:108910001B0103F0F0038CF80033430900F01F0043
:1089200002FA00F041F82300704700BF00ED00E0BC
:1089300000E100E0122301480B807047880100200D
:10894000042301480B8070479C0100202048D0F888
:10895000103AD0F8182A30B59B184FF01A040C8042
:1089600001D11C4830BD1B4AD0F8141A4FF0000E3C
:1089700010467546B3F1204F4FEA137C0CF13004DA
:108980000EF1020E2ABF0CF1370C847080F802C081
:10899000BEF1100FC5704FEA031300F10200E9D1D8
:1089A00000200446B1F1204F4FEA117303F1300C5F
:1089B00000F102002ABF373382F812C093740828EE
:1089C000D4744FEA011102F10202EBD1014830BD2B
:1089D0000070FF1FA0010020B42282804F224FF4BC
:1089E000A57C4FF4EB7102814FF487720023A0F84D
:1089F00002C0C1804FF4E17C962182814422037041
:108A0000A0F80AC0C18102824382704782B01F4B26
:108A1000002201920193019B1D4A04330193019BA3
:108A20001968936803F00C03042B07D0082B0AD0B5
:108A3000184B194AC3F8B42702B07047154BC3F856
:108A4000B41702B070475368506813F4800F00F0F9
:108A50003F00536813D1C3F388130F49B1FBF0F102
:108A600001FB03F30A4A0B495268C2F30142013287
:108A70005200B3FBF2F3C1F8B43702B07047C3F34E
:108A80008813B1FBF0F101FB03F3EBE75028004042
:108A900000380240681900200024F40001234377C5
:108AA00000207047D0E90B2108B583690B4483612E
:108AB0000AB108469047002008BD00BF436A1B6802
:108AC0001B6A5B685B78024613F0010008BF5077B1
:108AD000704700BF70B5224A224C234B94B0054624
:108AE000CDE90042214A0992A4F108020A922A7FA4
:108AF0000493201D0023CDE905039A42CDE90E33EE
:108B00000B931093139314BF0520042011936B6AE9
:108B10000C9002200122029018688DF80C200E465D
:108B200007928DF820208DF834208DF8482052F0DF
:108B3000BDF82B7F93B1330E04F8073C063C320C92
:108B4000330A22706370A670686A694610F0D4FD1B
:108B50006B6A186852F0AAF814B070BD073CEEE7D3
:108B600020210020C4010020BD8A00089D8A000841
:108B700010B5044694B050220649684654F004FDEE
:108B8000606A694610F0B8FD636A186852F08EF8A2
:108B900014B010BD60DB0508C2628161704700BF80
:108BA0002DE9F0410446406A00681E460F46904693
:108BB00052F07CF8237F002B3FD02A4DA06905237B
:108BC000EB67030E85F8453005F146039870020CFB
:108BD000000A58701A703B68C5F888300020D8F831
:108BE0000030C5F89030012E2363C5F8A0002BD0CB
:108BF000022E20D1D8F80420C5F89800796885F8AD
:108C00009400C5F89C1013441749C5F8A42001200E
:108C1000236385F8A800C5F8AC10144B617F606A27
:108C200003F11402002914BF1946114610F064FD27
:108C3000E36A8BB1206BBDE8F0810A4DA069042383
:108C4000EB6705F14503C1E7074B85F89460C5E97B
:108C50002630C5F8A400E0E7636A186852F026F8E9
:108C6000E8E700BF88010020A58A0008D4010020A1
:108C7000704700BF00B583B081610192049A0093F0
:108C8000C26201236A4601A9FFF78AFF03B05DF8BB
:108C900004FB00BF043070470D4B93F8C027D3F896
:108CA000BC170244D2B283F8C02793F8C027084407
:108CB0001206C3F8BC0705D593F8C02782F08002DE
:108CC00083F8C027034B012283F8C420704700BFFC
:108CD00068190020880100202DE9F047144FD7F8CB
:108CE000C457ED0A1ED00026B04607F2FC79D7F82B
:108CF000C8371048D3F828A0C7F8F487AC19641017
:108D000010234A46E102D0470F280BDD0A4B03F13E
:108D1000100C53F8041B013107D16345F9D12546E6
:108D2000B542E4DCE802BDE8F087661CF8E700BF66
:108D30006819002030210020642100201C4BD3F84A
:108D40000C18D3F810288A1A322A16D8D3F82428F7
:108D50008A4200D37047D3F8182822B3106892884B
:108D600010B444693231224218BF42835DF8044B8B
:108D700008BF0283C3F82418704793F81428D3F867
:108D8000181802F0010219B132B90A6889881183F2
:108D90000022C3F8242870470A688988518300227A
:108DA000C3F8242870473231C3F82418704700BF35
:108DB00068190020094A92F81438D2F8182803F0EC
:108DC00001031AB123B9136892881A8300207047EF
:108DD000136892885A830020704700BF68190020EA
:108DE0004FF40070034B1060D3F830380B60002054
:108DF000704700BF681900200020704701207047AD
:108E00000120704700207047012143F20102002336
:108E100043F2012C017202804FF60171FF22A0F88B
:108E200004C043818381C38101828274704700BF83
:108E3000154BFF224FF0FF3CF0B5C2700271027279
:108E400042724273827303F10C076646172516249B
:108E50004FF0150E002202EB820281189F4200F8AB
:108E600002E04C708D70CE7081F804C00BD093F985
:108E7000062093F807E01C7A5D7A93F90A6093F96B
:108E80000BC00633E7E7F0BDB0DB05084FF0000C80
:108E900001210222032380F805C08171C27103728F
:108EA000704700BF00230222037043708370C370B9
:108EB000027170472C22022302704370704700BF7A
:108EC0004FF4007141F20142002340F2593C01800D
:108ED00042804FF4E1610122A0F806C00381438182
:108EE0008181C281704700BF4FF0010C45210322F0
:108EF000002380F800C041708270C370704700BFCB
:108F00004FF4F07140F22E4C01804FF47A71A0F8CA
:108F10001EC041844FF4FA6C4FF4F561A0F820C0F4
:108F2000818440F2262C41F212310023A0F81CC0AB
:108F3000418141F2110C0E210722A0F808C080F8EF
:108F4000261040F2012C437183714374438240F236
:108F5000034140F205638270A0F814C0C18203830C
:108F600082767047114A002330B50360838002F196
:108F70000C054FF448744FF0290E4FF0280C03EB0A
:108F8000430300EB430100F813C081F801E0D378FC
:108F90008B70AA428C8008D092F9063092F807C0F4
:108FA00092F808E054890632E9E730BDC4DB0508D1
:108FB0002DE9F0430446406A344D006895B00E46F2
:108FC0009146984651F072FE314B0193314B049318
:108FD00005F1D0030093217F0223029305F1C8021B
:108FE000012300278DF80C3005920697002936D012
:108FF0008DF834308DF84830CDE90977330ECDE95E
:109000000E77CDE9107785F8C9300523CDF82C907F
:109010008DF82070CDF830801397CA350793330C44
:109020001D4F2B70330A6B70AE70D7F86408656AF9
:1090300010F01AFD637FA88033BB05A9284610F005
:109040005BFB636A186851F031FED7F8680810F0CE
:109050000BFD636A9880404615B0BDE8F0838DF83B
:1090600034308DF848300423CDE90911CDE90E11D3
:10907000CDE91011CDF82C908DF82010CDF830806E
:109080001391C9350793CAE76946D7E788010020DD
:10909000C8210020BD8A000868190020094910B5C0
:1090A0004B6C094C43F480434B644022002104F68E
:1090B0006C0054F0CCFA4FF0FF33C4F8AC38C4F86D
:1090C000AF3810BD003802406819002070B5224B3F
:1090D00093F8E42493F8E5349A4237D11F4D95F87C
:1090E0000436E3B195F808461D4B002040F20D3CD4
:1090F000B4B19A68998951601668196846F00106FA
:109100001660A1F848C08A8992B242F480728A81BE
:1091100095F804260130824203F11803E8DC70BDA3
:109120001A68118821F080010904090C11809988BE
:10913000D162118889B241F0800111805462998A0C
:109140009689314389B291819C82E1E750F0F2F82F
:109150000028C3D170BD00BF6819002004000010B2
:109160001C2200202DE9F0411E4B93F8E42493F8D3
:10917000E5349A422FD11C4F7D68002D12DD384610
:10918000002410F8086BA046013416B1037E012BB1
:109190001CD002691368AC4243F0010300F58070F3
:1091A0001360F1D111F020FED7F80C46002C0BDD36
:1091B0000E4A02EBC404116893888889083203437D
:1091C0009BB294428B81F6D1BDE8F08180F8F080AB
:1091D000FFF78CFADDE750F0ADF80028CBD1BDE801
:1091E000F08100BF68190020040000101406001070
:1091F0002DE9F04F037D02681F2B83B0044609D987
:109200005068A3F120052021A940014207D103B0F5
:10921000BDE8F08F1068202199400142F7D05149F4
:10922000514D4968C5F8301695F80816A7694F4E94
:1092300019BB8C2101FB0761D1F88C00D1F804E146
:10924000D0F800C0DEF80000B1F8908020F00100F6
:10925000CEF80000BCF80C1089B221EA0801ACF885
:109260000C10297801BB1F2B6FD9A3F120012023FB
:109270008B40D36003B0BDE8F08F8C2101FB076108
:10928000D1F88C10D1F810C00868DCF8001021F07B
:109290000101CCF80010818921F480710904090CC6
:1092A000818129780029DED04FF08C0808FB07F86F
:1092B00006EB08032E49D3F804A1D3F88C200193C0
:1092C000504608F11809D2F800B089444BF05CF818
:1092D000019BD5F838262649012083F8D800002ABA
:1092E0003AD0BBF800309BB243F08003ABF80030BB
:1092F00008F174084FF0FF334144CBF82C30584646
:109300004BF0C8F98C2303FB076600234946C6F8D7
:10931000A83050464BF0CEF8D6F8043116225A60E9
:109320001A6842F001021A60D6F88C20B6F8903024
:10933000126891890B439BB293810A49237D496846
:109340002268C5F834161F2B8FD8202101FA03F3A9
:10935000936003B0BDE8F08F11F046FD0449C5F8F5
:109360003806BEE7001000E0040000106819002075
:10937000EC190020F8B5164D1648174F00214FF490
:109380001A7254F064F905F688064FF0804105F62C
:109390006C043A46002301E054F8332091420BD08C
:1093A00001330E2BF8D100201C354FF0DBFDB54208
:1093B0000CD055F81C1CECE7084A02EBC3031C3523
:1093C00093F84C0D4FF0CEFDB542F2D1F8BD00BF81
:1093D000F4DB0508B41E00200000014018D7050882
:1093E0002DE9F04111F000FD1F4F204E05464FF0D2
:1093F00000087C68002C2ADD00231A4607EB0321B5
:10940000013391F8F9109C4242EA0102F6D142EA96
:109410000804E4B290467368C3F30803A3B9EFF3FA
:1094200011838BB914F006F9431BB3F5FA6F02DC14
:10943000B8F1000FDDD124B10D4B93F87429542AF3
:1094400009D02046BDE8F08111F0A0FCECE74446CD
:109450004FF00008DFE7B3F87C290132A3F87C293C
:109460002046BDE8F08100BF0400001000ED00E0E0
:1094700068190020BC4B1B780BB9012070472DE9FF
:10948000F04FBA4DBA49D5F80C28BA4BA1FB0212DD
:109490005209A3FB023A4FEADA0A0AEB8A0AA2EB64
:1094A0004A0A85B0B04A5FFA8AF3039302F61C13A6
:1094B00002F23C670193002307EB8A0A02F58169F7
:1094C0009846A94BD3F8243A434540F31781D9F87D
:1094D0001830D9F80460D3E93A34029311F084FCCF
:1094E000029B95F874C902904FEA860E95F8880998
:1094F0000EF1085E04F180610EEB431E3939BCF1B8
:10950000540F0EEB81110EEB801301D1A5F87E09EB
:10951000994240F26A811A68002A00F05E811A6C52
:10952000002A00F07081D3F88020002A00F06D81BD
:10953000D3F8C02003F58073002AE9D1A3EB0E0E07
:1095400099424FEAAE1E40F25081A4EB0E0145292C
:109550004FF0000428BF452103EB81119B462046B4
:1095600026460DE01A6C002A40F0D080D3F8802007
:10957000002A40F0F680D3F8C02003F580732AB9A2
:10958000994206D91A68002AECD04033994200F279
:10959000C180112E344640F22C81D6F1150200F123
:1095A00028817549029ED1F8D4309E45D5F88C3972
:1095B00038BFC1F8D4E0F11A002919DB03F5F42310
:1095C00003F590739E4288BF029B6B4988BF0533A9
:1095D000C5F88C39684BD3F8D430052B86BF053BD2
:1095E000DBB2002385F888394FF0FF33C1F8D4305F
:1095F00042B100FA02F2C4F11404012000FA04F4AA
:1096000044EA02005D4BC0F3C43203EB8202D2F89D
:10961000B81D00F01F0203EB8202D2F8B82D42EA17
:109620000131C0F3441203EB8202C0F3842003EB48
:109630008000D2F8B83D41EA0311D0F8B83D41EAC4
:10964000032181EA112383EA131303F00F030F2B85
:1096500040F0B180B1F5803F80F0AD80BCF1540F97
:109660004FEA111104D1B5F878390133A5F87839EA
:109670003D4AD2F82439B1F5606F03F10103C2F815
:10968000243900F0D480019B998197F858300398D1
:10969000834210D0DAF808203B689B1A3B60DAF866
:1096A00030207B689B1A7B600023CAF80830CAF818
:1096B000303087F858003B6801333B60DAF80830F7
:1096C0000133CAF808304FF6FF73994207D17B681F
:1096D00001337B60DAF830300133CAF83030019B57
:1096E00008F101081433B8F1080F07F15C070AF11B
:1096F0005C0A019309F120097FF4E3AE1A4A0123C1
:10970000012082F8203A05B0BDE8F08F80339942FD
:109710007FF63FAF5A469A1A9211541C184A82FBA0
:1097200004B2A2EBE472012AB8BF012290400124E6
:109730001644013A04FA02F210431C4622680AB3A6
:10974000226C002A63D0D4F88020002A61D0D4F89B
:10975000C02004F58074B2B1A142EFD89B462346E5
:109760000EE7C03312E700BF0400001068190020A4
:109770001F85EB51CDCCCCCC8801002018D7050833
:10978000565555554034A142E8D9E31A9B115A1C4D
:109790002F4B83FB02B3A3EBE273012BB8BF012372
:1097A00098401E440122013B02FA03F3184323466A
:1097B0009B462346E4E6BCF1540F2CD0254AD2F850
:1097C00024390133C2F82439224AD2F8203901332E
:1097D000C2F820394FF6FF7157E74033A3EB0E0E66
:1097E00099424FEAAE1E3FF6B0AE10B1013885F88F
:1097F0008809BCF1540F7FF472AFB5F87A390133A0
:10980000A5F87A396BE7803398E6C03396E6803462
:10981000B9E7C034B7E7B5F878390E4A0133A5F88F
:109820007839D2F824390133C2F82439CCE795F8D5
:10983000E53403EB430305EBC303434493F8F534EA
:109840000D2B7FF420AF019A802393771DE700BF93
:10985000565555550400001010B5044653F01CF938
:1098600081B22046BDE81040FEF79EBE38B50B4DD4
:1098700000EB400005F2445303EBC00393ED027A82
:10988000D3ED037AE7EE007AC4002C44B0EE670A09
:1098900053F002F9D4F84435186038BD04000010C4
:1098A0000C4AF8B5136855692B4003EA0005556169
:1098B0007DB1094F0126B5FA85F4C4F11F0407EB09
:1098C000840306FA04F4D3F86C0803689847A543A8
:1098D000F1D1F8BD003C014068190020038A2DE950
:1098E000F047B0F80C901FFA89F919EA03092BD058
:1098F00005460E464FF000474FF00008B9FA89F3CD
:1099000027FA03F2D24391B21B3B298209EA0209EA
:10991000042B16D8DFE803F0352C231A0300B36AB2
:10992000002B37D003F1FF3A1FFA8AFAC6F82880D5
:10993000746A34B123682046514698476468002C05
:10994000F8D1B9F1000FD9D1BDE8F0877068696B23
:10995000036889B29847B9F1000FCFD1F4E7B06836
:10996000A96B036889B29847B9F1000FC6D1EBE73C
:10997000F068E96B036889B29847B9F1000FBDD16F
:10998000E2E73069296C036889B29847B9F1000FA2
:10999000B4D1D9E7E96A1FFA81FAC9E70A4608B5DE
:1099A000054920B905484AF09BFF034808BD044813
:1099B0004AF096FF004808BDF8220020905406089F
:1099C000B854060810B5044C04480A4621464AF02B
:1099D00087FF204610BD00BFF8220020E054060893
:1099E00010B5044C04480A4621464AF079FF204647
:1099F00010BD00BFF8220020F454060810B5044C36
:109A000004480A4621464AF06BFF204610BD00BFBD
:109A1000F82200200055060838B590F82830012BB0
:109A2000044604D0407F40B10023637738BD406ACC
:109A300003681A7B92B9637F0BB9012038BD0A4DC8
:109A40000A49022305F529620FF0F4FE95F8913AD0
:109A500003F0010383F001006377E7E71B6A002B43
:109A6000E9D0002038BD00BF681900206002002046
:109A70002DE9F0410446154E90F82800637F144FFD
:109A800006F52968012805D00BB100236377012072
:109A9000BDE8F081606A05682A7B82B9002BF6D0A8
:109AA0000223424639460FF0C5FE96F8913A03F07C
:109AB00001036377002BEAD094F82800E2E72A6AD2
:109AC000002AE8D1002BE2D0EAE700BF68190020A5
:109AD00060020020F0B511F0010583B00AD190F8C2
:109AE0002860012E044607D0C368B3F1807F01D9F6
:109AF0000123237703B0F0BD0A4B476AD3F864080B
:109B00000FF0B2FFE368B880B3F1807FF2D9B721DC
:109B10008DF80410267733462A46384601A90FF0FF
:109B200089FEE7E7681900202DE9F047089F88467D
:109B300015460021202204461E4653F088FD4FB1F1
:109B40003B68E3811B0C23827B687A89E3821B0CD0
:109B500062822383404651F08BFAEB0619D4431EF0
:109B6000B8B108EB000701E0013B12D317F801CDB3
:109B7000BCF12E0FF8D1C01A421E032AA8BF03223F
:109B8000082B03F1010AA8BF08239146C2441A46D4
:109B900006E008280246C246A8BF08224FF0000986
:109BA0004FF0203341462360636004F108072046EC
:109BB00053F0EAFC174B23815146BB704A463846A6
:109BC00053F0E2FC611EE31D11F801CFACF1610E10
:109BD000BEF1190F9CBFACF1200C81F800C08B4284
:109BE000F2D1384604F10B0110F8013BA3F16102F8
:109BF000192A9CBF203B00F8013C8842F4D118236D
:109C00002373330CA382E572099B6683E361BDE88D
:109C1000F08700BF2020200008B54BF031FA0C4B34
:109C200093F8991D29220129A3F8F22AA3F8FA2A08
:109C300001D0012008BD0748C3F89C0D00F12001A8
:109C40004C304EF069FE044B002083F8230008BD21
:109C5000681900206402002000ED00E02DE9F04FBB
:109C6000DFF88894D9F80C08C9F8100887B0002BE1
:109C700000F0DA8001F5FE781344DFF874B4039342
:109C8000164601F12007C24621E0002E64D0D9F823
:109C90003C38B34200F0CC80D9F83838B34200F0F9
:109CA000FF80D9F84038D9F84418B3424BD8B142B4
:109CB00000F29981711A20464EF0DCFD039B0136BB
:109CC0009E4207F500770AF5007A00F0AD80D9F8DA
:109CD0004858B542A7F12004D7D8751BD9F8588841
:109CE00005F00702EB080492D8F8302002339342C3
:109CF00003D3D8F8382093420BD941461846059330
:109D00004EF088FD059B8046002800F08C81C9F844
:109D1000580898F80420002A40F03481D8F82850D8
:109D2000002D00F07981D8F830209B1A049A02EBBC
:109D3000C303D8F80C20204602EB43224FF40071F5
:109D40004346A847BAE7B142B4D920464FF400725F
:109D5000002153F07CFCB1E74FF4007231462046FD
:109D600053F075FC802387F89E310C2387F8A231CD
:109D7000D9F83838D44AD9F83018C4F8C6319342E3
:109D8000C4F8CA1100F33481D04AD14C82FB0302DB
:109D90001A44D817C0EB621284FB0254CD4D85FBE8
:109DA00003C5C0EB2530C2EB821587F8A1015B1B10
:109DB000801020F03F0001330343144487F8A031A2
:109DC000D317C3EBE4142244BF4B87F89F214A1EEC
:109DD0009A4200F31981BD4BBD4883FB0231114407
:109DE000D317C3EB611180FB0140BA4C84FB0254D2
:109DF000C3EB2433C1EB811487F8A531121B9B10F0
:109E000023F03F0301321343084487F8A431CB17F2
:109E1000C3EBE010014487F8A311552387F8DE3126
:109E2000AA2387F8DF3149E7002007B0BDE8F08FAB
:109E30004FF0FF3384F8EC3184F8ED3184F8EE31E3
:109E400084F8EF31D9F85038C4F8E8315223237040
:109E500063706123A37084F8E73141230025E37028
:109E600084F8E631722384F8E43184F8E5314FF464
:109E7000F0722946A7F11C0053F0E9FB5523C7F8FF
:109E8000D051C7F8D451C7F8D85184F8FE316FF0DB
:109E9000550384F8FC5184F8FD5184F8FF310DE737
:109EA00000214FF40072204653F0D1FB8A4A03CAC6
:109EB00047F81D0CEB2007F8200C582007F81F0C62
:109EC000902047F8191C07F81E0C002302220821D5
:109ED000F820E372227307F8131CA273E37307F8E8
:109EE000102C07F80B0CD9F8380884F82C20D9F876
:109EF00030286376121A2262D9F84008D9F844282B
:109F0000E376121A3F2020764FF0FF30A0763E20F5
:109F1000207701206377A377E37784F82D3084F8E6
:109F20002E3084F82F30626284F8300084F83130AB
:109F300087F82610802187F82010292187F8221021
:109F4000942187F823100E2187F824100D21634AED
:109F500087F82510552187F8DE11AA2187F8DF112F
:109F600003CA5F4BC7F82700C7F82B1003CB138831
:109F7000A7F82F309378C7F83200C7F8361087F863
:109F800031309BE64FF400720021204653F05FFB16
:109F9000049B002B4ED1D8F84030002B00F0AA8053
:109FA000049AD8F830304F49CDE9002220461122DA
:109FB000FFF7BAFDD8F840301A6C002A00F0AD80E7
:109FC000049A1B6BCDE90022474911223846FFF75E
:109FD000ABFDD8F8448007F120044FF4E075B8F1E8
:109FE000000F3FD16AE6F11A20464EF043FC65E6C9
:109FF000FF2387F89F3187F8A13187F8A031324BD2
:10A000004A1E9A427FF7E7AEFF2387F8A33187F80D
:10A01000A53187F8A43100E7294620464FF40072A5
:10A0200053F015FB4AE6A7F1240343F804BF9A4511
:10A03000FBD143E6D8F84030049AD8F84480002B8E
:10A040000CBF01230223C3EB02154346002B3FF450
:10A0500035AE013D9B6CF9D198464FF40075002B4D
:10A060003FF42CAE25442034234620354446049644
:10A0700098460EE05CF81C1B236BCDF800C0002650
:10A080000196FFF751FDA46C08F12008CCB1A8455A
:10A0900017D02379A44604F11C0E1122A8F1200048
:10A0A000002BE7D162792669236B216842F02102F7
:10A0B000CDE900E6FFF738FDA46C08F12008002C7C
:10A0C000E5D1049EFAE500BFFF03FB008320088270
:10A0D000818080809755454118550608245506080B
:10A0E0003055060810550608145506086819002052
:10A0F000DEADBEEF049BD9F83418CDE9003320461D
:10A100000822FFF711FDD8F84480B8F1000F3FF4A2
:10A11000D5AD3C464FF4F075A4E7049BCDE9003380
:10A1200052E700BF144B154910B5044618681B7957
:10A13000206284F82430152204F1250053F0D8FA67
:10A140000F4B93F8A02D4FF0010E84F83AE012B9AE
:10A1500084F83B2010BD03F6A45CBCE80F0020602F
:10A160006160A260E360BCE80F0084F83BE020611E
:10A170006161A261E36110BD3C55060844550608C3
:10A1800068190020084B10B5D3F8C43D18440C469C
:10A19000807D0FF01FFF18B1828803680CB11A830D
:10A1A00010BD5A83FCE700BF6819002010B42A498B
:10A1B0002A4A91F804367BB3D2F8B448A04239D089
:10A1C000012B29D0D2F8CC48844239D0022B23D09D
:10A1D000D2F8E448A04235D0032B1DD0D2F8FC4879
:10A1E000A04231D0042B17D0D2F81449A0422DD070
:10A1F000052B11D0D2F82C49A04229D0062B0BD028
:10A20000D2F84449A04225D0072B05D0D2F85C49AA
:10A21000844208BF07230ED003F1010C81F804C665
:10A2200003EB430102EBC1025DF8044BC2F8B40832
:10A23000184670470023DBB218465DF8044B7047A0
:10A240000123F8E70223F6E70323F4E70423F2E708
:10A250000523F0E70623EEE704000010681900204C
:10A2600038B5424C8C2303FB004393F8933003B979
:10A2700038BD94F8E4C494F8E5349C450ED003EB63
:10A28000430204EBC20292F8E8E40EF1FF35012D1F
:10A290004FEA430246D9BEF1030F3ED08C2202FBA7
:10A2A0000042A2F88410EFF31181902383F3128807
:10A2B000B2F8845092F8863043EA45030025C9B2CB
:10A2C0009BB282F8865081F3118829491A090D78CA
:10A2D00082EA13225A4005B1D2431B019BB202F01D
:10A2E0000F021A4391F808365BBB8C2303FB004432
:10A2F000D1F8283AD4F80C0101219847D4F8081174
:10A30000B4F890508A8AD4F804312A438A8258607B
:10A310001A6842F001021A6038BD5D1C05F00305A1
:10A320006545BBD0134404EBC303034493F8F51411
:10A330000029B3D08C2303FB0043012283F886203D
:10A34000ACE78C2303FB0044D1F8285AD4F88C30B6
:10A35000D4F808115B79086903F0FC031844042160
:10A36000A847D4F808318000988138BD68190020CA
:10A370000400001043680B4A23F0407323F48073F9
:10A3800043F48073436083681A4042F002028260A3
:10A39000C36A0139CAB223F4700141EA0251C162B1
:10A3A000704700BFFDF7FFC0704700BF0020FDF7FA
:10A3B00039BE00BF0120FDF735BE00BF0220FDF70A
:10A3C00031BE00BF10B1036882881A83704700BF96
:10A3D00010B1036882885A83704700BF10B40469C3
:10A3E0008269E468416814604024D46044690023B1
:10A3F0000C31C2E90433C2E90633C2E90833C2E9C9
:10A400000A33C2E90C3393609363516084B1C2692B
:10A41000E0689363C2E90233C2E90433C2E9063358
:10A42000C2E90833C2E90A33C2E90C33C2E90001C8
:10A430005DF8044B704700BF436800221A60037D3B
:10A440001F2B08D9203B2022016802FA03F343F0B6
:10A450001803CB6070472022016802FA03F343F02F
:10A4600018038B60704700BF0268136A11B1D96985
:10A4700001B3143330B49C681D689169DDB14FF4A9
:10A48000806088618D60104640690C6180B15968B8
:10A49000D369D9B10A464FF480619A609961224329
:10A4A00012F0010F14BF00224FF400521A621C6117
:10A4B00030BC704770478D61064D4FF0FF0C85F83A
:10A4C00044C105F5A27500688D60DDE7024A9A6017
:10A4D0009961E4E788010020302700200168F8B581
:10A4E000D1E9042304465568002B49D09861107DBA
:10A4F0005E681F2831D81768202202FA00F040F069
:10A500001800B8601A7D1F2A32D91868203A202313
:10A5100003FA02F242F01802C26000232B6033609B
:10A520003368896943F010033360284649F0C2FF5D
:10A5300023683046D96949F0BDFF2B68226843F093
:10A5400001032B603368526843F001033360938842
:10A550009BB243F003039380F8BD17682038202294
:10A5600002FA00F040F01800F8601A7D1F2ACCD8DB
:10A570001868202303FA02F242F018028260CCE746
:10A58000137D90611F2B1CD81068202202FA03F360
:10A5900043F01803836000232B602B68896943F024
:10A5A00010032B60284649F085FF2B68226843F092
:10A5B000010352682B6093889BB243F0020393809F
:10A5C000F8BD1068203B202202FA03F343F0180381
:10A5D000C360E0E72DE9F0417F4D804E07463C68BF
:10A5E00097F888806368B888012284F824201A8844
:10A5F00022F040021204120C1A802289824223D0D7
:10A60000198821F038010904AB424FEA114100F0EA
:10A61000BF80734A934200F0BB800246B2F5807F50
:10A62000A8BF4FF48072022AB8BF0222002A92FA11
:10A63000A2F2B2FA82F208BF4FF0FF32013A41EAC9
:10A64000C20292B21A802081397BA27A8A420CD04F
:10A650001A8822F003021204120C1A801A8892B28D
:10A66000002900F092801A80A1721A8892B242F0FA
:10A6700040021A80226A9168002900F0A3804FF0FE
:10A68000000C1432E64652F8100C8E4400EA060123
:10A6900020B1B1F1805F23D0616909B352F8140C85
:10A6A000143200EA060110B1B1F1805F18D052F8FF
:10A6B0000C1C0CF1010C0029E5D1227B82B1B8F110
:10A6C000000F0DD0BCF1010F6FD8BEF1070F6CD891
:10A6D0000CEB8C018900226A11440A7B002A64D0A9
:10A6E000226A92684FF00008002A53D0B8F1000F98
:10A6F00002D098F80C2022B1BA6812B11168928881
:10A700004A83226AD2F800E0226A5168226A92687B
:10A71000501E9AB1BEF1000F23D01EF801CB1A894A
:10A720009207FCD5A3F80CC01A89D207FCD59A89E8
:10A7300092B209B101F8012B0138EBD2236A1B7BDD
:10A74000E3B9236A1B697BB1236AD7F894001B69BC
:10A75000984701280DD0022806D100232362BDE8C6
:10A76000F0814FF0FF0CDAE7D4F82080236A14332D
:10A770002362236A9B686BB16368B7E7BB68002BF1
:10A78000DFD01A689B881383DBE742F003026AE795
:10A79000420843E7236A1B68DBB1236AD3E90072EE
:10A7A00022620022C3E9002219E700213846FFF7A0
:10A7B0005BFEBB6813B11A689B8853833846BDE8BB
:10A7C000F0418BE6227B002A8AD0B8F1000F82D1BB
:10A7D00086E72362C3E700BF003800400000FFFFA8
:10A7E000003C004038B5D0F8E0102B4B04465A68C6
:10A7F000D0F8D80071B1131A99420BDC94F8D0301C
:10A80000C4F8D820012B10D0D4F8D4300133C4F8C8
:10A81000D43038BDD4F8E430C4F8D8200344C4F8A8
:10A82000DC3094F8D030012BEED16168201D04F1AA
:10A83000E805EFF3118C102383F3128863681B6A19
:10A840000BB3D4F8F0302A461BB1D3691432002B75
:10A85000FBD10B6A6BB1996839B9934209D0196879
:10A8600029B15B6899680029F7D01433F3E7C3E98D
:10A8700000055FFA8CFC8CF31188D4F8D4300133D6
:10A88000C4F8D43038BD0D625FFA8CFC8CF31188AB
:10A89000FFF7A0FEB8E700BF001000E02DE9F0418F
:10A8A000826992F8DC30012B8AB005464CD0023B1D
:10A8B000012B54D892F84C31D2F89C202E4C63F0E6
:10A8C0007F0313708669D6F8A030D6F8108003F1A4
:10A8D000010E0FCCEC46ACE80F00D6F89C30CDE969
:10A8E000003E0FCCACE80F0094E8030006F110071F
:10A8F0008CE80300EFF31180102383F3128833698F
:10A900001B6A002B2FD0029B6A461BB1D3691432FD
:10A91000002BFBD1D8F8203073B1996839B9934234
:10A920000AD0196829B15B6899680029F7D01433F7
:10A93000F3E71F60C3F804D0C0B280F31188AA699E
:10A9400011690B6A002BFCD1D2F8A0305A8852BA98
:10A95000EA819A8852BA2A82DB885BBA6B8201202C
:10A960000AB0BDE8F081C8F820D0C0B280F31188E9
:10A970003846FFF72FFEE2E750E505082DE9F041E4
:10A9800090F8DC30D0F8A050012B8AB0044672D089
:10A9900016D8D0F89C304FF0FF321A605A609A6097
:10A9A000DA60D0F8E0300522B3F57A7FC0F8F02005
:10A9B0007CD8032380F8DC3001200AB0BDE8F081A8
:10A9C000023B012BF8D890F84D31D0F89C20524E24
:10A9D00063F07F031370D0F8A030D0F8108003F13B
:10A9E000010E00F110070FCEEC46ACE80F00D4F8D2
:10A9F0009C30CDE9003E0FCEACE80F0096E8030096
:10AA00008CE80300EFF31180102383F3128823698D
:10AA10001B6A002B73D0029B6A461BB1D3691432A8
:10AA2000002BFBD1D8F8203073B1996839B9934223
:10AA30000AD0196829B15B6899680029F7D01433E6
:10AA4000F3E71F60C3F804D0C0B280F31188226915
:10AA5000136A002BFCD16B885BBAA4F8D030AB88AA
:10AA60005BBAA4F8D230EB8801205BBAA4F8D430EA
:10AA70000AB0BDE8F08190F84C2190F84D319B1A56
:10AA80005B100133DBB205EB430235F813305BBAE0
:10AA9000A0F8D03053885BBAA0F8D23093885BBA64
:10AAA000A0F8D43001200AB0BDE8F08103691A7B18
:10AAB00072B35B6963B390F898304BB390F84C3144
:10AAC000D0F89C20C4F8A40063F07F03137090F8C2
:10AAD0004C1190F84D31D0F8A0201048C4F8040172
:10AAE0005B1A07330121C4F8FC30D4F89C3084F899
:10AAF00000110A44C4E93D3284F8DC105CE7C8F870
:10AB000020D0C0B280F311883846FFF763FD9EE77E
:10AB1000022384F8DC304FE750E505080180000887
:10AB2000D3B2012B23D870B502EB4202114C4FEA8D
:10AB3000820E4FF0000C22460EF10805634604E039
:10AB40000133152B11D012F81CCF6045F8D192F8C3
:10AB500001C08C45F4D15659002EF1D0C3EBC3038C
:10AB60000EEB83030433E01870BD002070BD00209D
:10AB7000704700BF78E5050810B40C4C002304F6BC
:10AB8000CC5C01E0152B0CD003EB430201331CF825
:10AB900002108142F6D122445DF8044B92F9CE0DA9
:10ABA00070474FF0FF305DF8044B70476819002084
:10ABB000D3B2022B21D830B502EB4202104D114C1A
:10ABC0004FEA820C0CF10C0E2A46002304E00133FC
:10ABD000172B10D052F82C4FA042F8D114798C4288
:10ABE000F5D152F80E40002CF1D02C2202FB03C309
:10ABF0000833E81830BD002030BD0020704700BF8A
:10AC000018D7050800000140002838D030B51C4D89
:10AC100090F804C0002305F6CC5401E0152B2CD08D
:10AC200003EB43020133A15C6145F7D12A44046878
:10AC300092F9CE3D90F805E0DAB2022A1DD803EB76
:10AC40004303104810494FEA830C02460CF10C05EF
:10AC5000002304E00133172B0FD052F82C1F8C4235
:10AC6000F8D111797145F5D151590029F2D02C2232
:10AC700002FB03C30833184430BD002030BD7047C9
:10AC80006819002018D70508000001400348D0F8D3
:10AC9000583113B100F5A47018477047880100209F
:10ACA0000348D0F87C3113B100F5B67018477047EF
:10ACB000880100200348D0F8A03113B100F5C87016
:10ACC00018477047880100200348D0F8C43113B1F9
:10ACD00000F5DA7018477047880100200348D0F863
:10ACE000E83113B100F5EC70184770478801002077
:10ACF0000348D0F80C3213B100F5FE7018477047C6
:10AD0000880100200348D0F8303213B100F50870F4
:10AD100018477047880100200348D0F8543213B117
:10AD200000F5117018477047880100200348D0F8DB
:10AD3000783213B100F51A70184770478801002067
:10AD40000348D0F89C3213B100F5237018477047C0
:10AD5000880100200348D0F8C03213B100F52C70F0
:10AD600018477047880100200348D0F8E43213B137
:10AD700000F5357018477047880100200348D0F867
:10AD8000083313B100F53E70184770478801002062
:10AD90000348D0F82C3313B100F5477018477047BB
:10ADA000880100200348D0F8503313B100F55070EB
:10ADB00018477047880100200348D0F8743313B156
:10ADC00000F559701847704788010020094B0A4A5E
:10ADD000013800EBC00003EB8000116BD0F8483164
:10ADE000064883420CBF4FF400134FF480030B431B
:10ADF0001363704788010020003802400060024061
:10AE000070B501383C4C3D4D00EBC00C04EB8C0C94
:10AE10009646DCF848613A4AAE420CBF4FF4001542
:10AE20004FF48005166B35431563CCF85811CCF8F8
:10AE300060313449DCF84C318B424FEAC0023ED0DD
:10AE400001F580618B423AD0A1F57A718B4247D0EF
:10AE500001F580618B4243D0A1F57A718B4241D0DC
:10AE600001F580618B423DD0A1F57A718B4235D0DE
:10AE700001F580618B4231D0A1F57A718B4233D0DC
:10AE800001F580618B422FD0A1F57A718B422DD0D4
:10AE900001F580618B4229D0A1F57A718B4227D0D0
:10AEA00001F580618B4223D0A1F57A718B4221D0CC
:10AEB000154D01F580618B4218BF002500E0134D50
:10AEC000104404EB8003CEF38711C3F8685193F864
:10AED0005D01BDE8704000224DF01CBF0C4DEFE756
:10AEE0000C4DEDE70C4DEBE70C4DE9E70C4DE7E7BA
:10AEF0000C4DE5E7044DE3E78801002000600240C7
:10AF000000380240106002400080002820800010BD
:10AF10000080001800880010008020102080002091
:10AF20000088002000802020800AA0F58010522890
:10AF300008D8054B184490F8F4330D2B02D8034A77
:10AF4000D05670470020704718D70508D855060816
:10AF500058B183884FF00042B3FA83F332FA03F317
:10AF600003D002490A6813430B607047003C01405C
:10AF70000120FEF795BC00BF0220FEF791BC00BF88
:10AF80000420FEF78DBC00BF0820FEF789BC00BF7F
:10AF90001020FEF785BC00BF4FF47870FEF780BC30
:10AFA0004FF47C40FEF77CBC30B50C4683B00546C0
:10AFB00018B3036803F13F4303F57E039B0A104A6D
:10AFC000134413F84C0C4DF0CDFFA988009104F008
:10AFD0000303C4F381028DF8043028688DF805203E
:10AFE000C4F300136946C4F341148DF806308DF89C
:10AFF000074049F01BF903B030BD4FF0FF33DEE7E7
:10B0000010E8050800B1CFE7704700BFF8B5CB786E
:10B0100013B900252846F8BD00F110070C46064676
:10B02000897838460EF04AFD05460028F1D0E078D0
:10B030000EF0D0FFB06123780133DBB210B1C371E1
:10B04000222383710921FFF7DDFFB069FFF7BAF909
:10B050000D4AD2F80C38632BFBD90C480EF004FDD6
:10B06000B082384643F054FC074630B9E0780EF021
:10B07000B1FF0FF00FF83D46CCE7306986F8D87085
:10B080004FF018FEC6E700BF6819002040420F00CD
:10B090000B4B10B5D3F8C43D03440446987D0EF025
:10B0A00099FF60B12E228271621CC2710121FFF7EB
:10B0B000A9FF20460021BDE81040FFF763B810BD8E
:10B0C0006819002070B50E4CD4F8246A002E15DDE6
:10B0D00004F58164002503E0B54204F120040DD09D
:10B0E000237F0135002BF7D0E0680028F4D0217DC4
:10B0F000FFF75AFFB54204F12004F1D1012070BDE1
:10B1000004000010F8B5037D85691F2B04464DD956
:10B110000168A3F120024E6820209040064234D0FE
:10B1200010239340C860CB604B68D340DE0700F12A
:10B130008380EFF31183502282F312882A6C116806
:10B14000C9075AD4516889B271B9D5E909608642F4
:10B1500050D0AF690744D76073D9301A80B25060BD
:10B16000AE62002185F86410116841F00101DBB284
:10B17000116083F3118895F86430002B44D1237D4E
:10B180001F2B27D92168A3F120024C68082090408A
:10B19000044200D0C8604C68042000FA02F2224247
:10B1A00003D0203B00FA03F3CB60F8BD02682020F7
:10B1B00016689840064219460ED0102199409060BA
:10B1C00091601168D940C807B3D5012101FA03F392
:10B1D0009360AEE722681946106808238B40184236
:10B1E00000D093601068042303FA01F10142DCD01F
:10B1F0009160F8BD012285F86420DBB283F31188E9
:10B2000095F86430002BBAD095F87C30002BB6D17D
:10B2100095F871000EF0DEFE2A6E938923F0080384
:10B220001B0401211B0C938185F87C100028A6D0FB
:10B230002021FFF7B9FEA2E7012303FA02F2CA6058
:10B2400077E72E69301A80B25060A96289E700BFA3
:10B2500070B50C4682B015460646002839D0036802
:10B2600003F13F4303F57E039B0A1B4A134413F883
:10B270004C0C4DF077FEB2880092B2FA82F304F0E3
:10B2800003028DF80420C4F3810230688DF8052094
:10B29000C3F11F03C4F30012C4F341148DF8074037
:10B2A000C3F3CC0400EB840403F007038DF80620FD
:10B2B0009B00226A0F269D4006FA03F322EA03034D
:10B2C0002362226A15436946256248F0AFFF02B047
:10B2D00070BD4FF0FF33C8E710E8050800B1B7E7CD
:10B2E000704700BF2DE9F043774D05EB001683B0A2
:10B2F000D6F80C3E002B00F0938004464FEA00186D
:10B3000096F8140E4DF02EFE96F8143E590903F0EF
:10B310001F0203294FF0010303FA02F300F09880A3
:10B32000042900F0858002297DD005EB0803013453
:10B3300093F8100E0EF04EFEE4B2814610B11223C7
:10B340008371C47105EB080393F8110E0EF042FEF1
:10B35000074610B11323C471837105EB080393F8FA
:10B36000120E0EF037FE064610B11423C47183711D
:10B370004544484695F8132E01924A21FFF7AEFF47
:10B38000019A38462A21FFF7A9FF019A0A2130467F
:10B39000FFF7A4FFD5F80C2E4C4B9A425DD04C4BD6
:10B3A0009A424AD04B4B9A4262D04B4B9A426AD057
:10B3B0004A4B9A4272D04A4B9A427AD04949908875
:10B3C000B1F88A43B1F88833B1F892532343B1F806
:10B3D0008C432343B1F88E4320F003002343B1F89C
:10B3E00090430004000C2343B1F8944390802B4316
:10B3F00010882343B1F89643B1F8981300F44150F4
:10B40000234303439BB21380938B23F400631B04F9
:10B410001B0C9383118213889BB243F0400313806B
:10B4200003B0BDE8F083304A516A0B4353627CE7B6
:10B430002D4A11690B43136177E703F50033196A4D
:10B4400041F480411962196A21F480411962B5E71B
:10B45000254A116A0B43136267E703F58433596A7F
:10B4600041F480515962596A21F480515962A5E72B
:10B4700003F5FE33196A41F400411962196A21F497
:10B48000004119629AE703F58233596A41F4005189
:10B490005962596A21F4005159628FE703F56843F4
:10B4A000596A41F480115962596A21F48011596234
:10B4B00084E703F56443596A41F400115962596AFB
:10B4C00021F40011596279E7681900200030014029
:10B4D00000380040003C0040003401400050014072
:10B4E000005401408801002000380240431C00F055
:10B4F000A8802DE9F04F00EB8003C44FDA0087B03D
:10B5000057F8029081000546019107EBC303B9F19A
:10B51000000F04D09C68002C4BD0A17911B107B06A
:10B52000BDE8F08FD3F80CA0BAF1000F00F09581C0
:10B530009AF80630002BF2D11832B818D9F80480E6
:10B54000BB50691CC0E90133C3601523A371C9B2A4
:10B550001623E1718AF807108AF8063099F8180066
:10B560004DF000FDB8F804302268A18823F4407340
:10B570001B041B0CA8F80430DAF800301183BAF869
:10B5800004201A8311212046FFF70EFD1121504699
:10B59000FFF70AFD09264FF0330B24B12268A1887A
:10B5A0001069014231D1BBF1010B45D04EF0B4FC22
:10B5B000F3E7D3F80CA0BAF1000F00F0A4819AF8D9
:10B5C0000630002BABD11832BB18D9F80480BC5020
:10B5D000C3E90144DC6016238AF806306B1C8AF844
:10B5E000073099F818004DF0BDFCB8F80430BAF8EF
:10B5F000042023F440731B041B0CA8F80430DAF871
:10B6000000301A83C2E7A188226851834EF028FCDB
:10B610002368A2881A834EF023FC013EBBD1332657
:10B6200024B12368A28819690A420DD1013E00F0B5
:10B63000FB804EF071FCF3E7002CE4D14EF010FCDF
:10B64000E9E77047A28823685A834EF009FCBAF1F3
:10B65000000F00F02481DAF80030BAF804205A8391
:10B660004EF0FEFB002C00F0EE802368A2881A83C7
:10B670004EF0F6FBDAF80030BAF804201A834EF0E8
:10B68000EFFB2368A2881B691A4240F0A080019B4F
:10B690002B4407EBC3039A7C002A40F095801A7C68
:10B6A00012212046FFF7D4FD019B2B4407EBC30377
:10B6B0009B7C002B00F08F803221BAF1000F07D065
:10B6C000019B2B4407EBC30350465A7CFFF7C0FD98
:10B6D0004F4B984500F0EF804E4B984500F0F680B8
:10B6E0004D4B984500F0FD80019B2B4407EBC307B1
:10B6F0004FF47A73BC8A03FB04F4B8F8043023F4E3
:10B7000040731B041B0CA8F80430B8F800309BB23F
:10B7100043F00103A8F80030B8F8045002A848F03C
:10B72000CFFD25F03F0504993C4B2D04A3FB0123DD
:10B730002D0C45EA9345A8F80450B8F8002022F0F3
:10B7400001021204120CA8F80020354A980C944209
:10B75000034642DC6200B1FBF2F292B20133042AEA
:10B7600038BF0422A8F82030A8F81C20B8F8003010
:10B770009BB243F00103A8F80030B8F8003023F47E
:10B78000816323F002031B041B0C4FF4804143F43C
:10B790008063A8F80030A8F80810B8F8003023F04B
:10B7A00080031B041B0C0022A8F8003099F81A0033
:10B7B00011464DF0AFFA002299F81900114607B072
:10B7C000BDE8F04F4DF0A6BA1A7C322169E7DAF8ED
:10B7D00000301B695BE712216FE704EB4404B1FB07
:10B7E000F4F18AB2C1F30B0109B942F001020D492B
:10B7F0004FF4967300FB03F3A1FB03139B09013382
:10B8000042F40042A8F82030AEE700BF68190020DB
:10B810000054004000580040005C004083DE1B43A1
:10B82000A0860100D34D6210002C7FF40BAF4EF0C8
:10B8300017FBBAF1000F5FD0DAF80030BAF8042035
:10B840005A834EF00DFB4EF00BFBDAF80030BAF8DD
:10B8500004201A834EF004FB26E71832BB18D9F8EF
:10B86000048047F802A0C3E901AAC3F80CA015237D
:10B87000A371431CE37199F818004DF073FBB8F8FD
:10B880000430A28823F440731B041B0CA8F8043076
:10B89000236811211A832046FFF786FB7AE64EF0D3
:10B8A000DFFA2368A2881A834EF0DAFA4EF0D8FA4B
:10B8B00023681B69EBE603F5F2331A6A42F40012BF
:10B8C0001A621A6A22F400121A620DE703F5F033C5
:10B8D0001A6A42F480021A621A6A22F480021A6218
:10B8E00002E703F5EE331A6A42F400021A621A6A9A
:10B8F00022F400021A62F7E64EF0B2FA4EF0B0FA05
:10B900004EF0AEFAD0E61832BB18D9F8048047F8EA
:10B9100002A0C3E901AAC3F80CA099F818004DF0E1
:10B9200021FBB8F8043023F440731B041B0CA8F867
:10B9300004302FE62DE9F84307460FF027FADFF829
:10B940004C8007EB8709044608EBC90542F20F76E5
:10B9500004E00FF01BFA031BB3420ADC6B7E002BE2
:10B96000F7D108EBC90898F8180080F00100BDE88D
:10B97000F883B8F83C3E013338469BB2A8F83C3E09
:10B98000FFF7B4FD0020BDE8F88300BF6819002070
:10B9900070B500EB8003274D05EBC30255F833303B
:10B9A0005C68A38A84B09BB20393039B13F4706F0B
:10B9B0001CBF01231376039B13F4E06F4FEA80064C
:10B9C0000CD1A38A304423F4706305EBC0051B043B
:10B9D0001B0C0022A3826A7604B070BD238BA3885F
:10B9E00023F480631B041B0CA380039B9A05E8D4FB
:10B9F00023889B05E5D42388D9050FD52388DA054C
:10BA0000FCD423889BB243F40073238023889B05D6
:10BA1000FCD40190FFF76AFD0198D2E723889BB21E
:10BA200043F400732380A38823F440731B041B0C8E
:10BA3000A380C6E7681900200020A9E70120A7E736
:10BA40000220A5E72DE9F84F2F4F00EB800407EB0C
:10BA5000C404D4F80480B8F1000F04D09A46637E81
:10BA600003F0FF0923B14FF000094846BDE8F88F05
:10BA70000E46934605460FF089F90A9B7600F6B20A
:10BA8000C4E908330123A67684F81BB084F81D901E
:10BA9000A37784F81CA0637684F81890B8F8042083
:10BAA0009105064622D4B8F80030DA0512D442F2E5
:10BAB0000F7404E00FF06AF9831BA3421ADCB8F894
:10BAC00000309B05F6D4B8F800309BB243F4807385
:10BAD000A8F80030B8F804309BB24FF0010943F4E5
:10BAE0004073A8F804304846BDE8F88F99464846A8
:10BAF000BDE8F88FB7F83C3E01339BB22846A7F863
:10BB00003C3EFFF7F3FCB0E768190020F8B590F869
:10BB100071301C09013C052C0FD81B4E06EB44026A
:10BB2000054632F8440C03F00F0340FA03F2D20743
:10BB300003D595F87C70012F01D00120F8BD07FADC
:10BB400003F3013B184034444FF0BEFF14F8382C87
:10BB50000E4C104454F8302004EBC0041069A38844
:10BB60001840EBD0EB6E002285F87C2093F8212062
:10BB700020460221FFF76CFB2A6E93899BB243F0AB
:10BB8000080338469381F8BD10E80508FC2300201F
:10BB9000094BD3F8402ED3F8441E40F22A4000232C
:10BBA00050604B620B889BB243F001030B8013681B
:10BBB00043F0010313607047681900201D4B1E48B5
:10BBC000196C1E4A10B441F08051012419640462BA
:10BBD0005321FF24CA205462506251625B6FDB0024
:10BBE00085B017D416480423002102910290029ACE
:10BBF0001A440292029A04331C2B1160F5D103916E
:10BC00000390039B0393039B0E4A1A6005B05DF8F3
:10BC1000044B70470A4B002201920193019B019350
:10BC2000019A084B12689A42DCD105B05DF8044BCA
:10BC3000704700BF0038024000000E42002800405C
:10BC4000502800403166654210B5174C84B0013968
:10BC5000002389B2A042ADF80C30ADF806308DF863
:10BC60000E30029113D0114B984210D003F580434F
:10BC700098420CD003F58063984208D003F58063A6
:10BC8000984204D00A4BD3F8B4375B0802E0084B63
:10BC9000D3F8B437B3FBF2F201A9013AADF80420AE
:10BCA00048F0AAFC04B010BD0004014000000140AF
:10BCB0006819002030B50446006EA268838923F419
:10BCC00000531B041B0C8381637995B013F0040FA0
:10BCD0004FF00001019214BF4FF480520A46ADF8B4
:10BCE00008201A031B0203F48063ADF80C3023799B
:10BCF000ADF80E1002F40052ADF80A20DA0744BF86
:10BD00000422ADF80E209B07ADF8101005D5BDF844
:10BD10000E3043F00803ADF80E3001A948F07EFD67
:10BD20006279236ED50700F18B8012F0080F9A8A92
:10BD300048D092B242F008029A829A8992B242F4B2
:10BD400000529A812279D00732D5E06B002800F0AA
:10BD500089800023E26D0893CDE90C33CDE91033DF
:10BD6000CDE912334FF480750A936369E1680E954B
:10BD700006920793626C05924FF480634FF480350E
:10BD80000B9309910F9548F0FFFA05A9E06B48F075
:10BD900091FBE26B216E136843F0010313608B8A01
:10BDA0009BB243F040038B82536822799BB2636558
:10BDB00091070DD4226E93899BB243F40053938173
:10BDC00015B030BD22F008021204120C9A82B4E7BA
:10BDD000206C002852D02369A26D0993A36CCDE991
:10BDE0000532402300254FF4803108934FF48063DF
:10BDF0000B930F91CDE90C55CDE91055CDE91255B6
:10BE000007950A950E9548F0BFFA206C05A948F0F1
:10BE100051FB236C226E586940F08000586118680D
:10BE200040F0160018605D60938A9BB243F0800377
:10BE300002F10C0193820B6843F040030B60BAE7F8
:10BE40001E498B4224D0A1F54C418B421ED001F5F6
:10BE500080618B421ED102200121FEF793F96279A5
:10BE6000236E62E74FF6DF711980D96841F0200137
:10BE7000D960D96841F01001D96099E7226ED36882
:10BE800043F0800302F10C01D360D4E70120E3E723
:10BE90000020E1E701F580618B420AD001F5806165
:10BEA0008B4208D001F544418B427FF43EAF052020
:10BEB000D2E70320D0E70420CEE700BF0010014006
:10BEC0002DE9F84F4D4C04EB8004D4F82C4A002C9B
:10BED0007DD0E56E002D76D01F46EB6A6361AB6ABC
:10BEE000A3616B8EE3602B8E23616B682366444BEA
:10BEF0002360444BA160A3660646204690460EF0A0
:10BF00000BFA94F871000EF065F8814695F8200060
:10BF100094F870B0A24600284ED10223390784F865
:10BF20007C3036D418F0020F10D0B9F1000F0DD0CC
:10BF30000B2389F80630731C89F807303B0648D478
:10BF400095F8212048462221FFF782F918F0010FC9
:10BF500004D1E26B9AB15046BDE8F88F58460EF016
:10BF600039F80028F5D00C220136C671827195F897
:10BF700021202221FFF76CF9E26B002AEBD195F822
:10BF8000241095F8220089094CF0C4FE5046BDE803
:10BF9000F88F0136F6B2B9F1000FDAD00B237A062A
:10BFA00089F8076089F8063009D595F821204221E3
:10BFB0004846FFF74DF9CCE74CF0D4FFADE795F8D4
:10BFC00021201221F4E7AA465046BDE8F88FA24688
:10BFD000C1E794F871000DF0FDFF226E938923F004
:10BFE00008031B0401211B0C938184F87C1000289A
:10BFF000ACD02021FEF7D8FFA8E700BF0400001056
:10C00000E0E705080DBB0008BFF34F8F0549064B5D
:10C01000CA6802F4E0621343CB60BFF34F8F00BFE6
:10C02000FDE700BF00ED00E00400FA0508B50021BF
:10C03000032048F0C1FA72B6FFF7E6FF08B5184CC6
:10C04000D4F8482E94F84E0E4AB1116893880969C5
:10C050000B40F8B9003B18BF0123002BF4D114208A
:10C0600011F034FD00BFD4F8483E63B11A689B88D4
:10C07000116994F84E2E0B4042B9003B18BF0123C2
:10C080000BB1FFF7D3FFFCF759FEEBE7B3FA83F3ED
:10C090005B09F5E7B3FA83F35B09002BD4D1DEE744
:10C0A0006819002008B572B6FFF7AEFF00B583B07F
:10C0B0000D49002200920091009B0C330093009BDD
:10C0C0001B68012B02D003B05DF804FB01920191C3
:10C0D000019B06490C330193019B1A600B6883F3A3
:10C0E00008884B689847FEE7502800400000FF1F73
:10C0F00038B5FFF763FDFFF7D9FF012048F06CFA70
:10C10000704A936823F003039360936813F00C0F55
:10C11000FBD113686B49002840D143F00103136041
:10C1200041F288330A6895075BD4013BFAD1664C2B
:10C13000664D644B664AEA60664A596FAA60596B5D
:10C14000654821F080015963596F41F0807159674A
:10C15000196B41F4CE0119635A6B5A639A6B9A6357
:10C160001A6C02431A64596C5C4A0A435A640EF012
:10C17000C5FDD4F8B4375A4AA2FB03239B09013BFF
:10C18000B3F1807F09D24FF0E022F020536100210B
:10C19000072385F823009161136138BD43F4803390
:10C1A00013600A68940341F2883304D4013BBED083
:10C1B0000A689403FAD5444C4A4A4B4BB0FBF3F35C
:10C1C000B0FBF2F0B3EB400F18BF18464FF48002FB
:10C1D000B3FBF0F3C4F8642EC4F8500EC4F8543E18
:10C1E00009E0394C002108220223C4F8641EC4F877
:10C1F000502EC4F8543E022048F0EEF903280FD820
:10C200003A4BD4F8541E03EBC0008588C28843889B
:10C21000C4F85C5EB3FBF1F3C4F8602EC4F8583E7A
:10C22000284B33491A6C42F080521A640A6842F46F
:10C2300040420A609A689A609A6842F400429A60A2
:10C240009A6842F4A0529A60D4F8640ED4F8502E42
:10C25000D4F8581E024342EA8112D4F85C1ED4F886
:10C26000600E490842EA0062013942EA01425A601E
:10C270001A6842F080721A601A689201FCD51D4A51
:10C2800040F205711160996821F003019960996885
:10C2900041F00201A2F580629960936803F00C03FB
:10C2A000082BFAD1D4F8540E1349D823B3FBF0F37A
:10C2B0009B0143F000530120C2F884308866FCF7EC
:10C2C000A5FB35E7003802406819002000ED00E0CA
:10C2D0000005FA0500000020FFC9FE36335F0700A5
:10C2E000D34D621080841E0040420F0010E8050804
:10C2F00000700040003C02400000474210B584B08E
:10C3000000230446ADF80C300068ADF806308DF817
:10C310000E3003F18043013903F5823389B298422C
:10C32000029114D0A3F58063984210D003F58043A6
:10C3300098420CD003F58063984208D003F58063DF
:10C34000984204D0204BD3F8B4375B0802E01E4B70
:10C35000D3F8B437B3FBF2F301A9013BADF80430D5
:10C3600048F04AF92168194A0B8819489BB243F0F2
:10C3700001030B80002301E050F83320914208D0E4
:10C3800001330E2BF8D1002004B0BDE81040FCF7BB
:10C39000B1BA104A02EBC30393F84D4D2046FCF7A7
:10C3A000A9FA1B2C05D1192004B0BDE81040FCF7F8
:10C3B000A1BA2E2C08BF2C2004D104B0BDE8104037
:10C3C000FCF798BA04B010BD6819002000000140C5
:10C3D00060E4050818D7050870B50468A30AA3F53A
:10C3E0008013522B51D83C4D2B4493F8F4530D2D10
:10C3F0004BD840798608002954D005EB850305EB1E
:10C400004303B4F80CE04FEA900C33440220334E5F
:10C4100000FA0CF040EA0E0006EB830C80B2CCF878
:10C420005015CCF86025A081EFF3118C502383F3D5
:10C4300012882C2305FB03F3F118D1F84C2562B3C5
:10C44000274BC1F87025043226482C2105FB01F149
:10C45000084414310B4453F8041B19B1116053F80C
:10C46000042C04329842F6D100235FFA8CFC13604E
:10C470008CF311882C2303FB0565D5F870352BB19F
:10C48000A3899BB243F00103A38170BDA38923F06C
:10C4900001031B041B0CA38170BD03F12402104B8C
:10C4A0001A44D1E7B4F80CC005EB8503304605EB20
:10C4B00043034FF0020E33441FFA8CFC074E0EFA72
:10C4C00000F02CEA0000A08106EB8300C0F85015B4
:10C4D000C0F86025A8E700BF18D705086819002034
:10C4E000B41E0020D81E002001490248FDF7F6B90D
:10C4F000B41E00200000014010B5064C064804F2AE
:10C500004C51FDF7EBF904F5DB610448BDE8104040
:10C51000FDF7E4B968190020000001400044014023
:10C5200002494FF08040FDF7D9B900BFE01E00205E
:10C5300001490248FDF7D2B90C1F00200004004059
:10C5400001490248FDF7CAB9381F00200008004021
:10C5500001490248FDF7C2B9641F0020000C0040E9
:10C5600001490248FDF7BAB9E81F00200004014064
:10C5700010B5064C064804F5D061FDF7AFF904F29A
:10C580005C710448BDE81040FDF7A8B968190020A7
:10C5900000040140001C004001490248FDF79EB91B
:10C5A000142000200040014001490248FDF796B9DF
:10C5B0006C2000200048014001490248FDF78EB977
:10C5C000982000200018004001490248FDF786B974
:10C5D000F02000200020004010B50C2937D8DFE8FB
:10C5E00001F0973636366636363637363636070039
:10C5F000038C5488B2F80CE023F480531B041B0C0A
:10C600000384038CB0F804C0818B21F4E6414EEA28
:10C61000040E0904148823F40053090C41EA042190
:10C620001B04754C1B0C43EA0E33A0421FFA8CFC12
:10C630009BB289B200F0AE8004F58064A04200F0A5
:10C64000A9809268A0F804C081830264038410BDAD
:10C65000038CB2F80CC0548823F480731B041B0CA9
:10C660000384038CB0F804E0818B23F400731B0473
:10C670004CEA040C21F073011B0C43EA0C2309045F
:10C68000B2F800C0090C41EA0C0C5B4988421FFA61
:10C690008EFE9BB268D001F58061884264D09268BA
:10C6A000A0F804E0A0F81CC0C263038410BD038C92
:10C6B000B2F80CC0548823F010031B041B0C038435
:10C6C000038CB0F804E0018B23F020031B044CEA38
:10C6D000040C21F4E6411B0C43EA0C130904B2F8E4
:10C6E00000C0090C41EA0C211FFA81FC4249884232
:10C6F0001FFA8EFE9BB269D001F58061884265D039
:10C700009268A0F804E0A0F818C08263038410BD0A
:10C71000038C5488B2F80CE023F001031B041B0CBB
:10C720000384038CB0F804C0018B21F073014EEA3E
:10C73000040E0904148823F00203090C1B0421438E
:10C740002D4C1B0C43EA0E03A0421FFA8CFC9BB23B
:10C7500028D004F58064A04224D09268A0F804C0D8
:10C7600001834263038410BDD189548A23F400639A
:10C7700043EA0121138A2EF4405E23434EEA031E4E
:10C7800094884FF6FF330B4043EA04231FFA8EFED2
:10C790009BB284E7148A2CF4804C4CEA841C1FFA68
:10C7A0008CFC4EE7D489B2F810E023F00803234351
:10C7B000548A2CF4407C4EEA040E948823F004033F
:10C7C0004CEA0E0C1FFA8CFC2343C6E7D189548A2D
:10C7D00023F0800343EA0111138A2EF4406E2343B1
:10C7E0004EEA830E94884FF6BF730B4043EA04135E
:10C7F0001FFA8EFE9BB283E7000001402DE9F04F47
:10C80000A24BDFF8A49293F87A3EA14EA14F8FB0CD
:10C81000CDE90139013BDBB200930025DFF88CB292
:10C82000DFF88CA25B46D3469A464FEA9A23A3F5DB
:10C830008013522B4CD8334493F8F4330D2B47D844
:10C84000FC56019B012B40F00181012C35D14FF0AA
:10C8500000084146204611F041FD11F0CDFD03785E
:10C8600013B1542B40F0F98008F104081FFA88F83E
:10C87000B8F1100FEDD14FF0000E8DB349460020F6
:10C880000CE0334493F8F4330D2B0ED8FB56A3423F
:10C890000ED00130A84201F580711EDA8A68136853
:10C8A0009B0AA3F58013522BEBD90023A342F0D1AE
:10C8B00053799BF805209A42EBD1774B5B454BD0DF
:10C8C0005BF81CAF4FEA9A23A3F58013522BB2D921
:10C8D000009B012BF1D90024B9E7BEF1000FECD188
:10C8E0005846FBF771FDC3B2022B9BF805C000F25E
:10C8F0003483431C5BB203EB43034FEA830E644B68
:10C90000664903F5727004E0984200F0268353F8FC
:10C910002C1F5145F8D11A796245F5D153F80E40D4
:10C92000002CF1D05E4800234268A24203F10103CB
:10C9300000F08980102B00F12400F5D14FF0FF3377
:10C94000584A03EBC30302EB830393F86431002BD3
:10C95000B3D1029BC3F808B0029B013503F5807385
:10C96000042D02937FF45AAFDFF848B10BF59E73A4
:10C970000027ABF5816A9846DAF8243ABB425FDDBE
:10C98000DBF80C50002D5BD09BF81030A888029388
:10C990002B68DAF80460019303F13F41B0FA80F3A9
:10C9A00001F57E010393002EC3F11F034FEA91218D
:10C9B000009340F38480002302E00133B3427BD034
:10C9C0001C0259F804208A42F7D14C440099029B7A
:10C9D0008BF8103003260137CBF80410CBF80C503D
:10C9E000CBF81840AE71EF71636CE26C0D464900F4
:10C9F0008E401E43012303FA01F111439AF80020EF
:10CA00006664E1647AB303FA05F11A46236D0B43B9
:10CA10002365019B89B21883D4F8A000FBF710FDB1
:10CA20002046FBF763FE0123082F8BF81C308BF8A0
:10CA30001D3088F811300BF1200B08F118089BD13C
:10CA40000FB0BDE8F08FDBB2013B79E7022B7FF43A
:10CA5000FEAE082C3FF4FBAE2FE74FF0010E002D89
:10CA60007FF40CAF29E70399C1F12F05009903FA70
:10CA700005F58B4099B2236D2B432365019B5883A9
:10CA8000D4F8A000FBF7DCFCCAE700BF681900205F
:10CA900018D70508D855060810E905080000014018
:10CAA000D0020020880100200C000010000401408A
:10CAB00030E805080C040010032B00F31F820AEB7A
:10CAC0000623320218690492002800F03F82996020
:10CAD0000131CAB283F805210692542283F8042159
:10CAE0000136026805924479CAF80460FBF76CFCD1
:10CAF000934AC3B2022B92F891EE844600F22D8243
:10CB0000461C76B206EB46068E498F48059AB6005B
:10CB1000002305E00133172B00F01F8251F82C0F82
:10CB20008242F7D10879A042F4D188590028F1D087
:10CB30002C2101FB03F30CEB4C0C03EB8C0C814B15
:10CB400063441969049B5344C3E906017F4B0021E8
:10CB50001E461C466368984216D00131102904F124
:10CB60002404F7D17A4B93F84021002A00F0E781A2
:10CB70007849794A794BCAF8681ACAF8602ACAF81B
:10CB8000703A0FB0BDE8F08F01F1010C5FFA8CFC38
:10CB90006F4B07960CF1FF3C0CEBCC0C03EB8C0CB1
:10CBA0009CF864310593002BE2D1049E069B8CF81F
:10CBB0006531F31103EB262000EB001368488C2449
:10CBC00000EB83003112674B04FB01F103EB4101E1
:10CBD0000AEB0603C3E93C145421019E8CF864114E
:10CBE0003321C3F8AC10DE60C3F8A8005E4B049993
:10CBF0009A4209EB010400F07681534B9A4200F00F
:10CC0000728103F580439A4200F06D8103F58063E1
:10CC10009A4200F0688103F580639A4200F06381D4
:10CC2000474BD3F8B407BEF1060F4FEA500000F0AF
:10CC300061814E4B4E49BEF1070F18BF9C464D4BCC
:10CC400008BF8C464C4918BF1946B0FBF1F1B0FB48
:10CC5000FCFC1046049A01390AEB020389B20CF17C
:10CC6000FF3CA3F8B0C0A3F868104FF00006019392
:10CC7000A165002302F154014944A4F85C60636596
:10CC800047F0BAFC019B3D4A1B6901931868038871
:10CC90009BB243F080030380038809920A210B9121
:10CCA0004FF48072022123F00103CDE90C121B0422
:10CCB000ADF828601B0C019E0380717909AAFFF76B
:10CCC0008BFC3079002840F02281049B079E0AEB00
:10CCD000030200231069D2F818C001680A8892B2D2
:10CCE00042F001020A807268944503F1010300F0EA
:10CCF0000A81102B06F12406F5D14FF0FF33144AB8
:10CD00001F4E03EBC30302EB83031E4AD3F84831E3
:10CD1000B3420CBF4FF400134FF48003166B334340
:10CD20001363427918480C2A9BBF184B03EB42034C
:10CD30000026B3F81C61049B53449E8200232EE01E
:10CD40006819002018D7050800000140D002002013
:10CD500088010020B1730108AD730108B97301089F
:10CD6000FC2700202C2B00200004014044950800E3
:10CD700010552200D0DD060040771B006000010046
:10CD800000600240003802401406001010E8050858
:10CD9000914200F0E0800133042B00F0E18050F874
:10CDA0003320002AF4D1DAF80C260132CAF80C2616
:10CDB0000AEBC302DB00C2F8101603446A499A88E2
:10CDC000059816439E80049B0AEB03069022234697
:10CDD000FEF716F8B0690268002342F01002026004
:10CDE000C4E92533A367C4F88830C4F89C30F269DD
:10CDF00062664FF48062E26704214FF40032C4E9B6
:10CE0000232140222267D6F8AC206267F268049B97
:10CE10001832A2664FF48052C4F88020D6F8A820B9
:10CE2000E26603F164014FF480424944C4F884206F
:10CE300047F040FBB069049BD0F800E0C4F81CE068
:10CE4000D0F814E0C4F820E0D0F804E0C4F824E0FE
:10CE500003F1AC01D0F808E0C4F828E00023D0F8D2
:10CE60000CE0C4F82CE0C4E93733C4F8B830C4F897
:10CE7000C030C4F8D030C4F8E430F369C4F8AC3042
:10CE80004FF48063C4F8C4304FF4403C0423C4E939
:10CE900035C3D6F8F430C4F8BC30F3681033C4F8A6
:10CEA000B0304FF40063C4F8C830D6F8F030C4F89E
:10CEB000B4304FF48042C4F8CC20494447F0FAFA29
:10CEC000B369A8881A6822635A6962635A68A263C0
:10CED0009A68E263DA6822641A6842F010021A6003
:10CEE0002B68019372E5214BBEF1060FD3F8B4070E
:10CEF0007FF49FAEDFF87CC01D49A6E61B4A0323E2
:10CF000082F8903E34E6DBB20593013BF7E60DF084
:10CF100061F8069038B1019B0221DA79FEF798F9A1
:10CF2000069B5422DA80019B1A68B2F844306FEAFB
:10CF300043436FEA53439BB2A2F84430C5E6542200
:10CF400083F84021069A83F8412111E6074A02231B
:10CF500082F8903E0CE6DB002FE700235B68FFDEE3
:10CF600000239B88FFDE00BF898400086819002029
:10CF7000A0BB0D00882A11000C2911D8DFE801F0B0
:10CF80002310101019101010111010100700838BAF
:10CF900023F400631B041B0C43EA022292B2828337
:10CFA0007047838B23F008031B041B0C1A438283F6
:10CFB0007047038B23F400631B041B0C43EA02221B
:10CFC00092B202837047038B23F008031B041B0CEF
:10CFD0001A430283704700BF2DE9F04FDFF870B2AB
:10CFE0009BF8004087B024B90124204607B0BDE873
:10CFF000F08F934ED6F80C580DF0F6FE9BF8B43A2D
:10D000000390002B00F058828E4AA2FB05328E4B13
:10D010005209A3FB0213DB0803EB8303A2EB4303D8
:10D02000DAB204920BF23C6202EB830300930BF63C
:10D030001C1306F1E40401934FF00009924635E019
:10D040003B680293009B5C330093019B3046143392
:10D05000019347F099F97A4B02988C2202FB09332D
:10D06000002583F8D85079792A46FFF785FF2246B4
:10D070007979FFF7B1FA79790822FFF77DFF40232C
:10D0800044F83C3CA4F14801304647F013FA3368B9
:10D0900043F0100333609BF8B43A09F10109994554
:10D0A0000AF15C0A04F18C0480F2D480DBF8383693
:10D0B000039AD31A04D454F8082C9342C0F2AB81DB
:10D0C0005F4B54F8587C266A8C2202FB093393F894
:10D0D000D830002BB4D03968736834F8542C0291DE
:10D0E0001FFA83FE8B89CEF1160E9BB223EA020350
:10D0F000BEF1070F8B81A5D9DBF824390133CBF8BA
:10D100002439A36A05939C4600225CF8045B012144
:10D1100090461BE0DCF80000B8F1140FA0EB05030B
:10D120001DDC13F1080548BF03F117052B1108EBAF
:10D1300025180546581E013102FA03F301228240E8
:10D140008E4542EA03020CF1040C08D38E45E1D867
:10D15000C8F11503DCF800504FF01508EAE7B8F104
:10D16000150F60D13948C2F38423C2F3441100EB98
:10D17000830300EB8101D3F83831D1F838111B0259
:10D1800043EA011302F01F0100EB8101C2F3C43234
:10D1900000EB8202D1F83811D2F838210B4343EA70
:10D1A000023383EA132282EA121202F00F020F2ADC
:10D1B00039D1C3F30F134FF6FF72934233D0B3F557
:10D1C000606F00F03681019A93819AF85820049D8F
:10D1D000AA4211D00098DAF800208168521ACAF8E1
:10D1E0000020016BDAF80420521ACAF80420002249
:10D1F000826002638AF85850DAF800200099013200
:10D20000CAF800208A6801328A604FF6FF729342A2
:10D210007FF418AFDAF804300133CAF804300B6B2E
:10D2200001330B630EE7DBF820390133CBF82039EB
:10D23000B9F1000F00F0E5804FF6FF73C5E700BFBE
:10D24000681900201F85EB51CDCCCCCC10E8050827
:10D250000400001001228BF8202ACBF83856002B4E
:10D260003FF4C2AE974890F89410890700F1BE8051
:10D27000D0F88C10086849798A40018C92B289B242
:10D2800021EA02010184018C89B20A43012B028444
:10D290003FF4AAAE8B4991F82021970700F1C08096
:10D2A000D1F8182110685479018C012289B2A2406A
:10D2B00092B221EA02010184018C89B20A43022B55
:10D2C00002843FF491AE7F4991F8AC21960700F1BA
:10D2D000C180D1F8A42110685479018C012289B24F
:10D2E000A24092B221EA02010184018C89B20A4370
:10D2F000032B02843FF478AE724991F838229507E7
:10D3000000F1B180D1F8302210685479018C0122EB
:10D3100089B2A24092B221EA02010184018C89B251
:10D320000A43042B02843FF45FAE664991F8C4229D
:10D33000940700F1A180D1F8BC2210685479018CC7
:10D34000012289B2A24092B221EA02010184018C39
:10D3500089B20A43052B02843FF446AE594991F83D
:10D360005023900700F19180D1F848231068547938
:10D37000018C012289B2A24092B221EA0201018409
:10D38000018C89B20A43062B02843FF42DAE4D492D
:10D3900091F8DC23920700F18180D1F8D423106842
:10D3A0005479018C012289B2A24092B221EA020191
:10D3B0000184018C89B20A43082B02847FF414AEE5
:10D3C000404A92F868349B0771D5D2F86024042350
:10D3D000116850790A8C83409BB292B222EA030210
:10D3E0000A840A8C92B213430B84FDE5354AD2F8C5
:10D3F0008C2010685479018C0422A24089B292B228
:10D400003EE705993048582250F0BEF83B68029339
:10D410004FF6FF73D9E60024204607B0BDE8F08F31
:10D42000284AD2F8182110685479018C042289B254
:10D430003DE7244991F8E52402EB420201EBC202E8
:10D440004A4492F8F5240D2A7FF4BDAE019980225A
:10D450008A77BAE61B4AD2F8A42110685479018C65
:10D46000042289B23CE7174AD2F830221068547976
:10D47000018C042289B24CE7124AD2F8BC2210680F
:10D480005479018C042289B25CE70E4AD2F8482311
:10D4900010685479018C042289B26CE7094AD2F8E9
:10D4A000D42310685479018C042289B27CE7054B9F
:10D4B000D3F8602401238BE701228BF8202ACBF8D4
:10D4C000383692E568190020CC0900102DE9F04F9C
:10D4D000002299B02F21074610F0E4FF00B3BE4EA2
:10D4E000D0F80080C6F8448E0446FDF78DFB024656
:10D4F000B0B1D0F804C0C6F840CEBCF1000F0FD0D8
:10D50000B64D002329464868844501F1240103F102
:10D5100001030FD0102BF6D1B14B93F8400118B195
:10D52000002019B0BDE8F08F2F2283F8402183F846
:10D530004101F6E7DBB2DFF8A892013B03EBC3033E
:10D5400009EB830393F864A1BAF1000FE8D13846E0
:10D550009768DFF8C0B22F22A3F864210CF03AFDDF
:10D560002F220346CBF8300520B1DA80E2792A2158
:10D57000FDF76EFE9B4A9C49002301E051F83320E1
:10D58000904500F0228101330E2BF7D100204BF0A3
:10D59000E9FCD6F8440E954A038823F001031B04E6
:10D5A0001B0C9042038000F070818E4B984216D085
:10D5B00003F58043984212D003F5806398420ED061
:10D5C00003F580639842D6F8B4270AD08849B1EBB6
:10D5D000520F4FEA520340F2528100210AE0D6F87E
:10D5E000B427834B9A4280F017814FF0010C002141
:10D5F000B2FBFCF37F4AADF804101B0A7E49A2FB84
:10D6000003231A09A1FB021252084FF000081B095C
:10D61000ABF82E2501A952000293ABF82C25ADF8EA
:10D620000C80ADF806808DF80E8046F0E5FFCDE960
:10D630000688CDF82080A379ADF81480602204928A
:10D640009A0740F1AF80DB0003F00803ADF81E300D
:10D650000423ADF81430D6F8440E617904AAFEF71D
:10D66000BBFF61790822FFF787FCB0F84430D6F899
:10D67000408E6FEA43436FEA53439BB2A0F84430B5
:10D6800003889BB243F080030380A3796179028C05
:10D690009B074CBF042301238B409BB292B222EA2A
:10D6A00003020284028C92B21343038403889BB268
:10D6B00043F0010303802A4600235168884502F1A4
:10D6C000240203F101037DD0102BF6D14FF0FF337C
:10D6D00003EBC30309EB8309484AD9F848314849A9
:10D6E0008B420CBF4FF400134FF48003116B0B43BC
:10D6F000136300236A68904505F1240503F10103D3
:10D700005DD0102BF6D13F49602200235046FDF733
:10D7100077FB404646F038FED6F8400E036823F00B
:10D7200001030025036046F02FFECDE91455CDE935
:10D730001655D6F8443E0E9512956279D6F8400EED
:10D74000099734331344304A0B9240220A930C92C7
:10D750004FF480434FF48052CDE9102340F22A4128
:10D760004FF440330D91139309A94FF480630F9345
:10D7700046F0A0FE6379D6F8441E0C2B04D8234A49
:10D7800002EB4303B3F81C518B89D6F8402E9BB2B1
:10D790001D438D811368012043F01003136019B0FD
:10D7A000BDE8F08F5B0003F00203ADF81C300123ED
:10D7B000ADF812304FF48073ADF820304BE75FFACC
:10D7C00083FAA0E7DBB2013B82E7114A02EBC30315
:10D7D00093F84C0DDBE600BF68190020D002002052
:10D7E000880100200000014060E4050800040140B9
:10D7F000006CDC02598B4F01ABAAAAAA0038024088
:10D8000000600240418700088889002010E8050870
:10D8100018D70508602A0020254B98420BD003F545
:10D820008043984207D003F58063984203D003F504
:10D830008063984222D102F1B7731E4903F5585311
:10D84000A1FB03139B0D013B99B2194B984201F1C7
:10D85000010C3FF4CDAE03F5804398423FF4C8AECF
:10D8600003F5806398423FF4C3AE03F580639842AA
:10D870003FF4BEAE5308B3FBFCF3BBE6530803F121
:10D88000B7730C4903F55853DAE7D6F8B4270A4BB7
:10D890009A42FFF4AAAE074902F1B77303F5585351
:10D8A000A1FB03139B0D013B99B201F1010C9FE613
:10D8B00000000140819F5E16006CDC02F0B50C4652
:10D8C00089B03C49BDF838609DF83C70013B054685
:10D8D00020689BB2049388424FF00003ADF81430E7
:10D8E000ADF80E308DF8163013D0334B984210D06F
:10D8F00003F5804398420CD003F58063984208D02A
:10D9000003F58063984204D02C4BD3F8B4375B08FE
:10D9100002E02A4BD3F8B437B3FBF2F203A9013A81
:10D92000ADF80C2046F068FE20686179A3790FB14C
:10D9300083F001030022CDE90622ADF81020602219
:10D9400003929A0729D5DB0003F00803ADF81A30DB
:10D950000423ADF8103003AA01910596FEF73CFEB2
:10D9600001990822FFF708FB2268B2F844306FEAF9
:10D9700043436FEA53439BB2A2F8443013881146E5
:10D980009BB243F0010321F8343B63796A60C81805
:10D9900000222860CA5009B0F0BD5B0003F002030A
:10D9A000ADF818300123ADF80E304FF48073ADF8A8
:10D9B0001C30D0E70004014000000140681900203D
:10D9C00070B5384C94F83C5584B00DB904B070BDB6
:10D9D00094F83D3584F85C3528460CF0FBFAC4F821
:10D9E0004C0508B13823C38094F834656EB3012E1A
:10D9F000ECD13146FDF706FB94F85C35002B49D19C
:10DA0000D4F84C3513B11A689B881383264D4FF414
:10DA1000E072D5F8B831C4F8582503A8012284F87B
:10DA20004825039346F09AFCD5F8BC31029302A82E
:10DA300046F094FC1D491E4C0B6C1E48002243F01E
:10DA400030030B6422850285C0E728463246382120
:10DA500010F028FD05460028B8D0C279D4F84C054E
:10DA60000221FDF73BFC144A94F85C35D2F8B42748
:10DA7000124801935208802329460096FFF71EFFA3
:10DA8000D4F8501580230122C4F858350B6084F86F
:10DA900048259BE7D4F84C35002BB7D01A689B88F3
:10DAA0005383B3E7602A002010E8050800380240DD
:10DAB000001000400014004068190020B02F002022
:10DAC0000B4B93F85C25D3F84C353AB113B11A6877
:10DAD0009B885383074B00221A827047002BF9D092
:10DAE0001A689B881383034B00221A82704700BF79
:10DAF000602A0020001000400B4B93F85C25D3F8FF
:10DB00004C353AB113B11A689B881383074B002236
:10DB10001A827047002BF9D01A689B885383034BF5
:10DB200000221A82704700BF602A002000140040C3
:10DB30002DE9F0415C4CDFED5D7AB4F83635DFED70
:10DB40005C6A94F8345504EB400007EE103AB0F8E4
:10DB50003E35B4F83A056422B8EEC77A02FB03F307
:10DB600027EE277A07EE903AF8EEE77A02FB0033C9
:10DB700027EE277A07EE903AF8EEE77A002687EE4E
:10DB8000270A0F46C4F8606520EE260A55B3012D1A
:10DB900001D0BDE8F081D4F8588507EE908AF8EE00
:10DBA000677A27EE800A4EF077FF002832D194F88A
:10DBB0005C35002B66D0D4F84C3513B11A689B88BD
:10DBC0001383B4F8380538440FF080FF94F85C35BF
:10DBD000002B5FD0D4F84C35002BDAD01A689B8824
:10DBE0005383D6E7D4F8583507EE903AF8EE677AC3
:10DBF00027EE800A4EF050FFD4F850252D4B1060D0
:10DC0000D3F80C38B4F8381519443944C4F86415FD
:10DC1000BDE8F081284A294B5062C2F82C805E6230
:10DC2000C3F82C80EFF31181502080F31288158007
:10DC3000C9B21D8081F3118895811E4A9D81D2F859
:10DC40000C38B4F8381519443944D2F80C389942D4
:10DC5000FBD81949194A0B88D4F84C0523F0010365
:10DC60001B041B0C0B80138823F001031B040024EE
:10DC70001B0C13808C81948100288AD003688288D1
:10DC80001A8386E7D4F84C35002B9AD01A689B8803
:10DC9000538396E7D4F84C35002B3FF47AAF1A68DB
:10DCA0009B88138375E700BF602A00200AD7233CB6
:10DCB000CA269B3E68190020001000400014004056
:10DCC000034B93F8482512B1042800D830E7704779
:10DCD000602A00201648174A174938B5174C184DC6
:10DCE000121A4FF051FCD4F88820164B164842F413
:10DCF0007002C4F888201A68002142F001021A60FC
:10DD000099601A6822F0847222F480321A60586096
:10DD10001A6822F480221A600C4AD960521B2846E5
:10DD20000B494FF031FCA560BDE83840FAF76EBEF4
:10DD300000000010040000107F07070800ED00E05D
:10DD4000000000200038024010300024880100202C
:10DD5000000000080548D0F8C83723B1DB6A13B1CA
:10DD600000F5F96018470248704700BF68190020A5
:10DD7000D0E9050838B5184CD4F868351B8843B984
:10DD8000164D002384F8743585F8C037C5F8BC37C4
:10DD900038BDD4F86C25002AF2DD012A09D0D4F868
:10DDA000703559880D4DA4F87615012384F878351F
:10DDB000E7E7D4F870158A8849880132521A9A42E6
:10DDC000F0D1064DD5F8C83700221B69C5F8F427F5
:10DDD00005F5F9609847D4E7602A0020681900200B
:10DDE0000748D0F8C4371BB1064B93F878350BB110
:10DDF00000207047D0F8C83700F5F9605B68184715
:10DE000068190020602A002030B4154A154D92F898
:10DE1000C03705F27C542344036095F874354460A0
:10DE200092F8C007834292F8C00712D8834204D305
:10DE3000002030BCC1E90000704792F8C027002BD9
:10DE4000C2F180020CBF0120022030BCC1E90023D6
:10DE500070471B1A0022012030BCC1E90032704714
:10DE600068190020602A00200E4B0F4A93F8C01753
:10DE700092F8740593F8C027904293F8C0270CD805
:10DE8000904238BF93F8C027D3F8BC373ABFC2F1ED
:10DE900080028018002018447047D3F8BC37801ADD
:10DEA0001844704768190020602A002030B51C4CC7
:10DEB0001C4D94F8C03794F8C01785B005F27C5219
:10DEC0001344029395F8743503928B421DD894F84D
:10DED000C027934211D294F8C0170193C1F1800179
:10DEE0000091D3B9012208B93F2906D90023694618
:10DEF00002A84DF06BF895F8743594F8C007C01A75
:10DF0000B0FA80F0400905B030BD94F8C017002287
:10DF1000591A019200910122E5E719440222E2E731
:10DF200068190020602A00202DE9F043164685B0CC
:10DF3000002936D0441E254D254F04EB01084FF033
:10DF4000000901E0A0452CD095F8740514F8013FB4
:10DF5000411C2844C9B280F87C350B0648BF00201C
:10DF600097F8C03785F874154ABF0146084685F80A
:10DF700074958B4297F8C0378ABFC3F18003C01AEB
:10DF8000C0183F28DED997F8C0378B42DAD0114B42
:10DF900093F8C430002BD5D00020FFF787FFA045B1
:10DFA000D2D1694602A8FFF72FFF20B1DDE9003288
:10DFB00013443F2B02D805B0BDE8F0830246334638
:10DFC00002A84DF003F805B0BDE8F083602A0020F8
:10DFD000681900208801002030B585B0694602A884
:10DFE000FFF712FF58B9094C04F5F965D4F8C837A2
:10DFF00028465B6898470028F8D005B030BD024637
:10E00000012302A84CF0E2FFEDE700BF68190020F1
:10E0100070B5124E1546D6F8C4370A4641199942D2
:10E020000F4988BF1D1A91F8741596F8C0379942A8
:10E0300082B0044603D00192FFF7CEFF019AD6F8D2
:10E04000C81708480023C6F8F4372B468D6A2146C6
:10E05000AC4602B0BDE87040604700BF68190020C0
:10E06000602A0020302100208C461346014662467B
:10E070001846CDE738B52448244C0023C4F8C437EB
:10E0800002461178022902F106022CD00133062B38
:10E09000F7D11F4DD4F8C8370022C5F87025F3B169
:10E0A000DA6AE2B11B489047D5F87035C5F86805C3
:10E0B000A3B19A885B88D21A436802FB0333C4F881
:10E0C000C437FAF709FE95F8742594F8C0379A42D8
:10E0D000054601D0FFF780FFC4F8BC5738BD0E4B92
:10E0E000C5F8683538BD0A4DD4F8C82703EB43039B
:10E0F00000EB4303C5F8703512B1D26A002AD1D1C2
:10E100000548C5F86805D4E75C3000206819002090
:10E11000602A002030210020D0E905082DE9F04FC9
:10E1200041F694628BB00021BD484FF090FA042074
:10E1300046F052FA0446052046F04EFA50EA04032F
:10E1400040F05C81B74B03934C220021B4484FF060
:10E150007EFA4C220021B2484FF079FA039BB04975
:10E16000D3F8CC33B04A0A600124C1E907334B62CB
:10E170000C714BF0A9FFFFF77DFF002108460BF063
:10E18000B9FFFAF7A9FDB0F1000B40F30881A74BE6
:10E19000A74D0193A24BA74E0024029403F14C0912
:10E1A0002746A04605F5C46A04E008F50068C345A3
:10E1B00040F3AE80019AD2F80C38C2F81038FAF762
:10E1C000BDFD202251464046FFF722FF9A49122208
:10E1D00050464FF079FA0028E7D1B84522D002998D
:10E1E000964BCDF8149001EB410203EB82004A1CE0
:10E1F00093490292049001F075FDDDE90403D9F81A
:10E200001C2043F84C0BC9E908228E4AC9F80C704F
:10E21000C9F82820A8EB07070122C9E90477C9F843
:10E2200008209946039BD3F8CC33C9F81C304746E5
:10E230001222A918335D91F82016994202F10102C9
:10E240000BD00024202AF4D12037BB455146384654
:10E2500054DBFFF7DDFE0022EBE70134152CF1D192
:10E26000D01979492022FFF7D3FE00230A2209A9F9
:10E270007548CDF824A001F0E3FE0490099800232E
:10E2800001300A2209A9099001F0DAFE07900998E5
:10E29000002301300A2209A9099001F0D1FE06905D
:10E2A0000998002301300A2209A9099001F0C8FE4B
:10E2B0000590099809A9013000230A22099001F06C
:10E2C000BFFE074609980023013019460A2209902B
:10E2D00001F0B6FE049989B1DDE9063243EA421243
:10E2E000059B7F0147EAC323A1F2BC7143EA6003A7
:10E2F00042EA412243EA0243C9F81C30029B642BE4
:10E3000000F0EC80474608F50068C3453FF752AF80
:10E31000029A642A00F0E280B84500F0E380474C9E
:10E320004749484E0C2303FB0244531C1A4620461F
:10E33000A8EB0705029301F0D5FCD9F81C30C9F809
:10E340000040C9E90375C9E908330123C9F814502D
:10E35000C9F82860C9F80830029B5D1C4C22304F78
:10E3600002FB05F57B19002118464FF070F94C228D
:10E3700000214FF06CF9039A3449D2F8CC2379513B
:10E38000029C4262C0E904BBC0E9072201220234B8
:10E39000866282604FEA4B03B3F1805F1EDA4C2243
:10E3A0001F4D02FB04F42B19184600214FF04FF9C2
:10E3B0004C2200214FF04BF90399CBF10062D1F8C8
:10E3C000CC130346520022482851C3E90422C3E972
:10E3D000071102225A71012259629A60104A956807
:10E3E0002DB913791BB11368002B40F089800021EF
:10E3F00008460BB0BDE8F04F0BF07CBE4FF47A72CC
:10E40000002321464DF0F8FA124B40F26D11A3FBA8
:10E4100000231B0C022440F2B2720D4625E000BF1F
:10E42000006500208801002064E2060868190020C9
:10E43000602A00207C55060858550608A0300020A8
:10E440006C55060869E000088030002094550608E5
:10E45000A455060807452EC2013212F00304A3EBAF
:10E4600001030CBF4FF4B77129469942F4DD7A4994
:10E47000002C3FD003910399D1F89C138B4272DB9F
:10E48000764D01245B1A55F8041F994204F10104EA
:10E49000F8DD013343EA4413A2F2BC7243EA42239B
:10E4A0006F4A039DB0FBF2F102FB11024FF4616071
:10E4B0003C24B2FBF0F100FB11221C20C5F8A003A4
:10E4C000B2FBF4F004FB1022521042EA401242EA7E
:10E4D000C12242EA0343C5F8CC3335E66423614EDA
:10E4E000029339E7029B01245D1C002B3FF452AFDD
:10E4F0005C4E33E70C4603911D21C4F8A013BAE724
:10E50000C2E911551564D56329462E46D46C02F133
:10E510004C0354B39C681E64481E8442C3E91166D0
:10E52000DE6312D0481C844216D08C427FF45FAF69
:10E53000084600283FF45BAF116CCC6B0134CC6310
:10E540001964936401461A46E0E700293FF44FAF8F
:10E55000884253F80C2CECD1117900293FF447AFD5
:10E5600053641A64EEE7012493E73F4902222646EA
:10E5700013E0CB6B0A635B011DBF03F6FF7702F16B
:10E58000FF3303EB17331346C1E90466C1E90D33CA
:10E5900051F84C0F5A1C0135C8B10B79002BE8D14A
:10E5A0000F690A63002F4AD14F691046531E486312
:10E5B000002F4DD007F6FF7703EB1733201A8B633C
:10E5C000C41851F84C0F5A1C01350028E5D12749D1
:10E5D0002748C1F85C583E220D46C1F838283F2232
:10E5E000013BC1F83C284022C1F840280191C1F804
:10E5F0004C38C1F850489A00990FC5F834084BB30D
:10E6000040F2FF10121841F10001520A42EAC152D1
:10E61000019C02F140010A4402EBC303C4F84828FC
:10E62000C4F84418134A1049C4F85418C4F85818C8
:10E630005802D90D42E90201C4F83038D7E607F68E
:10E64000FF77531E03EB17304F694863002FB1D19A
:10E650001346B3E70122DBE78801002024050020F0
:10E660008051010069E00008006500206819002061
:10E67000B05506089821002010B50A4CD4F8C837C8
:10E680005B6A13B104F5F9609847074AD4F8BC37C0
:10E69000D2F868255288013B134452421340C4F813
:10E6A000BC3710BD68190020602A00202DE9F04316
:10E6B000DFF8E890374F93B0FFF75CFBFFF7DAFC29
:10E6C00099F8C03797F874259A4201D0FFF784FC77
:10E6D000D9F8C4870025C9F8BC57B8F1000F11D08C
:10E6E0002D4E6C462A463146204601F0FBFA204664
:10E6F0004CF0BEFC2035014601222046FFF714FCF9
:10E70000A845EFD899F8C03797F874259A4201D0F8
:10E71000FFF762FCD7F868359B7B012B33D099F863
:10E72000C03797F874259A4201D0FFF755FC0027AF
:10E73000C9F8BC77B8F1000F28D0DFF85C903D46EF
:10E740006C462A46494609A801F0CCFA212200214C
:10E7500020464EF07CFF202221462846FFF758FC39
:10E760002022064609A9204615444EF0ADFF08B9FF
:10E77000202E00D00137A845E3D8B7FA87F040092A
:10E7800013B0BDE8F083FFF777FFC8E7012013B0AF
:10E79000BDE8F083602A0020B855060868190020FB
:10E7A000032108B50546084645F006FF72B6114B31
:10E7B000D3F8F02AD3F8F43A52EA03010AD100243C
:10E7C0002146042045F0F8FE2146052045F0F4FEE0
:10E7D000FDF71AFC0848D0F80C4829B24EF6602024
:10E7E00000FB01F1A41843F100030C1943EBE171A4
:10E7F000E7E700BF602A002068190020084B09499C
:10E800008B4202460AD2184602E01C30884205D2EA
:10E810000388C3F30B039A42F7D170470020704777
:10E820009CE4060894ED06088388C3F30B03934227
:10E83000A8BF134670B51A461D460C4606468068AA
:10E840004EF0A2FE62199442B569074B08D0074802
:10E8500014F8011B00FB03F3A24283EA0103F7D182
:10E860002B60012070BD00BFC59D1C81930100017C
:10E870000023037043708370C370704700230370DC
:10E8800043708370C370704700220123027042708E
:10E890008270C270037143718371C371704700BF8E
:10E8A000FF23037043708370C370704700230621F9
:10E8B0004FF47A72C0E9012301700373704700BFFF
:10E8C00010B50023411CFF2200F8132001F813208B
:10E8D00001330B2BF8D10B4B4FF0FF3103F10F0439
:10E8E00000228C4605E093F904C093F9051013F853
:10E8F000032F00F812C000EB420E9C428EF801106C
:10E90000F1D110BD64F305084FF0110C00B580F88B
:10E9100000C04FF0100C80F803C04FF0120C002222
:10E92000022180F806C04FF0130C0123827042715F
:10E93000C171027280F809C04FF0180E4FF0FF0C41
:10E940008172C174C2724F2137224370037180F803
:10E950000CE043738373C173037480F811C0827435
:10E9600080F814C05DF804FB03230370704700BFF8
:10E970000A44914219D000B501F1FF3C02F1FF3E7B
:10E9800041F221011CF8012F082380EA022010F433
:10E99000004F81EA40020ABF400090B280B2013BC2
:10E9A000F5D1E645EED15DF804FB7047704700BF36
:10E9B000D0ED007AD0ED016A30EE677AE6EE877A24
:10E9C000B0EE670AC0ED007A704700BFD0ED017A63
:10E9D000D0ED026A30EE677A90ED000AE6EE877AB3
:10E9E00037EEC07AC0ED017AA6EE870A80ED000A04
:10E9F000704700BF90ED017AD0ED036AD0ED027A46
:10EA000030EE470AA6EE807A90ED000A80ED017A9A
:10EA100037EE676AE6EE867A37EEC07AC0ED027AA4
:10EA2000A6EE870A80ED000A704700BFDFED277A67
:10EA3000B4EEE70AF1EE10FA0CDDDFED256A9FED8A
:10EA4000257AF0EE407AF4EEC77AF1EE10FA30EE65
:10EA5000660AF6DCDFED207AB4EEE70AF1EE10FA92
:10EA60000CD5DFED1B6A9FED1D7AF0EE407AF4EED7
:10EA7000C77AF1EE10FA30EE260AF6D4DFED187AF6
:10EA8000B4EEE70AF1EE10FA14DDDFED107A37EE9E
:10EA9000C00A60EE006A9FED136A9FED137ADFED06
:10EAA000137AA6EE867A20EE266AE6EE877AA6EE3E
:10EAB000270A7047DFED0E7AB4EEE70AF1EE10FA9E
:10EAC00044BFDFED057A37EEC00AE2E7DB0F4940CD
:10EAD000DB0FC940E4CB1641DB0F49C0E4CB16C1C4
:10EAE000DB0FC93F92E741B99730083C15A82ABE11
:10EAF000DB0FC9BFD0ED056AD0ED017A90ED007A49
:10EB000090ED066AD0ED025A90ED035A80ED050AA9
:10EB100066EEA77AC0ED066AE7EE007A90ED077A16
:10EB2000E5EE867A90ED086AD0ED045A80ED087A19
:10EB3000E5EE477AE5EEC67AB0EE670AC0ED077AF1
:10EB4000704700BFD0ED057A90ED006A90ED067A2F
:10EB5000D0ED035AE6EE007A90ED016AF0EE406ADD
:10EB6000A6EE267AB0EE670AD0ED047A90ED026A3E
:10EB700067EEC07AA5EEC07AE6EE267A80ED057AD9
:10EB8000C0ED067A704700BF2DE9F047089F3C466C
:10EB90000E4614F8011B002B054614BF4FF0300938
:10EBA0004FF0200941B3002A2CDD234600E0B2B12A
:10EBB00013F8010B9046013A0028F8D1A8F1020899
:10EBC0006AB1C24649462846B0475346002B0AF16F
:10EBD000FF3AF7DC397828EAE872013249B1D71BED
:10EBE0002846B047E01914F8011B0029F8D1BDE808
:10EBF000F0871046BDE8F087002A02F1FF38E0DC1C
:10EC00000846F4E70022EAE703685A1C026019701C
:10EC1000704700BF024B186803681B68184700BFA5
:10EC2000309A0020884210B54FF001043ED301FB1A
:10EC300004F4B0FBF4FC8C45F9D2CCB122BB08E063
:10EC4000A14203F801EBB4FBF1F211D8B0FBF2FCE6
:10EC50001446BCF1090F0CF1570E0CF1300204FB05
:10EC60001C00EDDCA14203F8012BB4FBF1F2EDD95D
:10EC700000221A7010BDA14203F801EBB4FBF1F2BF
:10EC8000F6D8B0FBF2FC1446BCF1090F0CF1370EBC
:10EC90000CF1300204FB1C00EDDCA14203F8012B57
:10ECA000B4FBF1F2EDD900221A7010BD8446002A9F
:10ECB000EAD1CEE70028BEBF2D23404201F8013B38
:10ECC000092870B54FF00103864607DD03EB830387
:10ECD0005B00B0FBF3F2092AF8D8EBB1104CBEFB95
:10ECE000F3FCA4FB0320C008BCF1090F0CF13006B3
:10ECF0000CF15705024607D8092B01F8016B03FBFD
:10ED00001CEE09D90346EAE7092B01F8015B03FB76
:10ED10001CEE01D91346E2E700230B7070BD00BF63
:10ED2000CDCCCCCC0378202B024600F10100F9D0E9
:10ED3000092BF7D02D2B28D02B2B03BF5378B7EE00
:10ED4000000A0246B7EE000AA3F13001C8B2092852
:10ED50009FED567A10D8F2EE046A07EE901AF8EE9C
:10ED6000E77A12F8013FE7EE267AA3F13001C8B244
:10ED70000928B0EE677AF0D92E2B5ED003F0DF03BE
:10ED8000452B07D020EE070A70475378BFEE000AE4
:10ED90000246D9E710B451782D2978D02B296AD0B2
:10EDA000A1F13003092B02F101026BD800240023EA
:10EDB00003EB830301EB430312F8011FA1F13000C1
:10EDC0000928A3F13003F3D9B3F59A7F1A4628BF77
:10EDD0004FF49A72072B66D9DFED356A1346F7EECA
:10EDE000007A083B072B67EEA67AFAD802F00702F2
:10EDF000DAB1F2EE046A012A67EEA67A15D0022A89
:10EE000067EEA67A11D0032A67EEA67A0DD0042AFF
:10EE100067EEA67A09D0053A67EEA67A05D067EEC6
:10EE2000A67A012A18BF67EEA67A6CB387EE277A16
:10EE30005DF8044B20EE070A70475378A3F13001C8
:10EE4000C8B2092802F1010298D8F2EE046AF0EE85
:10EE5000665A07EE901AF8EEE77A12F8013F87EE4D
:10EE6000A66AA3F13001C8B2092866EEA56A37EE9A
:10EE7000067AEED982E79178A1F13003092B02F1ED
:10EE8000020293D9F7EE007A27EE277AD0E791783D
:10EE9000A1F13003092B02F1020288BFF7EE007ADC
:10EEA000C4D8012483E7F7EE007AA1E70000000050
:10EEB00020BCBE4CF0B5067906F0E003402B03D130
:10EEC00045794FF0FF3406E0602B4FF00105F8D193
:10EED000447905FA04F40023012006F00706AB424A
:10EEE00000D1F0BD052E0FD8DFE806F00308101D95
:10EEF000242448B1C85CD75C78400FE020B1C856E4
:10EF0000D756C71B784278410133E8E70028FBD089
:10EF100031F8130032F81370784080B220420CBFF1
:10EF200001200020F0E70028EED031F9130032F97B
:10EF30001370E6E70028E7D051F8230052F8237059
:10EF4000DAE7037903F01803102B1CD004D82BB197
:10EF5000082B06D000207047182BFBD1B0F80B000F
:10EF60007047104BB0F80B0093F90030591C06BFE6
:10EF70000D4B1B78DBB203EB830203EBC20300EB08
:10EF8000830080B27047074BB0F80B0093F9013053
:10EF90005A1C06BF044B5B78DBB2C3EB031300EBD8
:10EFA0004300EEE7940500206C35002070B505465F
:10EFB000B0F80900FFF722FC054B1E7904462846ED
:10EFC000FFF7BFFF16B1E368184470BDA368FBE705
:10EFD000309A002038B505460C46FFF7E7FF2B793D
:10EFE00003F0E002602A03F007032AD1052B0CD8B6
:10EFF000DFE803F0030B0F0B1B1B6A79012393401F
:10F00000DBB2027814B11343037038BD22EA030364
:10F01000FAE76A79012393409BB2028814B1134343
:10F020000380F2E722EA0303FAE76A79012303FA8D
:10F0300002F2036814B113430360E6E723EA020314
:10F04000FAE7052BE1D8DFE803F00303050507071E
:10F050000470DAE70480D8E70460D6E7092900D015
:10F0600001B9704701394B0003F00802930001F029
:10F070000301A3EB9203C1EB0111C3EB0313C1EB3B
:10F08000011100229B00890002608180438070474B
:10F0900010B50021382204464EF0D9FA0D490E4A27
:10F0A0000E482061C4E905120D480E4AE0610123B3
:10F0B00041F61E614FF0090CE18484F808C0A37387
:10F0C00084F82130A26221460748BDE8104030F0A4
:10F0D000C7BB00BF1A046C07001975036400DC0588
:10F0E00043080E001E7D0101EC550608B5EEC00A6E
:10F0F000DFED337AF1EE10FACCBF30EE270A30EEB6
:10F10000670ADFED307A20EE270A70B5FDEEC07A8F
:10F1100086B017EE904A054684EAE470002303A9FE
:10F12000A0EBE470CDE90033029346F0D9FD002C4A
:10F13000ACBF20232D2303A88DF800304BF098FF9F
:10F1400001286E4626D0022830D0032803BF302382
:10F1500003A9304603A914BF30468DF801304EF0A4
:10F160007EFA30464BF084FF0338C4B22246314663
:10F1700028464EF009FA00232B5528464BF078FF1D
:10F180002E232B540130311928444EF084FA28469E
:10F1900006B070BD43F23002302303A93046ADF80B
:10F1A00001208DF803304EF05AFADAE743F23003CB
:10F1B00003A93046ADF801304EF051FAD1E700BF57
:10F1C0006F12033A00007A440AF0AEB913B568B181
:10F1D0004C1E14F8011F21B902B0BDE810400AF01E
:10F1E000B7B901900AF0A0F90198F2E702B010BD9A
:10F1F00008B520214EF042FA034620B11A78202AA1
:10F2000000F10100F8D0184608BDF8B5B8B10E4BB2
:10F210000138C70003EBC000CA43067B457B02F000
:10F22000010282EA0604A54209D0806828B18588D7
:10F230000068B24214BF058345833B445C73CB072F
:10F2400001D4FCF72FFFF8BD309A00202DE9F341DF
:10F25000124D134F002305F8283F044600EB8106AA
:10F26000B44203D10F4802B0BDE8F08139462846C8
:10F270004EF0F5F9214668464EF00DFA4FF00008C1
:10F28000202168464EF0FAF928B9694628464EF022
:10F29000E6F90434E4E780F80080F1E7309A0020D2
:10F2A00080AD0608589A0020014BD86C3BF0E6B9B7
:10F2B000309A00202DE9FF471E46C368BDF8307024
:10F2C000DDF8348004468946924643B3CBB20D2B19
:10F2D0009ABF1A4AD5560025BAF1FF3F21D02368BC
:10F2E000174A3146CDE9005A3846C0475246207980
:10F2F0005FFA89F1FBF714FC024600B10288D3B231
:10F300000393C2F30323120BCDE9005202930D4A7B
:10F31000236831463846C04704B0BDE8F0874D1C2D
:10F32000DAE77B06F8D42368074A0C95314638465D
:10F33000C44604B0BDE8F047604700BFD855060892
:10F34000849B0608919B0608B59B06082DE9F041B1
:10F35000154686B06A1C8846BDF830600D9F194678
:10F3600023D0030900F00F044033CDE90045164ACD
:10F3700005933046B847A8B198F80510D8F80000B2
:10F380002A46FBF715FC68B1028801780391C2F3A5
:10F390000321120BCDE900420291059B0B4A00218B
:10F3A0003046B84706B0BDE8F0817306FAD40309C9
:10F3B000074A00F00F000C9040333046BC4606B0C0
:10F3C000BDE8F041604700BFC49B0608D69B060815
:10F3D000FF9B06082DE9F04188B01E4603090E9FE9
:10F3E0009046403300F00F0451B307930EF014FF22
:10F3F000C279079BCDE900420546164A4146304690
:10F40000B847D0B12868FBF78FFDA9796A79DFF892
:10F4100054C0ED79079B009411F0020F4FEA92025D
:10F420000D4902F1010208BF6146CDE90102CDE9B3
:10F4300003150A4A00213046B84708B0BDE8F081FC
:10F44000074A0E9441463046BC4608B0BDE8F0413C
:10F45000604700BF139C06085D9D0608259C0608B2
:10F46000479C0608F1A9060870B585880B46044636
:10F47000C5F30B052A46002118464EF0E8F86169ED
:10F48000084A9142034602D3074A914205D319B173
:10F49000BDE870401846084770BD2A46BDE8704078
:10F4A0004EF072B894ED0608A3EF060838B5064C86
:10F4B000064DAC4206D2A16820461C34FFF7D4FFAB
:10F4C000AC42F8D338BD00BF9CE4060894ED0608B2
:10F4D0004840082310F0800F82EA40010ABF400034
:10F4E000C8B2C0B2013BF5D1704700BF30B5056866
:10F4F0008D4219D901F1FF3E6C1E00231EF801CF89
:10F50000082183EA0C0313F0800F82EA430C0ABF40
:10F510005B005FFA8CF3DBB20139F4D17445EDD1B5
:10F520006A1C02602B7030BD00236A1C02602B70C5
:10F5300030BD00BF07EE901AB8EE677ADFED7C7A37
:10F5400027EE000A60EE277ABDEEE77A17EE103A52
:10F550002033402B00F2DB809FED767AB4EEC70AB1
:10F56000F1EE10FAB0EE677A0CDDDFED735A9FED25
:10F57000736AF0EE476AF4EEC66AF1EE10FA37EEFF
:10F58000657AF6DCDFED6E6AB4EEE67AF1EE10FA3B
:10F590000CD5DFED695A9FED6B6AF0EE476AF4EE29
:10F5A000C66AF1EE10FA37EE257AF6D4DFED666A18
:10F5B000B4EEE67AF1EE10FA00F39D80DFED636AB7
:10F5C000B4EEE67AF1EE10FA44BFDFED5D6A36EE96
:10F5D000C77A27EE075ADFED5E5A9FED5E6ADFEDD0
:10F5E0005E6ADFED5E4AA5EE256A27EE054AE5EE86
:10F5F000066AF7EE005AA4EE267AF0EE656AE7EEA8
:10F60000646AE7EE245A86EEA54A9FED4F7A77EEBC
:10F61000877ABDEEE77A17EE103A2033402B6FD889
:10F620009FED4F7AB4EEC70AF1EE10FA0CDD9FEDB4
:10F63000426ADFED426AB0EE677AB4EEE67AF1EE46
:10F6400010FA77EEC67AF6DC9FED3D7AF4EEC77AD3
:10F65000F1EE10FA0CD59FED386ADFED3A6AB0EEA4
:10F66000677AB4EEE67AF1EE10FA77EE867AF6D49F
:10F670009FED357AF4EEC77AF1EE10FA4CDD9FED8E
:10F68000397A77EE677A67EEA74A9FED317A9FED78
:10F69000315ADFED316AA4EE875A67EEA43AE4EE00
:10F6A000856AB7EE006AE3EEA67AB6EE007A36EE29
:10F6B000676AB8EE005A67EE857A26EE077AB7EEEB
:10F6C000005AC5EE256A0023836143610362C3616A
:10F6D00080ED044A26EE877A26EE866A66EEA77AE1
:10F6E00080ED095A80ED007A80ED016A80ED027AA2
:10F6F000C0ED037A7047DFED1B6A36EEC77A68E724
:10F70000DFED197AB6EE007AB7EE006AD7E7B7EE0A
:10F71000004AF0EE445A78E79FED0C7AF4EEC77A8F
:10F72000F1EE10FA44BF9FED067A77EE677AAAE70A
:10F7300027D4D2360024F448DB0FC940E4CB16416D
:10F74000DB0F49C0E4CB16C1DB0FC93FDB0FC9BFDC
:10F7500092E741B99730083C15A82ABEF304353F1B
:10F7600000247448DB0F4940000000009FED2E7A12
:10F7700070EE077AFDEEE76A16EE903A2033402BE2
:10F780004FD8B4EEC70AF1EE10FA0CDD9FED276AF0
:10F79000DFED276AB0EE677AB4EEE67AF1EE10FAA2
:10F7A00077EEC67AF6DC9FED237AF4EEC77AF1EEB7
:10F7B00010FA0CD59FED1D6ADFED1F6AB0EE677A77
:10F7C000B4EEE67AF1EE10FA77EE867AF6D49FED93
:10F7D000167AF4EEC77AF1EE10FA1DDC9FED177A77
:10F7E000F4EEC77AF1EE10FA44BF9FED127A77EE8D
:10F7F000677A27EEA76ADFED125ADFED126A9FEDF6
:10F80000127AE6EE256A67EE865AA6EE267AE5EECD
:10F81000877AB0EE670A70479FED0C7A77EE677AC9
:10F82000E7E79FED0B0A7047DB0FC93FDB0FC940CD
:10F83000E4CB1641DB0F49C0E4CB16C1DB0FC9BFD7
:10F8400092E741B99730083C15A82ABEDB0F494022
:10F8500000000000F0EEC07AB0EEE07AB4EEE77A95
:10F86000F1EE10FAB4BFB0EE676AB0EE476AB5EEDB
:10F87000406AF1EE10FA46D0B4EEE77AF1EE10FAF3
:10F880008CBFF0EE675AF0EE475AC5EE866ADFEDA0
:10F890001F2ADFED1F3ADFED1F4A9FED1F5A9FED34
:10F8A0001F3A9FED1F4ADFED1F5AE6EEE23AA6EE41
:10F8B000834AE6EEA34AB7EE006AA6EEA45AA6EE85
:10F8C000846AE6EE855AC5EE866AB4EEE77AF1EE12
:10F8D00010FA48BFDFED147AF5EEC00A48BF77EEA4
:10F8E000E66AF1EE10FA48BFDFED107AB5EEC00A15
:10F8F00048BF77EEE66AF1EE10FA48BFF1EE666AAD
:10F90000B0EE660A7047DFED076ADEE739094E3D63
:10F91000E3B59E3E88FA163E45FE7F3F99FB243FA5
:10F9200069A2163EA7DFA834DB0FC93FDB0F4940B1
:10F9300090ED005A9FED4C0A35EE000A08B5FDEE39
:10F94000C07A17EE903A2033402B7BD8FFF76EF841
:10F95000F0EE403AFDEEC57A17EE903A2033402B98
:10F960007FD8B0EE450AFFF761F8B0EE405AD0ED0F
:10F97000014A9FED3D0A34EE800AFDEEC07A17EE93
:10F98000903A2033402B69D8FFF750F8F0EE405AF8
:10F99000FDEEE47A17EE903A2033402B5BD8B0EEC0
:10F9A000640AFFF743F8F0EE404A90ED023A9FED0B
:10F9B0002E0A33EE000AFDEEC07A17EE903A20339D
:10F9C000402B45D8FFF732F8B0EE404AFDEEC37A3F
:10F9D00017EE903A2033402B37D8B0EE430AFFF7AA
:10F9E00025F8F0EE407A24EE233A27EEA36A24EEBF
:10F9F000057A67EE856AB0EE462AF0EE432AA7EE56
:10FA0000242AE6EEE42AA6EE247AE3EE646A24EEE3
:10FA1000254A65EEE77A25EE655A65EEA35A81ED33
:10FA2000004AC1ED017AC1ED024A81ED032AC1ED20
:10FA3000042A81ED055AC1ED066A81ED077AC1ED10
:10FA4000085A08BDDFED093A84E7DFED087ACAE716
:10FA50009FED064ABAE7DFED054AA6E7DFED035A58
:10FA600096E79FED025A82E7DB0FC93F00000000D6
:10FA70002DE9F04389B0541C03941478002C00F055
:10FA800000810025074688461E46A94609E0214612
:10FA90003846C047039A0135531C03931478002C51
:10FAA00040D0252CF3D1931CCDE903395078302870
:10FAB00002BFD31C03939078A0F13003DBB20CBFDC
:10FAC00001240024092B40F292806C2838D0782839
:10FAD00022D857282AD9A0F15803202B1CD8DFE8B8
:10FAE00003F0AA1B1B1B1B1B1B1B1B1B1B8B931B32
:10FAF0001B1B1B1B1B1B1B1BA51B1B1B1B111B9D54
:10FB00001B1BAA0056F8043B049A009300234146AD
:10FB10003846FFF739F80544039A531C03931478C9
:10FB2000002CBED1284609B0BDE8F0830028F9D0EA
:10FB30002528F1D125213846C0470135039AABE786
:10FB4000039B5A1C039219787829A5D8572949D9BB
:10FB5000A1F15803202B9FD801A050F823F000BF3B
:10FB60004FFC000899FA000899FA000899FA000871
:10FB700099FA000899FA000899FA000899FA000819
:10FB800099FA000899FA000899FA0008F9FB0008A8
:10FB900067FC000899FA000899FA000899FA000829
:10FBA00099FA000899FA000899FA000899FA0008E9
:10FBB00099FA000899FA00082FFC000899FA000841
:10FBC00099FA000899FA000899FA000805FB00085C
:10FBD00099FA000873FC000899FA000899FA0008DD
:10FBE0004FFC000800299DD02529A3D054E704AA82
:10FBF00003A949F0B5F868E756F8041B3846C9B2BE
:10FC0000C0470135039A47E756F8040B05A9FFF7EB
:10FC100051F805AB0093049A234678E756F8040B95
:10FC200005AB00220A21FEF7FDFFF2E7039A56F822
:10FC3000043B1D6030E7A0F15802B2FA82F256F898
:10FC4000040B520905AB1021FEF7ECFFE1E7A1F12F
:10FC50005802B2FA82F256F8040B520905AB102191
:10FC6000FEF7E0FFD5E756F8040B05A9FFF722F8E9
:10FC7000CFE756F8040B05AB00220A21FEF7D2FFAE
:10FC8000C7E725464EE773B5114C01920646206D35
:10FC90000D46A0B10F49FFF799FA206D3146FFF7E5
:10FCA00095FA0D49206DFFF791FA0C49019B206DE3
:10FCB0002A46FFF7DDFE0A49206DFFF787FA94F820
:10FCC000543013B1012384F8553002B070BD00BF29
:10FCD000309A0020599C060878A00608C9F100084F
:10FCE000669C06080EB400B584B005AB019053F8CD
:10FCF000042B0649039301A8FFF7BAFE019B0022DB
:10FD00001A7004B05DF804EB03B0704709EC00080A
:10FD10002DE9F043002483B0064604802146304696
:10FD2000013437F087FE082CF8D10023DFF8688013
:10FD300086F8EA30C6F8EC30C6F8F030C6F8F43091
:10FD4000C6F8F8301F46FC3699463A46414601A8A7
:10FD5000FFF7C8FF3546032401AA12F8013B6BB137
:10FD6000013C05F8013BF8D10137082F85F80090D8
:10FD700006F10406E9D103B0BDE8F0832846224627
:10FD80002021254401374DF062FC082F85F80090B2
:10FD900006F10406D9D1EEE7F8550608F7B5114E7D
:10FDA00007463046002300F8563F0C460E4B0F49DD
:10FDB000002F08BF194615464DF051FC0C4F04EBBF
:10FDC00045055636AC4202D10A4803B0F0BD39466B
:10FDD00034F8022B6846FFF785FF694630464DF040
:10FDE0003EFCEFE7309A0020739C06086A9C0608E8
:10FDF0007C9C0608869A0020F7B50C4E0C4F002319
:10FE000006F8873F044600EB4105AC4202D10948A1
:10FE100003B0F0BD394634F8022B6846FFF762FFA5
:10FE2000694630464DF01BFCEFE700BF309A0020DA
:10FE30000A9D0608B79A0020F8B5084F4E1E0546E1
:10FE400001F11F0416F8012F28463946FFF74AFF33
:10FE5000A64205F10205F5D1F8BD00BF819C060858
:10FE60000246531C084605D1034B1A681B790A60E9
:10FE70000B717047014935E7BF9B06080B9D0608CB
:10FE800010B5013114460EF0C7F928B9054B1A68B0
:10FE90001B792260237110BDC27903492046BDE859
:10FEA00010401FE7BF9B0608209C060803685A1CE9
:10FEB000026019700368090A5A1C026019707047C1
:10FEC00002681146531C036011F802CB0160D31C79
:10FED0005178036093781B0443EA0123111D0160EC
:10FEE000D07843EA0C0343EA00607047A0F1300386
:10FEF000092B07D920F02000413819288CBF002099
:10FF00000120704701207047303809288CBF00203D
:10FF100001207047413819288CBF0020012070470C
:10FF2000613819288CBF002001207047202805D097
:10FF3000093804288CBF0020012070470120704739
:10FF4000A0F14103192B98BF20307047A0F1610345
:10FF5000192B98BF2038704710B500F100440246B5
:10FF6000013C04E0B3EB0E0015D1A24214D012F80C
:10FF7000013BA3F14100192811F8010BA0F1410C3C
:10FF800098BF2033BCF1190F00F1200EEAD91B1ADB
:10FF900004D10028E9D110BD002010BD184610BDC5
:10FFA00002B310B58446841804E0B3EB0E0014D1FC
:10FFB000A44513D01CF8013B11F8010BA3F1410239
:10FFC000192AA0F1410298BF2033192A00F1200E0E
:10FFD000EBD91B1A04D10028EAD110BD002010BDB6
:10FFE000184610BD1046704770B5044608460D46C9
:10FFF0004BF03EF8064602E014F8013F43B12046BC
:020000040801F1
:1000000032462946FFF7CCFF0028F5D1204670BDC7
:100010001C46204670BD38B507490546FFF7E4FF8A
:100020000649041E284618BF0124FFF7DDFF08B16A
:1000300044F00204204638BD869C060842B50608F6
:100040002DE9F041044686469EF800C0BCF1200F21
:100050007046ACF109050EF1010EF5D0042DF3D96F
:10006000BCF12B0F5BD0BCF12D0F3BD1102A4FF010
:10007000010600F1010E58D19EF800C0BCF1300F0E
:100080005FD04FF010086FF070450F2742460EF119
:10009000010E00200DE0ACF1300C5FFA8CFC9445B1
:1000A0000FDA854274462DD32AD008FB00C01EF813
:1000B00001CBBCF1390FEED94CF0200CBCF1600F34
:1000C0000BD801B10C600EB323B1B0F1004F28BFC3
:1000D0004FF000404042BDE8F081ACF1570C5FFAB0
:1000E0008CFCDCE7102A864649D04FF0FF35B5FB83
:1000F000F2F502FB05F7FF43FFB290460026C6E784
:100100006745D2D21E404FF0FF30D0E7002BE2D03F
:100110006FF00043984228BF1846BDE8F081102ACE
:100120004FF0000600F1010EA6D04FF0FF35B5FBF1
:10013000F2F502FB05F7FF4390F801C0FFB29046CD
:10014000A5E79EF801C0ACF1410019280EF10104A9
:10015000624601D80CF12002782A4FF0100805D031
:10016000A6466FF070450F27424690E79EF802C002
:100170006FF070450EF1020E0F27424687E700260A
:100180007AE773B50E4611490546FFF7E5FE18B943
:100190003070012002B070BD2C78602C8CBF613CA7
:1001A000413C072C10D8013501230A2201A9284619
:1001B000FFF746FF019B9D4206D00F2804D801346B
:1001C00040EA04143470E4E70020E3E7BF9B06082C
:1001D00001230A22002133E770B50D461446FFF7CC
:1001E00007F80646A0B1FFF7F3FF40F63403984244
:1001F000A8BF1846B0F5617FB8BF4FF46170A0F595
:1002000061731920B3FBF0F32B7023780133237053
:100210003046FEF7EDFF0646A0B1FFF7D9FF40F6E6
:1002200034039842A8BF1846B0F5617FB8BF4FF4B9
:100230006170A0F561731920B3FBF0F36B70237844
:1002400001332370304670BD2DE9F04117461E463C
:1002500005464FF47A720023384631464BF0CCFB0A
:100260004349444A014482FB0143C8170B44C0EB95
:10027000631382FB03021A44D8173F4CC0EB62128F
:1002800084FB02044FEAE27C3C48CCEBA40C80FBEC
:100290000C404FEAEC74C4EBE010C3EB0314A1EB89
:1002A0008401A971C2EB0211A3EB81036B710CEB0A
:1002B0004C03A2EBC30240F2B55303FB10CCBCF5D8
:1002C000896F2A714FEA800043DA40F2DA239C45B5
:1002D00046DCBCF5B77FB4BF00220122284B02EBFD
:1002E000420103EBC1034FEA42085B8D91B2254CFA
:1002F00008EB020E04EBCE0416344FF00B0E01E0B7
:1003000034F8023D63451FDDBEF1010EF8D11C4BF0
:10031000424403EBC2024FF0010E938A85F802E0DB
:1003200000F5FA600CF1010C0844ACEB030C2880DA
:1003300085F803C04FF47A720023384631464BF0FB
:100340005BFB2A81BDE8F0810EF1010E5FFA8EFEA3
:10035000E4E7032140F296530A464FF00608C6E749
:10036000022140F229430A464FF00408BFE700BFCC
:1003700080BC92C789888888ABAAAA2A73B06D16F8
:1003800064F3050878F3050808B50C4BD3E900239E
:1003900052EA030C09D1002340F20112428083800B
:1003A000837103800381184608BD054909688A18CE
:1003B00043F10003FFF748FF012008BD503500203E
:1003C0007421002090422DE9F0410B460446154669
:1003D0000AD2B0FBF5F6134A05FB16441846135D26
:1003E00000F8013BBDE8F081B0FBF2F69642B6FBA7
:1003F000F2F706D20B4A05FB1767D15D03F8011B24
:10040000EAE7BA42B7FBF2F807D9064A05FB1878C3
:1004100012F8081003F8011BEDE74046FFF7D2FF82
:100420000346F2E7005606087D4B9A88B3F808C0E9
:1004300058899989B2F57A7F88BF4FF47A7230B5BE
:1004400088BF9A80DA88774CB2F57A7F84BF4FF400
:100450007A72DA80BCF57A7F84BF4FF47A7CA3F895
:1004600008C0B0F57A7F88BF0020DA8988BF58813C
:10047000B1F57A7F84BF4FF47A719981B2F57A7FB2
:1004800084BF0022DA8184459CBF002018819142FC
:1004900098BF0022598B98BF9A819A8B914284BF52
:1004A00000225A83604B1B8883B0002B43D06279B3
:1004B0005E4D012A63D9AA78062A97BF5C499FED51
:1004C0005D7A01EB820191ED1D7A2979002940F0D6
:1004D00084805949087807EE903A06EE900AF8EEC3
:1004E000E77AB8EEE66AAB79C6EE276A002B6CD1E4
:1004F000B4EEE67AF1EE10FA1DDD67EE277ABCEE77
:10050000E77A8DED017A9DF8042007EE102AB8EE07
:10051000C77AF4EEC77AF1EE10FAC4BF0132D2B254
:10052000002A6ED0102AA8BF1022D2B282421346EF
:1005300038BF03460B7063782278032B95BF3F4981
:100540003E49C3EB0313002394BF01EB43016370E7
:100550003B4B032AC3F8B8139DBF02EB820103F59E
:10056000947302EBC102002294BF03EB820322705A
:10057000344A88BF03F59473136003B030BDAA7981
:10058000002A98D0AA78072A09D0B3F57A6F93D9B0
:10059000294908780228B8BF022008708CE7062293
:1005A000B3F57A6FAA702ED82A79002AC3D12249CE
:1005B0009FED257A087807EE903A06EE900AF8EE5D
:1005C000E77AB8EEE66AC6EE276A37EE077AB4EE47
:1005D000E67AF1EE10FAAEDD8FE7042A02D8002A9F
:1005E000A9D002E0053A032AA5D9B7EE000A80EEA9
:1005F000070A4CF051FA2B88984228BF18462880E9
:1006000099E7012291E70C490A78022AB8BF022231
:100610000A702A79002A8ED19FED0B7A5AE700BF23
:10062000943700206C3500201C0F0010D0270020CC
:1006300064F305086F1203384C370020E09A00205D
:10064000309A00205437002017B7D1382DE9F04FE9
:10065000BC4B83B01B78A3F11702022A00AF13D959
:10066000B94A12F83310002940F0E282DB001A4444
:1006700052784AB1B54A3A60134493F890302BB996
:10068000B04A1823137001E0B04B3B60B04DDFF867
:10069000ECB295F8C493AF4E05F57D74A0464FF0CB
:1006A000000A33E010F0010254D1142900F0BC829A
:1006B0004308810801F0333103F077330B44C1085C
:1006C00001F01131C31A5B1A03EB131303F00F335C
:1006D000ABFB03C1C909C1EB0121591A830302D540
:1006E000012900F0A18201290BD9082900F29C827E
:1006F0000AB1304205D149464AF058F8002800F0C6
:100700009382954B08F10C08984528D098F904106D
:10071000D8F80000A1F11E03DBB2012BC2D898F873
:100720000630022BA8BF022388F8063098F807305D
:10073000022BA8BF022388F8073098F80830022B54
:1007400020F04100A8BF0223C8F8000088F8083054
:100750000022ADE70AF1010A5FFA8AFAA8E70AF176
:10076000FF3ABAF1020F00F25F824FF00008022058
:1007700085F8648411F06CFE95F86834022B00F063
:10078000E882002800F05283744BDFF8F4A17B600C
:10079000734B95F8C1B403F524764FF47A794FF092
:1007A00000085A88B2F57A7FB3F8462088BFA3F8CC
:1007B0000290B2F57A7F9A8888BFA3F84690B2F586
:1007C0007A7FDA8888BFA3F804909988B2F57A7F97
:1007D00084BF0022A3F806809142B3F85A10B3F800
:1007E0005C2098BFA3F80480914293F86B2088BFE7
:1007F000A3F85A80013A632A84BF642283F86B20ED
:1008000093F86C200132D2B2092A88BF83F86C8039
:1008100003F166001946002291F80AE010F801CBB6
:100820000132E64538BF00F8018C032A01F10601C8
:10083000F2D1BBF1010F18BF83F88580A4339E422B
:10084000AFD1484B9B78042B00F0CF823BB9454A8F
:100850001388B3F5F07F84BF4FF4F0731380424EDA
:10086000FFF7E2FD95F8D4144048FEF7F7FBF17965
:1008700006F10800FEF7F2FB717D06F11600FEF7A7
:10088000EDFBB5F8F224B5F8F0341343B5F8F424D1
:1008900013431BB213B10123A5F8F6347B68344A25
:1008A0001B681A40002A00F0D982D90700F1438260
:1008B0005A0440F1C8812F497A680B401360DAF876
:1008C00000200A40CAF8002013F4004200F016820B
:1008D000002285F8CB2385F8DB23D90440F1188268
:1008E00095F80335DFF89080022B04BF012385F8CB
:1008F000033508F1780B434602E006339B450CD0E4
:100900001A78072AF9D19978DA78914202D35A797C
:10091000002AF2D0072023F0E3F800234FF4806090
:1009200085F8643411F094FD002800F07382124EB3
:10093000B14699F8051081B399F8000058B34346C1
:1009400023E000BF2136002028EB050864F30508EA
:10095000309A0020BC020200909E0020F43B002050
:10096000589B0020D0270020183C0020149F002016
:1009700009600002F6DFFFFD389F00208180808043
:10098000A835002006339B4507D01A788A42F9D152
:100990005A79002AF6D023F0A3F809F10609CB45CD
:1009A000C7D1B44B93F80280B8F1080F00F0F28180
:1009B00095F8C22495F8C104AF4BDFF8F8E2DAF8F5
:1009C0000010A2F10102B2FA82F25209A0F1010074
:1009D0001A71B0FA80F09EF8012040091870032ABD
:1009E000C1F3C030987084BF00238EF80130A34B50
:1009F000A34A987B7B681B6813400A407968CAF851
:100A000000200B60002800F0D081DFF8ACA2BAF81B
:100A10000430002B40F0D6819A4A136813F07F4FC0
:100A20001CBF00231360936823F4007323F00203B8
:100A300013B140F2022393601379013B042B84BF6E
:100A400001231371A8F105088F4BB8F1030F93F838
:100A5000009040F24981B9F1000F1ED000237B6065
:100A6000844A6FF00703A3EB020802F1080A04E0CE
:100A700008EB0A034B4580F0EA801AF8010B0028C6
:100A8000F6D00DF0F3FB0028F2D083799B07EFD569
:100A90007A680123002A40F0DF80764B9B7913B1FE
:100AA000744A00239371794BDA8812F00C0F03D14A
:100AB000C2F30312022A02D94FF42062DA801A89A3
:100AC00012F00C0F03D1C2F30312022A02D940F62E
:100AD00001221A8195F88D3595F881259A4295F86D
:100AE000803505D9002285F8812553B1A5F88425E4
:100AF00095F88C259A423EBF002385F88035A5F8ED
:100B0000843595F8763695F882256148D7F80090B7
:100B10009A4284BF002385F8823500F1780A10F8E4
:100B2000013C03EB43034B444FF0030893F868E1A7
:100B300093F869C193F86A1103461A787245A8BF01
:100B4000724603F8012B5A796245A8BF62465A7172
:100B50009A788A42A8BF0A46B8F101089A70ECD187
:100B60001E308245DBD1D5F8EC23002A00F0348119
:100B70004FF0000C01203378282B08D17378043310
:100B800000FA03F313421CBF9A434FF0010C0636E0
:100B9000B345F0D1BCF1000F01D0C5F8EC23DFF86C
:100BA000F4A00AF10809534613F8012B072A00F2B2
:100BB00085809945F8D1EB4688B06B46FF211846F1
:100BC00020224CF044FD3349034611F8012B53F821
:100BD0002200013079D1894543F82220F5D1B5F8BA
:100BE000BA24B5F8B8349A42DD4602D32A4BC5F888
:100BF000B834FF23294985F8A83694F90430142B1A
:100C000004D0226831EA020200F0EC80244B0C345C
:100C10009C42F2D1234B5A79022A01D100225A7107
:100C20000C37BD46BDE8F08F1F4811F0CDFB9CE5A9
:100C300002EBC301DB00496800297FF418AD1B48B3
:100C40001721017013E51E077ED5194934E67A682D
:100C50000023002A3FF421AF06494A7C002A7FF492
:100C600022AF4A79012A3FF418AF002B7FF415AF69
:100C700019E700BFD0270020E06400206C35002079
:100C8000FEDFDDFD5C370020C00D0010CC3A0020F7
:100C9000E39A0020E3270020AE014A010100020090
:100CA000909E0020FC260020249E0020213600205B
:100CB000FE9FFFFD94370020F4640020EB4688B0CF
:100CC0002022FF2168464CF0C2FC0AF8018B08F193
:100CD0000108B8F1080F82D00AF8018B08F1010869
:100CE000B8F1080FF1D17AE7624A00231371B9F124
:100CF000000F00F0AA8001237B60B1E695F8CB13CA
:100D000000293FF4EAADD90485F8DB233FF5E8ADCF
:100D10001A067FF5E5AD584B1978182906D8574BB8
:100D200001228A401340002B7FF4DAADDFF868819E
:100D300008F1780BF1E552497A680B401360DAF854
:100D400000200A40CAF8002098047FF5BDAD4D4947
:100D5000B2E500283FF418AD4B4E4C4B90F904E03F
:100D60003078414603F16C0C4FF0FF0893F90820EE
:100D7000724504BF00F1FF3083F8088003F10C03D3
:100D800004BFC0B201216345F0D100293FF4FCAC9F
:100D90003070F9E41A469B79002B3FF409AE537C7E
:100DA000012B04BF0223537402E639480243CAF8F8
:100DB0000020DFF8E8A003430B60BAF80430002BF2
:100DC0003FF42AAE9AF800000DF050FA00287FF4A4
:100DD00023AEAAF804001FE6282022F081FED5F8F1
:100DE000EC23C5E685F8A83614E77A68136823F47F
:100DF00080531360DAF800301E4A23F48053CAF897
:100E00000030538CB3F57A7FBFF429AD4FF47A7379
:100E1000538424E57A68136823F000631360DAF8DA
:100E2000003023F00063CAF8003080E5194ADFF88B
:100E300070A013687A6023F080031360DAF8003042
:100E400023F08003CAF80030A2E4537C002B7FF427
:100E50002AAE5379012B7FF426AE1EE67A6843F062
:100E600008031360DAF8002042F00802CAF80020F4
:100E70001BE500BFD02700202136002000410001E3
:100E8000F79FFFFDF6BFFFFDAC350020B035002019
:100E900020061500F43B0020389F0020F464002059
:100EA000A83500202DE9F04FDFF80C82754BD8F8FB
:100EB0000C2002F2DC52C8F80C20734A934283B033
:100EC00080F0DC8003F11C059B46704B704E4FF0A8
:100ED000010A9F1C6D4B5A88002A00F0B880BB188D
:100EE000B34280F0B4803C4608E01A881C461344A4
:100EF000002A00F0AC80B34280F0A980052A40F2BD
:100F0000A68035F81C2C6188C2F30B029142ECD10B
:100F100062799207E9D1238855F8141C94F804905B
:100F200001935846FEF7A0FA35F81C2CB9EB123F96
:100F300000F095804FF0000A35F8181C55F8140C95
:100F4000C1F30B0146F072FD55F8043C18604E4B9E
:100F50000BF11C0B9B4505F11C05BBD34D4A4E4BB9
:100F60004E4F12681A60FFF771FB3B784C4C4D4DA9
:100F70007A784D4E03EB830103EBC10304F59471C2
:100F800001EB83032B60C2EB021204F1B00303EB0D
:100F90004202C4F8B82321F0B7FF4FF0FF332868AE
:100FA00073602DF055FB22F0EFFD04F5A16304F50D
:100FB000B06102E006338B425BD01A78002AF9D187
:100FC0009D78D878854202D358790028F2D094F8D9
:100FD0000035327203EB830303EB83039B00632B27
:100FE000B4F80425D8BF6423C8F80430642303FB95
:100FF00002F2632ADCBF1A46C8F808304FF000033B
:10100000C8BFC8F80820C8E90732284AA8F8243021
:10101000C8E90333C8E9053388F82630244B9362C6
:101020002EF0DAFCB4F8AC0694F8AE1623F032FCDD
:1010300039F0C4FB18F090F81E4A1268C8F80C206A
:101040000123504688F8253003B0BDE8F08F55F8ED
:10105000141C5846FEF708FA4FF0000A6CE7019B93
:10106000A11D9A1F5846FDF7DFFB00287FF464AFEF
:1010700060E7FA7B003A18BF0122A8E74FF0010AA7
:101080006CE700BF9CE4060894ED060800400008E9
:1010900000800008F43B0020A83500206C350020BB
:1010A000309A00205437002094050020AC14001022
:1010B000209F0020742100206837002038B51C4B89
:1010C0000122032805461A7020D96A1CD2B25200A8
:1010D0001848402A28BF4022002300F5D661022488
:1010E0004FF0140ECC54023301EB030C9A420CF86F
:1010F00001ECF7D8FF2D08BF02220244FF2382F83B
:10110000B036BDE838400E2011F0C2BB05EB8503B8
:1011100009480A4A05EBC30300EB8300084B15702E
:1011200018602DF095FA23F06BFF24F03FF8CCE720
:10113000E0140010309A0020589B00206C350020ED
:1011400054370020054BD3F8F426012142F4001255
:1011500083F8F116C3F8F426704700BF309A0020D8
:10116000F8B5164D6B78BE2B26D1022229464FF6D4
:10117000FF70FDF7FDFB124FAC1C22884AB1A61888
:10118000BE4219D2052A17D92146FDF7F1FB344694
:10119000F3E721460222FDF7EBFB0222A118FDF73F
:1011A000E7FB0634074B641BA3F8F84641F60F53E0
:1011B000C31A58425841F8BD0020FCE7004000081F
:1011C00000800008309A0020F8B50468C4F30D04CC
:1011D00006460F460CB335683F6843F099F9092875
:1011E00040F08780444C236923F4407323612369D2
:1011F00043F400732361236943F0010323612F60EB
:1012000043F086F92369092823F00103236170D193
:10121000336804333360002034E0384B384A93425B
:101220002AD302F58042934225D302F580429342AD
:1012300029D3344A934228D902F58032934226D9E1
:1012400002F50032934224D902F50032934222D9AA
:1012500002F50032934220D902F5003293421ED9A2
:1012600002F5802293421CD9B3F1016F1BD348F0E1
:1012700043FB47F0CDFD082443F04AF9092814D078
:101280004FF0FF30F8BD1024F6E71824F4E72024CF
:10129000F2E72824F0E73024EEE73824ECE7402496
:1012A000EAE74824E8E75824E6E7134D2B6923F4DE
:1012B00040732B612B6943F400732B612B6923F07E
:1012C000F8032B612B691C4344F002042C612B6949
:1012D00043F480332B6143F01BF92B6923F00203A5
:1012E0002B612B69092823F0F8032B613FF473AFBE
:1012F000C6E76FF00100C5E7003C0240004000086F
:1013000000400008FFFF00082DE9F041574F3B78EF
:10131000B12B8AB06FD1FFF723FF80F00104E4B254
:10132000534B544DB3F87731534EADF8003004F0C1
:101330000104B54261D3002C00F0968010220021F8
:1013400006A84CF084F94D4B0497DB1B05934C4BDE
:10135000484F1A69002ABFBF4A4A5A6002F18832D0
:101360005A6001228DF82420F322DA6069460222B5
:1013700004A80025089549F0B1FC022269464FF601
:10138000FF70FDF7F5FA0446B74243D3022201A9E4
:1013900004A80025ADF8045049F0A0FC022201A9E0
:1013A0002046FDF7E5FA40BAC043ADF80800022236
:1013B00004A802A949F092FC079868B106ABC0F1F5
:1013C0000402294618444CF042F9089818B906A9B5
:1013D00004A8FFF7F9FE08909DF82430089823B17F
:1013E000274A136943F000431361B0FA80F04009C3
:1013F0000AB0BDE8F081012492E7A988A868C1F38A
:101400000B0146F013FBAB691B681C35834218BF08
:1014100001248EE7B7F804808DF80D50C8F30B084F
:1014200008F10603ADF808303B88C3F30B02ADF8B2
:101430000A201B0B062202A904A88DF80C3049F0E3
:101440004DFC062202A92046FDF792FAB96804462F
:10145000424604A849F042FCB96820464246FDF7DE
:1014600087FA1C3704468FE70120C1E700400008D7
:1014700064F305089CE4060894ED06080080000863
:10148000003C024023016745F8B5144D144E154F3A
:10149000FFF7DCF8EB68012403F2DC53EB6086F81D
:1014A000FA46FFF731FF28B13B78B12B02D1FFF7A5
:1014B00057FE18B9032C0DD00134F2E70A4A002375
:1014C000116886F8FA360122E96085F8252086F849
:1014D000FB36F8BD48F010FA47F09AFC6837002058
:1014E000309A0020004000087421002008B50B4904
:1014F0000B4A01230B709373FFF7C6FFFFF7D2FC73
:10150000084B41F20241FF22A3F8B01683F8B2263D
:10151000BDE808400E2011F0BBB900BFE014001078
:101520006C350020309A002090F88730DFED6A5A41
:1015300003EE903A90F88B3006EE103A90F889302E
:1015400004EE103A90F88A30F8EEE33A04EE903A5E
:1015500090F88D3063EEA57AB8EEC66A03EE903A45
:1015600026EE256AB8EEC44AF8EEE44AF8EEE33A0D
:1015700026EE276A24EE254A64EEA54A63EEA53AD4
:10158000F0B5564D24EE064A64EEA74A63EEA73A3C
:1015900000210626F7EE002AA5F10C0C00F1660EDC
:1015A00006FB01F2B7EE005AAC1890F886700244C0
:1015B000F0EE456A15E0012904F1060402F1060285
:1015C000EED190F8883007EE903A90F8903006EE21
:1015D000903AF8EEE77AF8EEE66A27EEA55A66EE5C
:1015E000A56A237807EE103A66EE867AB8EEC77AD7
:1015F00027EE277AFDEEC77A17EE903AFA2BA8BFAE
:10160000FA2323EAE3731372637807EE103A66EE67
:10161000847AB8EEC77A27EE277AFDEEC77A17EEFE
:10162000903AFA2BA8BFFA2323EAE37353725CF8CB
:10163000213007EE903A002BF8EEE77A49DDA378E7
:1016400007EE103AB8EE477A90F88C3037EE677AAA
:1016500003EE103A87EE272AB8EEC33AB0EE627A6C
:1016600023EE253AA2EE037A64EEA77A66EEA36A29
:1016700067EE857A27EE877AFDEEE77ABDEEC77AC8
:1016800017EE103AFA2BA8BFFA2323EAE3739372FA
:1016900017EE903AFA2BA8BFFA2323EAE3730EF869
:1016A0000130A38807EE903AF8EEE77A013167EE51
:1016B000A67AFDEEE77A17EE903AB3F57A7FA8BFE7
:1016C0004FF47A7323EAE3738F429381BFF673AFCB
:1016D000F0BDB7EE007AC7E70AD7233CECF4050863
:1016E00090F88E306BB3B0F85A308BB190F88F20F1
:1016F00002EB82036421C3EB0313B3FBF1F3A0F805
:101700005A30962312FB03F3B3FBF1F3A0F85C30DD
:1017100043884BB190F88F3003EB8303C3EB031383
:101720006422B3FBF2F34380B0F846304BB190F83B
:101730008F30962213FB02F36422B3FBF2F3A0F87E
:101740004630704790F821304BB3438B83B190F80B
:101750002230FA2213FB02F203EB8303B3F57A7F04
:10176000A8BF4FF47A7364218383B2FBF1F2428302
:10177000838843B190F82230FA2213FB02F36422EB
:10178000B3FBF2F38380C3884BB190F8223003EBB4
:101790008303B3F57A7FA8BF4FF47A73C380704791
:1017A00070B50A4C0A4E002594F8863013B12046D5
:1017B000FFF7BAFE2046FFF793FF01353046FFF7EB
:1017C000C1FF042D04F1A404EED170BD589B00208C
:1017D00094370020034BD3F8FC0608B107F0B8BEDD
:1017E000704700BF309A002008B50B4605490246F5
:1017F000D1F8FC0628B10449FEF73AF9BDE80840E3
:10180000E8E708BD309A0020C9F10008024B014604
:10181000D3F8FC06FDF7DABC309A002008B5044680
:101820000848FFF7F3FFFFF7D5FF074BD86C10F020
:10183000ADFF0CF0E7F8012C01D147F0E9FAFAF717
:1018400031FC00BF899C0608309A00200048DDE783
:10185000EFA906080CB4C30607B500D561B9049812
:1018600005A90191FFF7C0FFFFF7F0FF012003B0CA
:101870005DF804EB02B070470020F8E708B5FFF709
:10188000C5FFBDE80840E1E710B504460348FFF78F
:10189000BDFF2046BDE81040F0E700BF959C06085C
:1018A00008B50948FFF7F0FFFFF794FF074B002446
:1018B00083F80047C3F8004883F8044823F046FD46
:1018C0002046FFF7ABFF00BF9A9C0608309A002025
:1018D000034B0146D3F8FC0608B107F025BE70475C
:1018E000309A00200CB407B510F020000BD079B965
:1018F0002320FFF7EDFF049805A90191FFF774FF7E
:10190000FFF7A4FF012003B05DF804EB02B07047BD
:101910000020F8E70FB407B504A951F8040B0191B2
:10192000FFF762FF03B05DF804EB04B07047154B9E
:101930001B6870B52BB31448144EFFF79FFFFFF7D9
:1019400049FFFCF717FA0025FCF74AFA044640B1B4
:10195000132010F09DFFFFF779FFBDE870400C48A1
:101960008CE73046FFF7D6FF782D06D80135FFF714
:1019700031FF64200CF0AAF8E6E7FFF767FF254681
:10198000F5E770BD2C210020C19C06083ECA060860
:10199000DB9C060838B50B4B03EBC0050C4695F8ED
:1019A0000C23094803EB8203D3F89C11FFF7B2FF25
:1019B00095F812332BB1611C0448BDE83840C9B218
:1019C000A8E738BD64F30508EDB306080A9D0608CC
:1019D0000FB407B504A951F8040B0191FFF704FFF8
:1019E000FFF734FF03B05DF804EB04B070472DE956
:1019F000F041037903F0E002402A50D004D85AB1F4
:101A0000202A29D0BDE8F081602A4BD0802AF9D164
:101A100082794179254812E003F00703052B16D897
:101A2000DFE803F0101510150309D0F80510204861
:101A3000BDE8F041CCE7D0F8052051421D48BDE893
:101A4000F041C5E7B0F80720B0F80510F6E7B0F9A7
:101A50000720B0F90510F1E74679174D174805EB57
:101A6000C605FFF7D3FE95F8287400240123A7428A
:101A700002D8BDE8F041E9E6D5F8246456F8242000
:101A80004FEA84084AB113B90D48FFF7BFFE56F874
:101A900008100C48FFF73EFF00230134E7E74179C7
:101AA0000948C5E7BDE8F041084891E7309D0608C0
:101AB000E19C0608F79C060864F305080E9D0608DD
:101AC000C1A00608EDB306081F9D0608479D06083D
:101AD0002DE9F04387B0FCF73DF90269838901885D
:101AE0000292826801924288009242681B4EDFF89F
:101AF00080801B4FDFF87C9004461A48FFF768FF90
:101B0000002515B94046FFF7B9FE3B689D4213DA40
:101B100033781548052B96BF09EB83030022D3F8D1
:101B2000F425B3880093294673880135FFF750FFE9
:101B3000062D06F10606E4D147F038F9818843887E
:101B4000CB1A616803FB01110591FCF78DF905992A
:101B50000246064807B0BDE8F04339E75C30002094
:101B6000CC2F00205F9D0608C99D0608D89D060859
:101B7000BD9D060864F305080249034801F521618B
:101B80000EC925E70070FF1FF59D060810B57521E9
:101B900004462EF0F5F901460948FFF719FF1A210E
:101BA00020462EF0EDF901460648FFF711FF1B21F4
:101BB00020462EF0E5F9BDE810400146024807E74F
:101BC000099E06081C9E06082F9E060838B50B4D78
:101BD000E87810F0FD0405D10948FFF7F9FE20462A
:101BE000FFF7D4FFEB78013B012B06D80548FFF740
:101BF000EFFEBDE838400120C8E738BD943700202B
:101C0000429E06084D9E06082DE9F04F784B794913
:101C10001A687948794BB2FBF3F299B0FFF77AFE74
:101C2000774BDFF854C20FCBDCF808400CAF87E8E5
:101C30000F00744B0793A608734B089316F0020627
:101C4000C4F3810418AB18BFDCF8045003EB840321
:101C500018BFC5F3805553F8301C002E00F0C68025
:101C600018AB03EB850555F8442C684C6848694E61
:101C7000694FDFF80882DFF8CC91FFF74BFEB4F82C
:101C800006284FF47A73B2FBF3F103FB11220A200A
:101C9000B4F9083892B2B2FBF0F26048FFF798FE50
:101CA0005F4A60496048FFF735FEFFF7CFFD5F4BA5
:101CB0005F4A997B5F4B604806EB8101D31AD1F8EC
:101CC0001C16B4F8F826FFF783FE5C48FFF79EFD6C
:101CD00094F80A185A48FFF71DFE5A48FFF796FD78
:101CE00094F80B185848FFF715FEFFF7AFFD57485B
:101CF000FFF78CFD00210A46FB7F0B4113F0010F1B
:101D000001F1010508D012B14846FFF77FFD2946D1
:101D10004046FFF7FFFD0122072D2946ECD14C4D2F
:101D200095F86A1505F5EC7305F13C02012918BF19
:101D3000134693F8DC30032B02D04648FFF7EAFD48
:101D4000454B95F86A15A3F5CE72012918BF1346C5
:101D500093F8DC30012B02D14048FFF7DBFD3E4B0E
:101D600095F86A15A3F5CE72012918BF13461B69B1
:101D70005B7B012B02D93A48FFF7CCFD394FDFF8E6
:101D800000A1DFF800B1FFF761FDD4F80C38039330
:101D9000002507F1200957F8041B002974D00123FE
:101DA00003FA05F8039B18EA030F1DD018F01F0F64
:101DB0001AD01AF8050059F8252052F8202035B11C
:101DC0002948CDE90412FFF721FDDDE90412584648
:101DD000FFF7A0FDB8F1020F06D1244B93F82110B4
:101DE00011B12348FFF796FD0135D4E7214A3CE7BE
:101DF0001C210020609E0608659E060840420F00D8
:101E000070F90508829E0608879E0608309A002011
:101E10008C9E060864F3050894370020949E0608FB
:101E2000F0FF001000080000B59E06086C35002089
:101E30000080000800400008D99E0608089F060898
:101E40001A9F0608229F0608249F06082C9F060852
:101E50001C0F0010459F0608F41000104D9F060847
:101E6000529F060888F90508C1A00608E014001072
:101E7000609F0608F1A90608003802403C9F06084A
:101E8000A00500205A9F0608FFF7E0FC7E4B7F4824
:101E90001A687F4B1978137A527A06EB8101D1F8D0
:101EA0005816FFF795FD7B497B48FFF733FD7B49CB
:101EB0007B48FFF72FFDFFF7C9FC7A4B7A4819687A
:101EC0004FF47A73B1FBF3F1FFF724FD09A8FEF795
:101ED0005BFA38B109A910A849F02EF8734810A987
:101EE000FFF718FDFFF7B2FCD4F89828002A00F09D
:101EF000878007EE902ADFED6E6AB8EEE77AC6EECD
:101F0000877AFDEEE77A17EE903AB4F8D00F58B121
:101F100007EE900ADFED666AF8EEE77A86EEA77ABA
:101F2000FDEEC77A17EE900AD4F818585DB107EEA7
:101F3000905ADFED5F6AF8EEE77A86EEA77AFDEE5B
:101F4000C77A17EE905A5B49B1F85C106429A8BFB4
:101F50006421CDE900055848FFF73AFD94F8D23FD7
:101F600094F8D32FB4F8D41F544806EB8303D3F866
:101F70006C36FFF72DFD524B5248198889B2FFF796
:101F800027FDFBF7E7FE016921B182684E48120D7B
:101F9000FFF71EFD4D48FFF739FC4D4B1B681B0634
:101FA0005ED54C4F3B78032B8CBF4B484B48FFF71B
:101FB0002DFC94F86834022B24D14948FFF726FC05
:101FC0003B78042B43D84748FFF720FC3B7C002B91
:101FD00044D006EBC303D3F8C4164348FFF79AFC7A
:101FE000FFF734FC4148424FFFF710FCD4F8F446A9
:101FF0000125002C38D1FFF729FC19B0BDE8F08F7E
:10200000134682E7022010F045FA054608B9394820
:10201000D4E738F0B9FB95F9041006EB80000131E4
:10202000D0F880263448FFF775FC94F86B34012B08
:1020300004D13248FFF7EAFB3148BFE7AB793148BA
:1020400006EB8303D3F88016FFF764FCF4E794F8FB
:102050006A340BB92C48B7E72C48B5E72C49BCE7E4
:102060002C48FFF7D3FBBBE794FAA4F3B3FA83F34E
:1020700005FA03F206EB83033846D3F8F81624EA90
:102080000204FFF747FCB4E7503B0020649F0608BA
:102090004E3B0020769F0608979F0608A59F0608DE
:1020A000AB9F060874210020B19F0608CB9F06084D
:1020B00000247449E0140010DE9F060824A00608DE
:1020C000A42700204BA006085AA0060875A0060801
:1020D000A835002030AA00207BA0060887A00608AB
:1020E00097A0060891CA0608DFA00608FBA006080C
:1020F000EBA006089DA00608A7A00608BBA006083E
:10210000C0A0060876AC0608C4A00608D4A006083D
:10211000589E0608EFA006082DE9F04FDFF8708101
:1021200098F8033099B0002B00F094804F48504E3F
:10213000DFF860B1DFF86091DFF860A1FFF79EFB88
:1021400000252F460BA9E8B217F062FA9DF834304B
:10215000002B53D0139C54B107EE904A9FED450AD3
:10216000F8EE677A80EE270A4AF096FC04460B9A4E
:1021700029465846FFF7CEFB109A002A6CD002FB86
:1021800004F04FF47A73B0FBF3F30993DDF848C021
:10219000BCF1000F62D00CFB04F142F21073B1FBF2
:1021A000F3F198F80330082D18BF7F18002B57D093
:1021B0001798079015980690169805900A2311987D
:1021C0004FF47A7EB0FBFEFE0998CDF810E0B1FB2B
:1021D000F3FE03FB1E11CDE902E10999B1FBF3F116
:1021E00003FB1100CDE90010BCFBF3F32146504680
:1021F000FFF7EEFB0023C6E90D33B36201351F2D57
:1022000006F140069ED198F8033003B31A4C1B48E0
:1022100054E939124FF47A73D208B1FBF3F354F84E
:10222000DC1CFFF7D5FB0A221548B7FBF2F102FBD5
:102230001172FFF7CDFB134B1B78432B04D154E9EC
:1022400036211148FFF7C4FB002344F8DC3C19B0E9
:10225000BDE8F08F0D486AE7099297E76146A0E76D
:1022600021464846FFF7B4FBC4E700BF11A10608AA
:1022700040A200208096184B28AB0020B8A1060889
:10228000D8A10608DC220020FCA106086FA10608E0
:102290006C35002079A10608FBA3060888A1060872
:1022A00037B52B4D2B48FFF7B1FA95F8DD33002BEE
:1022B0004CD0294C2948FFF7E1FA94F8F4302BB1BF
:1022C00094F8F63013B194F8F53073B994ED400AF0
:1022D00023488DED010AFFF799FAB5F8D03F9DED3F
:1022E000010A33BB1F48FFF7C9FAB4F8F8101E48BB
:1022F000FFF710FB94F8F43013B31C48FFF7BEFA55
:10230000B4F8FC101A48FFF705FB94F8F630CBB18F
:102310001648FFF7B3FAB4F8FA101648FFF7FAFABE
:1023200094F8F53083B1114803B0BDE83040FFF7B1
:10233000A5BA4AF0B1FB81B20F48FFF749FBD4E7D9
:102340000E48DBE70D48E4E70C48EDE70C48EBE707
:10235000309A002026A20608E01400103CA20608CD
:1023600043A206085DA206086CA206088CA2060815
:102370009CA20608B6A2060867A2060895A206084F
:10238000BEE106082DE9F04F6E4B1B7887B0002B9D
:1023900000F0D1806C4D6D48A968DFF8F4A1FFF71B
:1023A00017FB69686A48FFF713FB6A4B6A48D3E971
:1023B0000031C91A694B53F8D02CB1FBF2F2FFF788
:1023C00007FBFFF743FA6648FFF758FA6548FFF73F
:1023D00055FA4FF00008644B1B785FFA88F4A3426B
:1023E00022D8624C624FFFF731FA2646002556F894
:1023F000041B38460135FFF78DFA162DF7D1FFF78C
:1024000025FA5B4E0125234661681B683046C91AD0
:102410000135FFF77FFA162D04F10404F3D107B05C
:10242000BDE8F04FFFF712BA524B142603EB8403BA
:1024300006FB045693ED450AB6F80E904AF02CFBC5
:1024400096F81EE01EF0010F14BF52222D221EF03E
:10245000020F14BF54232D231EF0040F07EE903AF1
:1024600014BF56232D231EF0080F14BF4FF0430C4A
:102470004FF02D0C81B21EF0800F4FF03C0BB1FBE2
:10248000FBF105914FF0640114BF4FF0530E4FF074
:102490002D0E80B201FB09F1671CCDE902E100932A
:1024A000049017EE903ACDF804C039465046FFF735
:1024B00031FAB37FDB073AD55C232F4A6343D11847
:1024C000D05891ED010A70B1DFED2C7AB8EE400AD8
:1024D00020EE270A07EE900AF8EE677A80EE270AC8
:1024E0004AF0DAFA00B2642290FBF2F102FB110228
:1024F0002348FFF70FFA142101FB075701FB04548F
:10250000F988628A0491218B0391E18A0291A18B5F
:102510000191A18A009102F0030319214B4319484C
:10252000218A9208FFF754FA08F1010853E7164888
:10253000FFF76CF9DFE7154807B0BDE8F04FFFF78C
:102540009DB900BF0400001020090010D6A20608A3
:10255000E6A2060834060010FDA2060828AB0020FB
:102560002AA3060886A30608C00D0010CC09001097
:1025700036A40608E01400104006001000401C4677
:10258000FFA3060814A406080BA406083AA406082C
:10259000E2A306080EB403B503AA52F8041B019285
:1025A000FDF771FB064BD3F8FC261AB90549186DE7
:1025B000FCF70CFE02B05DF804EB03B0704700BFFF
:1025C000309A0020EFA906082DE9F04798460B79CC
:1025D00003F0E004402C81460F46164631D1684D89
:1025E000DFF8A081DFF8C091002422E03B7903F0FE
:1025F0000703013B042B04D8DFE803F006080B0EA9
:102600002000315D28460AE03157FBE736F8141008
:10261000F8E736F91410F5E756F824104046FFF7AE
:1026200079F97B79013BA34202DD4846FFF7EEF8DA
:1026300001347B79A342D9DCBDE8F08756F8241039
:10264000E0E703F00703052B58D8DFE803F0030C9D
:10265000141619313578602C5ED045D8002C66D020
:10266000202C7CD0E8E796F90050602C54D03BD861
:10267000002CF5D148E03588EDE7B6F90050F4E7D5
:10268000D6F800A0202C554669D02BD8002CD3D1E9
:1026900051463C48FFF73EF9D7F805108A4518D84F
:1026A000B8F1000FC8D03848BDE8F047FFF732B99D
:1026B000202C356853D015D8002CBDD12946304880
:1026C000FFF728F9D7F80510A94202DB4B42AB42CD
:1026D000E6DDFFF7BBF83A682C492B464846BDE8D3
:1026E000F04757E7602C17D0802CA5D13178284BC4
:1026F0002848002914BF31461946D5E7202C2DD093
:1027000007D8002C98D12546B7F90540B7F90760DE
:1027100011E0602CE8D100257B7945FA03F3DB0753
:10272000BDE8F0474CBF1C481C48FFF7F3B8B7F8AA
:102730000540B7F8076012482946FFF7EBF8AC42AE
:10274000C7DCAE42C5DBB8F1000F3FF475AF3246CF
:1027500021461348BDE8F047FFF7DCB800257A7939
:10276000104B03EBC20393F828249542B1DAD3F857
:10277000243453F82500BDE8F047FFF747B800BF01
:102780000B9D0608F49C060856A406085CA40608DF
:102790000DCB0608EDB306085C9D0608BEE10608F1
:1027A00068AD060864F30508229F060813B50446C1
:1027B000084601920091FCF7F9FBDDE9001302469F
:1027C000204602B0BDE81040FEE60EB403B503AAF1
:1027D00052F8041B0192FDF756FA054B0549186D96
:1027E000FCF7F4FC02B05DF804EB03B0704700BFE7
:1027F000309A0020EFA906080049E6E776A406080B
:1028000038B50C46054615492046FDF7A5FB30B9FD
:10281000FEF7C6FF1248BDE83840FFF72FB8114950
:102820002046FDF799FBA8B90F4A82F8AE0182F85D
:10283000B60182F8520282F85A0282F8F60282F851
:10284000FE0282F89A0382F8A203084A82F8210065
:102850000748E0E72846BDE83840CDE785A40608EC
:102860008BA40608A6A40608309A002094370020FE
:10287000AEA4060801490246A7E700BFCAA406089D
:10288000F8B5064608460C46FDF7A2FC2021054691
:1028900020464AF0F3FE044618B93046BDE8F84039
:1028A000E8E7114F114E3B7832789A4201D0FBF79E
:1028B00093FB0F4B20461D6048F0DAFB01220146D6
:1028C0002046FBF731FB3B7832789A4201D0FBF788
:1028D00083FB204648F0CCFB2A460146BDE8F84081
:1028E0000448FFF775B800BF28210020D42F00202E
:1028F00024210020E1A406082DE9F041064688B015
:1029000008460D46FDF764FC2021044628464AF09F
:10291000B5FE20B9304608B0BDE8F041AAE7FDF7A2
:1029200057FC2246054601460F48FFF751F885B18E
:10293000202D2A46694628BF20222046FBF768FB47
:10294000E84606460027B74208DBAD1B3444002E9C
:10295000EDD1FEF77BFF08B0BDE8F08118F8010B60
:10296000FEF7B6FF0137EEE7F7A406082DE9F043BE
:10297000064687B008460C4648F07AFB082843D143
:10298000671E03AD073429463A46A84612F8010FE0
:10299000FDF7DCFAA24201F8010BF7D10023DFF8C2
:1029A0007C908DF8143017F8010FFDF7CFFAC1B203
:1029B00005F8010B484601914AF060FE20B10199EB
:1029C00028464AF05BFE28B13046FFF715FF07B0F6
:1029D000BDE8F083A742E6D10F4940462CF040FF06
:1029E0000D480E49082310F8012B11F8014B18323D
:1029F0006A44013B02F80C4CF5D109488DF81430BB
:102A000003A9FEF7E5FFE2E70028E9D0304607B06A
:102A1000BDE8F0432EE700BFEC9D0020FC680608EF
:102A20000FA5060807B5009313460A460249FFF7AB
:102A3000CCFE03B05DF804FB16A5060810B50446ED
:102A40000748FEF71BFFFBF731FE20B1BDE8104041
:102A50000448FEF713BF20460349BDE81040B4E622
:102A60002FA5060839A5060841A506082DE9F0415D
:102A7000144B1B6888B00446F3B11A6804A9D56AE0
:102A800018466A46A847064688B1DFF8448004AC79
:102A90006D46002735F8022B34F8021B40460137FB
:102AA000FEF796FFBE42F5DC08B0BDE8F0810649AE
:102AB0002046FFF78AFEF7E7044908B0BDE8F04179
:102AC00083E600BFC437002062A506087AA5060881
:102AD00048A5060813B504460846019148F0C8FA0F
:102AE000024670B1102804D1019909484AF0ECFD62
:102AF00038B1074B074A0849204602B0BDE81040EC
:102B000063E60349054802B0BDE81040FEF760BF28
:102B100081A5060892A506089DA50608C7A5060872
:102B200013B504460846019148F0A2FA01990246FD
:102B300068B1042803D109484AF0C6FD38B1074BF3
:102B4000074A0849204602B0BDE810403DE6034967
:102B5000054802B0BDE81040FEF73ABFD5A506080B
:102B6000DAA506089DA50608EAA506082DE9F043A2
:102B700006469BB008460C4648F07AFA0027054600
:102B80001C22394602A801974AF061FD25B3402D69
:102B900007D03A4940232A4630461BB0BDE8F043EF
:102BA00013E60DF1040804F14009022221466846AB
:102BB0004AF09EFD0023102209A968468DF8027094
:102BC000FDF73EFA099B0DF10202934221D1023436
:102BD000A14508F8010BE8D100213D220AA809917E
:102BE00009AC4AF034FD002D3AD0254B1D78C5B113
:102BF0002449202201A84AF000FD90B12046214935
:102C0000FDF71AF9204A214923463046FFF7DDFD3A
:102C100004E01A781E493046FFF7D7FD1BB0BDE827
:102C2000F0831C4B1B79DBB9D5B9164A01AD2B4695
:102C300003CBA342106051601D4602F10802F6D199
:102C4000154B10490122204603F8CC2CFDF7F4F86F
:102C50001248FEF719FE12482146FEF7B9FEDDE7DD
:102C60000D4B13F8CC3C1BB9054B1B78002BF2D055
:102C700004492046FDF7E0F8EDE700BFFDA5060892
:102C8000082700200C2700203BA606089DA5060863
:102C90001FA60608309A002028AB002045A606088B
:102CA00054A606082DE9F74F834608460D4648F01E
:102CB000DFF9364F0446D7F80090B8B93448354D9F
:102CC000354FFEF7A3FD012655F8041B49B106FA5E
:102CD00004F313EA090F02D03846FEF71BFE013455
:102CE000F2E703B0BDE8F04FFEF7B0BD02462B4956
:102CF0002846FDF755F978B92948264C294DFEF7A5
:102D000085FD54F8041B0029EBD00B78002BF8D07C
:102D10002846FEF7FFFDF4E72B782D2B1D4B03BF54
:102D2000013504F1FF344FF0010A4FF0000A00268C
:102D300053F8048BB8F1000F06D11B492A465846B8
:102D400003B0BDE8F04F40E52246414628460193D6
:102D5000FDF726F9019BB0B90123B340BAF1000F8A
:102D60000CD029EA030311483B60FEF74FFD0D48E4
:102D7000414603B0BDE8F04FFEF72ABE49EA03031F
:102D80000B483B60F1E70136D2E700BFF43B00207F
:102D900061A60608C4FA05086BA6060874A1060811
:102DA0006FA60608EBA006087AA606088BA60608FA
:102DB00094A606082DE9F74F814608460E461746A9
:102DC000984648F055F90446E8B93F483F4DFEF7AC
:102DD000A1FD20460FF0EEF83B68184206D02046D1
:102DE0000FF0FAF801462846FEF794FD0134182C3E
:102DF000EFD13B6813B93648FEF708FD03B0BDE8D4
:102E0000F04FFEF723BD024632493046FDF7C8F8C1
:102E10000546A8B93048FEF7F9FC2C462F4D204650
:102E20000FF0C8F810EA080F06D020460FF0D4F8CB
:102E300001462846FEF76EFD0134192CEFD1DDE77F
:102E400033782D2B48F0807303BF013604F1FF3433
:102E5000012500254FF0000A019350460FF0BCF801
:102E60002246834601463046FDF79AF800BB50469D
:102E70000FF0A0F8019B03421AD08DB1BAF1180FE0
:102E80001CBF3B6840EA03081548C7F80080FEF7FE
:102E9000BDFC1248594603B0BDE8F04FFEF798BD9F
:102EA000BAF1180F1CBF3D6885433D600D48EEE741
:102EB0000AF1010ABAF1190FCFD10B49324648463F
:102EC00003B0BDE8F04F80E49CA60608EAA006081F
:102ED000A6A6060874A106086FA60608EBA00608B9
:102EE0008BA6060894A606087AA60608014A40F2B0
:102EF00002235FE764370020014A6FF07F4359E700
:102F00005C37002008B50A4B13F8C82C032A0AD1F5
:102F100013F8C73C092B06D12CF02AFDBDE8084068
:102F20000448FEF755BDBDE8084003494DE400BF25
:102F300028AB0020ADA60608B8A6060870B5054661
:102F400008461646FDF744F90C4B1A7890420446A1
:102F500005D201460A48FEF73BFD204670BD2EB162
:102F6000FF2803D10748FEF733FDF6E70649013A8B
:102F70002846FFF72AFC4FF0FF34EEE7C00D0010A3
:102F8000C7A60608D8A60608EBA606082DE9F04F46
:102F9000074691B08248834D0E46FEF719FD8249DF
:102FA00045F8A8DC002305F8A43C06220123097893
:102FB0003046402405F8A34C0AF0ECFC0A200AF045
:102FC00085FD15F8A43C0C2BDAB240F2E4809DF8A4
:102FD0000C50FE2D36D0FF2D0BBF15240F240126DB
:102FE0000026944240F0D780611EC9B268463CF08A
:102FF000C3FA04F140030DEB030414F8413C83428F
:1030000040F0C48006F1FF389DF80D3067485FFA44
:1030100088F8B8F1010F8DBF03F01F079DF80E70FF
:103020009DF80F4061378CBF5C091D46FEF7EEFB33
:10303000022E64D0013C042C5FD8DFE804F0055870
:103040005A5E5C000226CCE75948DFF8C091DFF8F1
:10305000C0B1FEF713FC5748FEF7D8FB6C464FF0A3
:10306000000A14F8011B48460AF1010AFEF752FC57
:10307000BAF10C0F49D1FEF7E9FB022E4FD06422C2
:10308000B5FBF2F102FB11524B483B46D2B2C9B23A
:10309000FEF79EFCB8F1010F71D8484A484B9DF8E5
:1030A00010104848484D002914BF11461946FEF734
:1030B0008FFC9DF81110454B4548002914BF194657
:1030C0002946FEF785FC022E59D19DF81240414851
:1030D000FEF79CFB4CB3FF2C37D00A22B4FBF2F175
:1030E00002FB11423C48D2B2FEF772FC20E03B48A2
:1030F000ABE73B48A9E73B48A7E73B48A5E70023E8
:103100008DF83F300DF11F009FE7384B03FB0AF2AB
:10311000B2F1553FA5D85846FEF778FBA1E73448F1
:103120003A462946FEF754FCB7E72846FEF7A6FBC9
:103130009DF813402F48FEF769FB44B1FF2C21D0C6
:103140002D482146FEF744FC04E02C48EEE71E48DB
:10315000FEF794FB1C4E294FDFF870800DF113052C
:10316000002415F8013F7BB1FF2B0CBF3A464246C5
:10317000214623480134FEF72BFC042CF1D111B079
:10318000BDE8F08F1D48E3E73246F1E71D493846B8
:10319000FFF71BFBF3E71C48FEF770FBEFE700BFF0
:1031A00031A7060828AB0020C00D001042A7060872
:1031B0004DA7060873A7060885A7060811A70608E5
:1031C0001AA70608BCA7060821A7060815B5060811
:1031D000D3A70608DAA70608EEA7060854A706082C
:1031E0005CA7060864A70608589E0608ABAAAAAA08
:1031F000A1A70608F6A706080B9D060825A706083E
:1032000006A8060811A8060821A80608819C060839
:103210000DCB06082DE9F84FDFF8A880DFF888907D
:10322000DFF8A4A007460C46204647F021FF0646DB
:1032300058B91D4B1D481A781D4B03EB8203D3F878
:10324000D817BDE8F84FFEF7C3BB024641462046FB
:10325000FCF7A6FE60B1DFF864B000255BF8041B44
:10326000B1B9224638461349BDE8F84FFFF7ADBA69
:103270001148124C124DFEF7C9FA54F8041B19B14B
:103280002846FEF747FBF8E7BDE8F84FFEF7DEBA41
:1032900032462046FCF784FE01350028DED189F84D
:1032A00000505446C0E700BF213600202AA8060877
:1032B00064F305087AA606086FA6060840FB050811
:1032C000EBA0060874A10608F1A9060838B50D465A
:1032D00004461A4905222846FCF762FE68B9184BD5
:1032E00093F8542022B9012183F8541083F8552013
:1032F000BDE838401348FEF7C1BA134903222846F7
:10330000FCF74EFEA0B90E4D95F8543063B195F818
:1033100055304BB10D492046FFF757FA002385F889
:10332000543085F8553038BD0948FEF7A7FAF5E75F
:1033300020460849BDE83840FFF747BA6CB4060894
:10334000309A002034A80608BEB506084AA8060828
:1033500081A8060895A80608F8B5194C94F85430C9
:1033600005467BB194F8553063B11649FFF72DFA45
:1033700028461549FFF729FA002084F8540084F8FC
:103380005500F8BD114B13F8CC5CBDB1104B18784B
:103390000028F6D10F4B104A03F120071646186893
:1033A0005968144603C40833BB422246F7D10123AF
:1033B00086F83B300BF0C0F82846E2E70120E0E752
:1033C000309A00204AA80608A4A8060828AB0020C6
:1033D000082700200C270020903C002008B5FFF7AC
:1033E000BBFF50B1054B01229A73FEF74DF804481C
:1033F000FEF74AFA0020FEF711FA08BD6C350020EE
:10340000C2A8060808B5034610462AB1DB0600D557
:1034100011B1FEF739FA002008BDF8B50C4E33792A
:1034200005468BB9F8BD25B12388C3F30B039D4234
:1034300004D0D4E90201A2884AF0A6F81C34BC42A8
:10344000F1D300233371EDE7024C034FF7E700BFE0
:10345000309A00209CE4060894ED06082DE9F74F09
:10346000064601AA08462E49DFF8C480DFF8C4905A
:10347000DFF8ACA04AF0BEF84FF0000B04465D4602
:10348000012714BBBBF1000F27D1264C002D43D0E0
:1034900025482946FEF79CFA23790BB905F08EFBE7
:1034A000FCF704F8002384F85530FEF779F915B1DC
:1034B0002846FFF7B2FF9FB13046FFF74DFF78B1C6
:1034C000FDF7E2FF0020FEF7A9F9BBF1000F0AD0DB
:1034D0002046FCF77DFE85B2C5B93046FFF78CF972
:1034E00003B0BDE8F08F41462046FCF77DFD80B972
:1034F00049462046FCF778FD0028EED05F4601AA39
:10350000514600204AF076F80446BAE74FF0000B27
:10351000F5E74FF0010BF2E70448FEF7B5F9BFE716
:1035200080AD0608309A0020D2A80608F5A8060843
:10353000C9A80608A3B406082DE9F04F85B01646C1
:1035400001911A46824600213046FFF75BFF324C5C
:1035500006F0100305464FF000090293FEF73AF912
:103560002379019A03F01803934203D0002A48D12B
:10357000182B46D1284B4FF00D0B0BFB0933B3F83A
:103580000900FBF73BF980462046FBF7DAFCD8E957
:1035900002210746024401442046FBF78BFC80F0E1
:1035A00001012A460390C9B23046FFF72BFFDDE93F
:1035B0000223054602B123BB174A0BFB09FB52F855
:1035C0000BB0B2060FD573B9144803935946FEF7F2
:1035D000A1F9D8F80820039B3A4421465046FEF74B
:1035E000F3FFFEF733F90E485946FEF793F9D8F882
:1035F0000C2000233A4421465046FEF7E5FFFEF733
:1036000025F909F1010940F26923994504F10D04F6
:10361000A4D105B0BDE8F08FD40306080BA90608B5
:103620000CA9060820B10078B0FA80F04009704774
:10363000012070472DE9F34106460846FFF7F2FFE7
:103640000D46074670B1002401A9204642F048FB10
:10365000013401463046FFF7EDFF122CF4D102B0E1
:10366000BDE8F0810846FCF7B3FDC4B2112C72D856
:10367000681CFBF7BDFD3C4D8046E8B93B4B03EBB6
:10368000440313F8A01C8A1E51425141374B03EBEF
:10369000440313F8A02CAA5C002955D013F89F3CD2
:1036A000192040F2EE2100FB03133148214602B0FD
:1036B000BDE8F041FEF78CB90178284649F0DEFFFD
:1036C00070B1032C94BF002201222A4902EB42026E
:1036D000431B0A4452FA83F393F84878032F05D129
:1036E000304602B0BDE8F041FFF786B84046FBF730
:1036F0007FFD08B3022FF3D1FCF76AFD40F6CA0242
:1037000080B29042194BA8BF104640F2EE22904280
:1037100003EB4403B8BF1046A0F2EE201922B0FB21
:10372000F2F003F89F0CBB1E594259410F4B03EBBB
:10373000440303F8A07CA9E7022FF4D1304602B07D
:10374000BDE8F041FFF796B80B48214602B0BDE84E
:10375000F041FEF73DB9094911233A46304602B01F
:10376000BDE8F041FFF75EB9F86A060828AB002013
:1037700016A9060864F3050826A9060833A9060851
:103780002DE9F04F024691B00846FFF74BFF0B467C
:10379000044628B1104611B0BDE8F04FFFF76AB8F3
:1037A0004FF0FF32CDE90820A64ADFF8E082D26C64
:1037B000DFF8DC9292F83810DFF8D8A2CDE90C10CF
:1037C000CDE90E02CDE90A009F4907AA184649F043
:1037D00011FF27460546049426464DB9089A0C9FCA
:1037E000BA4262D19948FEF7F3F811B0BDE8F08F04
:1037F000062F12D8DFE807F0041E2328454C51009D
:1038000051462846FCF7F0FB78B14FF480600EF08B
:1038100041FE90F90430089301248B4907AA002047
:1038200049F0E8FE01370546D7E72846FCF7D0FC0B
:103830000890F2E72846FCF7CBFC0990EDE7284614
:10384000FCF7E9FB0A90E8E7284647F011FC4146FF
:10385000024605902846FCF7A3FB18B3059A494693
:103860002846FCF79DFB06460028D6D02846FCF7E4
:10387000AFFC04280646D0D901467548FEF7A8F8E3
:10388000B3E72846FCF7A4FC00230C900F93C4E791
:103890002846FCF79DFC0D90BFE72846FCF7BBFBD4
:1038A0000E90BAE701230493B7E7DFF8EC8151B239
:1038B000434613F9010B884208D00135092DF8D190
:1038C000002164480131FEF783F88EE76248012148
:1038D000FEF77EF87AB2002318F9011B8A4200F045
:1038E0000C810133092BF7D13A460121E9E7A7F111
:1038F000140253425341059308AD002303F101081C
:10390000EB68A3BB95F900B058460EF08BFDD5F8D7
:1039100004A020B1D0F80090B9F1000F5ED1BAF147
:10392000000F19D14FF461436B604FF0010AAB688F
:103930000BB90323AB600023D5F8049002932A7AD5
:103940001946CDE9009258461A460EF0A5FEE860E9
:1039500028B94248414691E74FF0000AE7E74A4656
:103960004146BAF1000F37D03D48FDF7D3FFB8F11B
:10397000020F05F110054FF00103BFD1059BDDF8E3
:103980003C800B9D53B13748FDF778FFD8F80030E5
:103990001B6A1BB134492A4640469847049B002BBA
:1039A0004ED03249324B142F18BF19463148FEF71A
:1039B0000FF8142F09D1049B03B936B12B68DB69CA
:1039C0001BB12D49324628469847002C66D100226B
:1039D0004146284642F038F92848C6E7C5F80C9019
:1039E000BAF1000F25D0264841465246FDF792FF16
:1039F0005146484603F0ECFCD5F808A0BAF1000F98
:103A00000FD099F8042092450BD01E4853464146EA
:103A1000FDF780FFD9F800305FFA8AF19B694846CC
:103A20009847D9F82C30002BA1D00023C9F82C30AE
:103A30009DE7D9F8082014484146FDF76BFFDBE706
:103A40000B49B3E7309A002080AD060871A906083B
:103A500059A90608B5AA06088AA9060896A906085B
:103A6000B2A9060869AA0608D17301083BA906088D
:103A7000F1A9060892AA06080BF20008D6A90608C2
:103A8000F2A9060844AA06081FAA060853A90608B0
:103A9000A8A6060848A906081CEB050806F062FB64
:103AA00005200AF013F81A4FDFF86C9000264FF04B
:103AB000030A99F80030B34289D917F801BBBBF16A
:103AC000000F15D058460AF0D1FB044680B1584685
:103AD00006F080FA08B1A0F806A001210490F7F7DB
:103AE00091FAA379049813F0010F03D0F6F770FC54
:103AF0000136DEE7F6F766FCFAE706483A460221A9
:103B0000FDF766FF099B002B3FF4F1AE0023F2E6C0
:103B1000D82700208AA90608C00D001010B5044659
:103B200008460B46FFF77EFD28B9094903221846CF
:103B3000FCF736FA28B90748FDF7A6FE0120FDF785
:103B40006DFE20460449BDE81040FEF73EBE00BFB2
:103B5000C7AA0608CBAA060895A806082DE9F74FBC
:103B600005460846FFF75EFD0B46044618B9334A82
:103B700012F87C7C2FB9284603B0BDE8F04FFEF761
:103B80003BBE2F49DFF8C480DFF8C490DFF8C4A043
:103B900001AA184649F02EFD264610B906F0F0FAA3
:103BA00008E056B9012201462846FFF7C7F9421C32
:103BB00004461AD103B0BDE8F08FFCF709FB2F28AB
:103BC000834634D80FB106F0CDFABBF1060F13D0FF
:103BD0001C49012309785FFA8BF2E0B209F0DAFEA2
:103BE00059464846FDF7F4FE0027154901AA002072
:103BF000013649F0FFFCD0E7DAF800301B0112D59E
:103C0000FF2C0ED0E1B22846FFF7C0F9E8E72846BE
:103C1000FFF7BCF901370B4B1A78F9B28A42F6D894
:103C2000DEE70027F7E70848FDF728FED8E72F2250
:103C300041462846FEF7C9FDD7E700BF28AB002064
:103C400080AD0608C00D0010B8A60608FEAA06083A
:103C5000EDAA0608A83500202DE9F04F064685B0EC
:103C60000846FFF7DFFC0B46044628B1304605B096
:103C7000BDE8F04FFEF7FEBD3049DFF8D090DFF829
:103C8000D0A0DFF8D0B003AA184649F0B3FC27460D
:103C90000546A0465DB92A4B3A46D86CA1B241F020
:103CA00055FD68BB27493046FEF78FFD28E0B8F187
:103CB000000F06D0B8F1010F25D03046FEF7DAFD2F
:103CC0001EE0284647F0D4F94946024601902846AE
:103CD000FCF766F950B3019A51462846FCF760F9A3
:103CE00030B3019A59462846FCF75AF910B3019AA5
:103CF00015492846FCF754F9F0B13046FEF77CFD33
:103D000005B0BDE8F08FBB1E5A425A4129463046E5
:103D1000FFF714F9421C0446F2D0084903AA002018
:103D200049F068FC08F101080546B3E74746F4E7A7
:103D30000127F2E70227F0E70427EEE780AD060847
:103D4000309A00202AAB060827AB06081EAB0608EF
:103D500021AB060824AB06082DE9F7438046084648
:103D6000FFF760FC0B46054628B14046FEF782FD92
:103D700003B0BDE8F0832E49DFF8B49001AA1846DD
:103D800049F038FC2F4604462E467CB9022DECD172
:103D9000A7F57A73B3F57A7F21D926494FF4FA63F0
:103DA0004FF47A724046FEF73DFEE1E74DB1012D3A
:103DB00010D001AA4946002049F01CFC01350446F8
:103DC000E3E7012221464046FFF7B8F8431C0646C8
:103DD000EFD1CDE72046FCF7FBF90746E9E7164BA4
:103DE0001B68B8B25B689847FF2EBCEEC00A0CD1C6
:103DF000124BF8EE407A1A78114BA24213DC10EE07
:103E0000101A1048FDF7E4FDB2E70F4B0F48F8EE2B
:103E1000407A03EB860310EE102A43ED1E7A3146FA
:103E2000FDF7D6FDA4E7E3EC017A0134E5E700BF36
:103E300080AD060838AC0608DC140010C00D001078
:103E4000B0AA002055AB060828AB002048AB0608F6
:103E5000F8B507460846FFF7E5FBC8B11F4B5E699A
:103E6000013630460EF0B8F834460546F0B9013454
:103E7000192CA8BF002420460EF0AEF80546A8B9BC
:103E8000B442F4D138461649BDE8F840FEF79DBC6F
:103E90000846FCF79DF904460EF09EF8054628B941
:103EA00021461048BDE8F840FDF792BD0B4B5C6120
:103EB0000EF0B8FC0C4821462A46FDF789FD182C67
:103EC0009DBF0A480C2101FB04000020BDE8F8401A
:103ED00098BF90F850080EF0DBBC00BF940500209E
:103EE00064AB060878AB06088EAB060864F30508D9
:103EF00038B5124D04460846FFF794FB60B1104BED
:103F0000104893F900104B1C0ABF0F4BC9B2197827
:103F1000BDE83840FDF75CBD0846FCF759F90328B9
:103F200004D8C0B2FDF7CAF82946E4E7204607499D
:103F3000BDE838400322FEF748BC00BFF1A90608DF
:103F400094050020A7AB06086C350020B7AB060827
:103F500038B5124D04460846FFF764FB60B1104BBC
:103F6000104893F901104B1C0ABF0F4BC9B2597886
:103F7000BDE83840FDF72CBD0846FCF729F90328B9
:103F800004D8C0B216F0C8FC2946E4E72046074929
:103F9000BDE838400322FEF718BC00BFF1A90608AF
:103FA00094050020A3AB06086C350020B2AB0608D0
:103FB0002DE9F74F444BDFF82CA11A785B788AF88B
:103FC0000130424B8AF800201B79054688460BB920
:103FD00004F0F4FDFBF76AFA00263D4CB1460D23D0
:103FE0003B4A7343414652F803B05846FBF7FCFF87
:103FF000002841D0B9F1000F01D0FDF727FC35486A
:104000005946FDF787FC002221462846FEF7CEFBE5
:10401000FDF71CFC237903F01803082B46D0102B66
:1040200049D02046FDF7E3FC294A0D2303FB062374
:10403000B3F80900FAF7E2FB0746D8B12046FAF7D1
:1040400080FFD7E902210090024401442046FAF79C
:1040500031FF78B9019059461F48FDF75BFC019A82
:10406000B9681346009A28460A442146FEF7ACFA7E
:10407000FDF7ECFB09F10109013640F269239E428C
:1040800004F10D04ABD10020FFF7C7F9FF238AF834
:1040900000308AF80130B9F1000F11D10F494246C2
:1040A000284603B0BDE8F04FFEF78FBB0C49284609
:1040B000FFF71EFFB5E70A492846FFF749FFB0E7BB
:1040C00003B0BDE8F08F00BF6C350020309A0020AF
:1040D000D403060810A90608D2AB06087AA606087B
:1040E000F1A90608940500202DE9F74F0746084678
:1040F0000E4646F0BDFF044620B1012826D1327895
:104100002A2A23D1B348B44EDFF8E892FDF7B6FB74
:104110000025B2464FF00D0B40F269280BFB05F36A
:1041200048465AF80310FDF7F5FB221E18BF01227E
:10413000314638460135FEF739FBFDF787FB45452B
:1041400006F10D06EAD103B0BDE8F08F3D213046FF
:1041500049F094FA002800F0378101460A4611F828
:10416000014D202CFAD0921B0130814610F8011B22
:104170002029FAD0DFF860B25FFA82FA4FF0000827
:104180000D2303FB08F10BEB010452465BF8011011
:1041900000913046FBF704FF0546002857D10099EF
:1041A000084646F065FF824551D1267906F0E001C8
:1041B000402900F0CC800ED8002956D0202900F0EC
:1041C0009E8038468549FEF700FB204603B0BDE8D7
:1041D000F04FFDF70CBC602900F092808029F0D1EF
:1041E000484646F045FFE379A679DB0705460CD53E
:1041F0002046FAF7DBFE0378014633B12A464846EB
:1042000049F062FA002840F0D980002D00F0D680F5
:10421000AE42C0F0D3800D2303FB08B3204693F8D1
:1042200005A0FAF7C3FE3246002149F010FAAA456C
:104230002CD86B492A46484649F046FA30B3204606
:10424000FAF7B4FE2A46494649F09EF91EE008F105
:10425000010840F26923984592D1624932463846B6
:1042600003B0BDE8F04FFEF7B0BA06F00703042B29
:104270001CD10B460A224846FBF7E2FED4F8053073
:10428000834201469DD32046FAF7A4FE0D2303FB8B
:1042900008F855485BF80810FDF73CFB0022214662
:1042A000384603B0BDE8F04FFEF780BA052B0FD1BA
:1042B00001230A224846FBF7C3FED4F805308342A7
:1042C0000146FFF67EAF5B4283423FF77AAFDAE703
:1042D0004846FBF77DFFB4F80550B4F8071016F018
:1042E000050FAAB218BF2AB28BB218BF0BB2904208
:1042F000FFF667AF98423FF764AF0146C3E76579C1
:104300003A4A02EBC505002695F828240092B246E9
:104310003346009AB24202D9BAF1000F03D0002B03
:104320003FF44FAFB2E7D5F8241451F8260060B13E
:1043300049460193FBF710FE019B30B931462046F8
:104340004FF0010AFAF746FE53460136E1E763797A
:10435000009306F00706013E009BAB4296DD4846FF
:10436000814610F8013B202BFAD02046FAF71EFEBA
:104370008246042E04D8DFE806F0031010161F0052
:104380004846FBF725FF0AF8050048462C2149F06E
:1043900075F9013500F10109DEE74846FBF718FF22
:1043A0002AF81500F1E700230A2200214846FBF70E
:1043B00047FE4AF82500E8E70123F5E70C493246B5
:1043C0003846FEF702FAFCE63146384603B0BDE84F
:1043D000F04FEDE5E2AB0608D403060830AC060862
:1043E0000DCB06087AA6060825AC060864F3050876
:1043F000F5AB060810A906082DE9F04F914689B0E3
:104400000C461A4600218046FEF7FCFFDFF8ECB0B0
:1044100006464D460027B9F1000F6CD0294606220A
:10442000204649F0EAF80028324614BF0121002155
:1044300040460CBF4FF0010A4FF0000AFEF7E2FFC2
:104440000646287814F05CFE079010B3687914F0E3
:1044500057FE079BEA785B790793AB7895F801E004
:104460004FF461714FF0190C1CFB03131CFB02127B
:10447000297900B14079CDF804E0CDE90232079BFB
:104480000093CDE904103B465A4651464046FDF79D
:1044900029FA207814F034FE079010B3607914F0F4
:1044A0002FFE079BE2785B790793A37894F801E0ED
:1044B0004FF461714FF0190C1CFB03131CFB02122B
:1044C000217900B14079CDF804E0CDE90232079BB3
:1044D0000093CDE904103B465A4651464046FDF74D
:1044E000B9F90137142F04F1060405F1060592D13C
:1044F00009B0BDE8F08FCA46CBE700BF3EAC060866
:104500002DE9F041064686B00846FFF78BF80F46C6
:10451000054638B100235D491A46012006B0BDE8C2
:10452000F04169E70846FBF753FE1328044600F301
:10453000A38006264643781C8DF81750FAF758FEDC
:10454000534D074670B1FBF743FEC0B214F0EEFDC9
:1045500040B1AB19027983F808259DF81730013373
:104560008DF817303846FAF743FE074668B1FBF777
:104570002FFE0D2809D8062303FB045383F80905F1
:104580009DF8173001338DF81730DFF80081B11C2A
:104590000DF1170241443846FBF71EFEFAF728FEDC
:1045A000074668B1FBF714FE012809D8062303FB70
:1045B000045383F80C059DF8173001338DF817303C
:1045C0003846FAF715FE80B1FBF702FEC0B214F0D0
:1045D000ADFD50B1062303FB0453027983F80D258A
:1045E0009DF8173001338DF817309DF81720042AF5
:1045F0004FF006032FD103FB04530022A3F80C2530
:104600001FF0C2FA062303FB04554FF4617695F8B8
:10461000080514F075FD95F80B2595F80A75192312
:10462000804695F80D0513FB076713FB026614F02F
:1046300067FD437998F80520039395F80C350097AA
:10464000CDE90163134895F809352146FDF7C0F916
:1046500006B0BDE8F081052A05D103FB0453002212
:1046600083F80D25CCE7062A1FBF08EB06020023BE
:1046700048F806309380C3E7074913232A4630469B
:1046800006B0BDE8F041FEF7CDB900BF389F00206D
:10469000309A00203EAC060857AC06082DE9F04FD2
:1046A000174689B01A460C4600218146FEF7AAFE3D
:1046B0003B4EDFF8F4B007F16C0380463D460793AC
:1046C00094F90410374A002392F90800884263D015
:1046D0000133092B02F10C02F6D1079B0C359D42E8
:1046E00004F10C04ECD109B0BDE8F08F29460C228E
:1046F000204648F082FF0028424614BF01210021D5
:1047000048460CBF4FF0010A4FF0000AFEF77AFE50
:10471000EA7995F9043006EB82028046D2F88026C9
:1047200004922A7A06EB82025146D2F8802603923E
:10473000AA7906EB82024846D2F8802602926A796C
:1047400006EB8202D2F8802601922A6800925A462D
:10475000FDF7C8F8E27994F9043006EB820251467D
:10476000D2F880260492227A06EB82024846D2F8DA
:1047700080260392A27906EB8202D2F8802602926A
:10478000627906EB8202D2F88026019222680092BA
:104790005A46FDF75FF8A0E7002FA7D1BA46D9E740
:1047A00064F30508B03500205DAC06082DE9F04340
:1047B00080468BB00846FEF735FF38B100234D49DF
:1047C0001A4601200BB0BDE8F04367E7CDE90700CA
:1047D000099008464D1CFBF7FBFC44B220460DF047
:1047E000DDFD0646002843D08DF8204001242846F0
:1047F000FAF7FEFC054638B100230A221946FBF7FA
:104800001FFC01340790E4B2DFF8F090002728463F
:10481000FAF7EEFC054618B3FBF7DAFC364900223E
:1048200051F804CB6045D3B203D00132102AF7D13E
:10483000002309EB8302D2F88026904210D1022F88
:104840001DD0032F20D05A1E012FD2B212D00B2A16
:1048500003D88DF821300134E4B20137042FD6D1CA
:10486000052C17D840460BB0BDE8F043FEF702B860
:104870000446BCE7042AF0D88DF82230EBE7052B7C
:10488000EBD88DF82430E6E79A1E0D2AE5D88DF88E
:104890002330E0E707AB03CB9DF823203060186896
:1048A000164B716003EB8202B060D2F8802604924E
:1048B0009DF8242003EB82020021D2F88026039287
:1048C0009DF8222003EB82020846D2F8802602924D
:1048D0009DF8212003EB8203094AD3F88036019327
:1048E000079B00939DF92030FCF7B4FF0BB0BDE8A7
:1048F000F08300BF249E0020E4F9050864F3050856
:104900005DAC06082DE9F04F8BB00C4608920021F3
:104910001A460746FEF776FDDFF8B4B0089D099009
:1049200000264FF019094FF46178089B002B4BD0FB
:1049300029460A22204648F060FE0028099A14BF42
:104940000121002138460CBF4FF0010A4FF0000A48
:10495000FEF758FD2A890692EA8805922A79049280
:10496000EA780392AA78099019FB028202926A7887
:1049700019FB028201922A78009233465A46514628
:104980003846FCF7AFFF22890692E2880592227929
:104990000492E2780392A27819FB02820292627872
:1049A00019FB0282019214F80A2B009233465A46F0
:1049B000514638460136FCF74DFF1E2E05F10A051B
:1049C000B3D10BB0BDE8F08FDDF820A0DBE700BF6E
:1049D0007AAC06082DE9F04380468BB00846FEF716
:1049E00021FE0F46044638B1002365491A460120CE
:1049F0000BB0BDE8F04385E70846FBF7E9FB1D284F
:104A0000054600F3B3800A264643781C8DF82740FC
:104A1000FAF7EEFB044630B1FBF7DAFB9DF82730DE
:104A200001338DF827302046FAF7E2FB554C074654
:104A300068B1FBF7CDFB0D2809D80A2303FB05431A
:104A400003F8580C9DF8273001338DF82730DFF834
:104A50003091711C0DF1270249443846FBF7BCFB2D
:104A6000FAF7C6FB074668B1FBF7B2FB222809D864
:104A70000A2303FB054303F8550C9DF82730013347
:104A80008DF827303846FAF7B3FB074668B1FBF7D5
:104A90009FFB0D2809D80A2303FB054303F8540C98
:104AA0009DF8273001338DF827309DF82730062BED
:104AB0000CD009EB0602002349F80630404653604B
:104AC0001381FDF7D7FE0BB0BDE8F0830A2606FB85
:104AD00005460023384626F8523C26F8503CFAF7A3
:104AE00087FB074640B1FBF773FB9DF8273026F89C
:104AF000520C01338DF827303846FAF779FB58B15C
:104B0000FBF766FB0A2303FB054323F8500C9DF8D3
:104B1000273001338DF827301B4B4FF0FF325A609E
:104B20000A2202FB05424FF4617032F8503C0693B2
:104B300032F8523C059312F8543C049312F8553C59
:104B4000039312F8561C192313FB0101029112F86A
:104B5000571C13FB0103019312F8583C00930021EA
:104B60000A4A2B460846FCF775FEACE708491D23A8
:104B7000224640460BB0BDE8F043FDF753BF00BFEF
:104B8000D0AA002028AB0020940500207AAC0608AB
:104B900057AC06082DE9F04F2DED088BDFF82CA15E
:104BA00095B0804691461F460C4616464FF0000BC6
:104BB00094ED008AB5EE408AF1EE10FA7FD0D4ED84
:104BC000019A94ED029AD4ED038AB9F1000F49D00D
:104BD000D6ED00BA96ED01BAD6ED02AA96ED03AA7B
:104BE000B4EE6B8AF1EE10FA6ED1F4EE4B9AF1EE60
:104BF00010FA69D1B4EE6A9AF1EE10FA64D1F4EECB
:104C00004A8AF1EE10FA0CBF012100213A460D4606
:104C1000404681F00101FEF7F5FBB0EE6B0A074656
:104C200011A8FAF763FAB0EE4B0A07900EA8FAF74C
:104C30005DFAB0EE6A0A06900BA8FAF757FAB0EEE2
:104C40004A0A059008A8FAF751FA0599069A079BAF
:104C5000039002910192009352465B4629464046DA
:104C6000FCF740FEB0EE480A11A8FAF73FFAB0EEA2
:104C7000690A05460EA8FAF739FAB0EE490A069015
:104C80000BA8FAF733FAB0EE680A059008A8FAF70D
:104C90002DFA069B059A0390CDE9005302925B46DC
:104CA0005246002140460BF1010BFCF7D3FDBBF14E
:104CB000080F04F1100406F110067FF479AF15B067
:104CC000BDEC088BBDE8F08F00219FE79DAC060886
:104CD0002DE9F74FDFF89891DFF8988105460F46E8
:104CE0003846FEF79FFC064638B1002359491A465C
:104CF000012003B0BDE8F04F4CE705224946384695
:104D0000FBF74EF960B9534B00221A601A611A6220
:104D10001A631A641A651A661A6703B0BDE8F08F41
:104D20004D4904223846FBF73BF904463846002C2F
:104D300044D1FAF75DFA83460028EED046F098F9A0
:104D4000464BC2B253F804ABBAF1000F07D1444945
:104D50003A46284603B0BDE8F04FFDF736BD514650
:104D60005846CDE90023FBF71BF90134DDE90023A8
:104D700006460028E6D1374A03461746002101338C
:104D8000082B42F8101BFAD108EBC403D3F804C077
:104D9000BCF1000F03D018F834E0764505DB31484C
:104DA000314F5146FCF714FE9AE70CEB06130FCB7C
:104DB00007EB061484E80F000136EEE7FBF708FA6C
:104DC000072804463DD83846FAF712FA064658B383
:104DD000F9F7A8FF1F4B03EB041383ED000A01272B
:104DE0003046FAF705FA064638B1F9F79BFF194B3A
:104DF00003EB041383ED010A01373046FAF7F8F9A3
:104E0000064638B1F9F78EFF124B03EB041383ED1E
:104E1000020A01373046FAF7EBF938B9284603B0F1
:104E2000BDE8F04FFDF726BD0746D9E7F9F77AFF51
:104E30000848032F00EB041484ED030A3FF455AF38
:104E4000ECE70A4907233246284603B0BDE8F04F95
:104E5000FDF7E8BD28360020B1AC060840FB050888
:104E60007AA60608B6AC0608F1A9060857AC0608EB
:104E700053A9060828EB05082DE9F74F92460C4682
:104E80001A4600218146FEF7BDFADFF870B0804671
:104E900056460025BAF1000F2ED031460422204696
:104EA00048F0ABFB0028424614BF012100214846D0
:104EB0000CBF01270027FEF7A5FA738801933AF883
:104EC0002530009380462B465A4639464846FCF723
:104ED00009FD6388019334F8043B00935A462B463E
:104EE000394648460135FCF7B5FC042D06F10406A9
:104EF000D0D103B0BDE8F08F5746EAE7C0AC060852
:104F00002DE9F34105460846FEF78CFB0C460746A3
:104F100038B1002333491A46012002B0BDE8F04100
:104F2000AAE731492046FBF717F8034670B92D4A26
:104F30004FF47A704FF4FA610133042B10805180E2
:104F400002F10402F8D102B0BDE8F0812046FBF77F
:104F50003FF90328064641D82046FAF749F90746A3
:104F600070B1FBF735F94FF0010804463846FAF7FF
:104F70003FF948B9284602B0BDE8F041FDF77ABCD8
:104F800040F2EE248046F1E7FBF722F9B8F1000F7A
:104F9000F0D0A4F2EE2240F2DC539A4203D8A0F201
:104FA000EE229A420AD9114940F6CA0340F2EE2293
:104FB000284602B0BDE8F041FDF734BD0C4B0D4A68
:104FC00003EB86030021A3F8D440A3F8D600CDE973
:104FD000004033460846FCF73DFCB4E7064903238E
:104FE0003A46E5E7FCAB002053A90608D1AC060819
:104FF00028AB0020C0AC060833A906082DE9F04F05
:1050000089468FB0174600211A460646FEF7FAF980
:10501000DFF878A0054600240DF1240B59F8243060
:105020000293594602A840F0BDFD67B357F82430FB
:10503000029A0393934218BF01212A4608BF002118
:1050400030460CBF4FF001084FF00008FEF7DAF9C8
:1050500004A9054603A840F0A5FD04A90091234634
:10506000524641463046FCF73DFC2346CDF800B0A1
:105070005246414630460134FCF7ECFB202CCDD1A2
:105080000FB0BDE8F08FB846EFE700BFDFAC060811
:10509000F0B5074689B00846FEF7C4FA0E46054645
:1050A00038B1002319491A46012009B0BDE8F04083
:1050B000A4E70846FBF78CF81F2804461DD83046A5
:1050C000FAF796F80146204635F0ECFC78B10F4827
:1050D00003AE314600EB840040F064FD0C4A0096BC
:1050E000234629462846FCF7B5FB09B0F0BD3846F3
:1050F00009B0BDE8F040FDF77FBB06491F232A46F3
:10510000384609B0BDE8F040FDF78CBC0CAC00207F
:10511000DFAC060857AC06082DE9F04F924685B083
:105120000C461A4600218146FEF76CF9DFF874B090
:10513000804655460026BAF1000F31D02946042298
:10514000204648F05AFA0028424614BF01210021A7
:1051500048460CBF01270027FEF754F9EB7802936D
:10516000AB7801932B880093804633465A463946E4
:105170004846FCF7B7FBE3780293A378019334F831
:10518000043B00935A463346394648460136FCF7FD
:1051900061FB102E05F10405CDD105B0BDE8F08FFF
:1051A0005746E8E7E9AC0608F0B5074685B008467B
:1051B000FEF738FA0E46054638B100231C491A4658
:1051C000012005B0BDE8F040A6E70846FBF700F86F
:1051D0000F28044623DC3046FAF70AF80146204639
:1051E00035F0DEFBA8B1134B04F1200203EB820380
:1051F000294693F8E720029293F8E6200192B3F84B
:10520000E43000930C4A23462846FCF723FB05B004
:10521000F0BD384605B0BDE8F040FDF7EDBA0749EE
:105220000F232A46384605B0BDE8F040FDF7FABB2B
:105230008CAC002028AB0020E9AC060857AC06086F
:105240002DE9F04F87B0144603911A460021054618
:10525000FEF7D8F8DFF830B106464FF00008062315
:1052600003FB08F7C0374FF00009039BDB5D049395
:10527000002C00F08580E35D049A05939A4218BFE4
:105280000121324608BF002128460CBF4FF0010A19
:105290004FF0000AFEF7B6F8059B0646CDE90093ED
:1052A0005A46434651462846FCF71CFB049B5A4687
:1052B000CDE9009351464346284609F10109FCF720
:1052C000C9FAB9F1060F07F10107CED108F10108BB
:1052D000B8F1060FC3D1DFF8B0B0E427039BA7F104
:1052E000E40913F807A0002C4CD0E35D04939A4521
:1052F000324614BF0121002128460CBF4FF001089F
:105300004FF00008FEF77EF8049B0646CDE90093B7
:105310005A46062341462846FCF7E4FACDE9009AAE
:10532000194A0623414628460137FCF793FAEF2F26
:10533000D4D1039B93F8EF70B4B194F8EF80474554
:10534000324614BF0121002128460CBF012400244D
:10535000FEF758F8002300930B4ACDF8048007238A
:1053600021462846FCF7BEFA00230093064A01971F
:10537000072321462846FCF76DFA07B0BDE8F08FF9
:10538000A24693E7A046C9E7FBAC0608F0B5054680
:1053900087B00846FEF746F90B46044638B10023AD
:1053A0001C491A46012007B0BDE8F04048E71A49F9
:1053B000194F02AA184648F01DF903AEB8B1032CE4
:1053C00004D12846FDF756FA07B0F0BDFAF700FF02
:1053D00002AA46F8040B39460020013448F00AF9C5
:1053E000ECE70E4832462146FCF7F2FAECE7032CD4
:1053F000E7D1DDE90346059B01931A463146E0B249
:1054000035F012FB019B0028EBD12846FDF7F4F99B
:10541000DAE700BF0CAC002080AD0608FBAC060844
:105420002DE9F04F0F4689B0164600211A46054671
:10543000FDF7E8FFDFF83CB10790B84634464FF07F
:105440000009002E7ED021460C22404648F0D5F8B7
:105450000028079A14BF0121002128460CBF4FF0F5
:10546000010A4FF0000AFDF7CDFF94F90B200492DA
:1054700094F90A200392B4F908200292B4F90620A4
:105480000192B4F90420079000924B465A465146C7
:105490002846FCF727FA98F90B20049298F90A207D
:1054A0000392B8F908200292B8F906200192B8F9DF
:1054B000042000924B465A465146284609F10109FC
:1054C000FCF7C8F9B9F1080F08F10C0804F10C0455
:1054D000B7D1DFF8A49000240C2303FB04FA9EB399
:1054E0004FF00008012303FA08FB56F80A2057F88A
:1054F0000A3053403BEA030314BF0121002112EAA2
:105500000B0F08D0CDF8008023464A462846079165
:10551000FCF7E8F9079957F80A301BEA030F06D0A1
:10552000CDF8008023464A462846FCF793F908F157
:105530000108B8F10E0FD5D10134082CCCD109B037
:10554000BDE8F08FB246A6E7B04657F80A2001231F
:1055500003FA08F3134207D0CDF8008023464A46E9
:1055600001212846FCF776F908F10108B8F10E0F81
:10557000EBD1E1E70FAD060827AD0608F0B506460A
:105580008BB00846FEF74EF80D46044620B30023C4
:105590003F491A4601200BB0BDE8F04040E72D2BF3
:1055A00003D0A3F13002092A4BD8052C05DD304683
:1055B0000BB0BDE8F040FDF75DB92846FAF708FEEC
:1055C0000AAB621C03EB440424F80C0C15F8013FF1
:1055D000303B092BFAD914462B78002BDFD1062C4F
:1055E000E5D1BDF81C20BDF91C30072ADFD8BDF974
:1055F0001E10A1F5FA7292B2B2F5FA6F1AD8BDF97F
:105600002040A4F5FA7292B2B2F5FA6F12D8BDF941
:105610002270B9420EDCBC420CDBA1420ADCBDF9AF
:1056200024C00CF1640292B2C82A03D8BDF92650F6
:10563000112D11DD174930460BB0BDE8F040FDF7E4
:10564000C4B8202B02D101352246C4E730460BB046
:10565000BDE8F040FDF7D0B80F4A0C2000FB032254
:105660006DB2A2F8D811A2F8DA41A2F8DC7182F882
:10567000DEC182F8DF5100910021CDE903C5CDE9FB
:105680000147064A0846FCF7E5F80BB0F0BD00BF3D
:10569000FCAC00203CAD060828AB00200FAD06088E
:1056A0002DE9F04F89468DB0164600211A4607466F
:1056B000FDF7A8FEDFF8DCA005460024C4EBC40318
:1056C00009EB030259F8030091889279089040F39E
:1056D0000748ADF824108DF82620B8F1000F54D0FB
:1056E000002E55D0F218F058918893790A90ADF8B1
:1056F0002C1007220AA908A88DF82E3047F07DFF4C
:1057000000282A4614BF0121002138460CBF4FF063
:10571000010B4FF0000BFDF775FE9DF82E30069340
:105720009DF92D3005939DF92C3004939DF82B3075
:1057300003939DF92A3002939DF8293001939DF837
:105740002830009305462346524659463846FCF712
:10575000C9F89DF8263006939DF9253005939DF9EB
:10576000243004939DF82330CDE902839DF8213045
:1057700001939DF8203000935246234659463846FF
:105780000134FCF767F8102C98D10DB0BDE8F08F0C
:10579000B346DEE752AD06082DE9F04F9D4FDFF826
:1057A000A882DFF8A8928DB006460D46284645F03F
:1057B0005FFC034630B99849024601200DB0BDE8B0
:1057C000F04F6DE7052239462846FAF7E9FB044613
:1057D000C8B9924D0146702205F50D7047F037FFAC
:1057E000C5F8D441C5F8E041C5F8EC41C5F8F84129
:1057F000C5F80442C5F81042C5F81C42C5F8284255
:105800000DB0BDE8F08F042241462846FAF7C8FBE8
:10581000044638BB2846F9F7EBFC82460028EFD057
:1058200045F026FCDFF828B202465BF8041B39B9C4
:105830007B492A4630460DB0BDE8F04FFCF7C5BFA6
:105840005046CDE90012FAF7ABFB019A40B9204669
:1058500028F0CCFF0099734D4846FCF7B9F8A5E74E
:105860000134E2E7704907222846FAF799FB074618
:1058700000287AD12021284647F000FF044670BB5B
:105880006A486B4DFCF746F8214628460134FCF780
:1058900041F80E2CF8D1FBF7D9FFDFF8B891654F2E
:1058A000DFF8B481002421464846FCF733F80C2683
:1058B000DFF8A8A166430025F2595F480123AB40F9
:1058C000134214BF414651460135FCF723F80E2D13
:1058D000F2D10134FBF7BAFF082CE4D190E7574925
:1058E000564D03AA47F086FE04AC002848D0022F8C
:1058F00011D1049A072A07D805990D2904D80378ED
:10590000722B13D06E2B22D04D4908230022304633
:10591000FDF788F874E7FAF75BFC03AA44F8040B78
:1059200029460020013747F065FEDEE73B4B0C209F
:1059300000FB0233012000FA01F1D3F8D40108433F
:10594000C3F8D40138493046FFF726FF58E7334BF8
:105950000C2000FB0233012202FA01F1D3F8D4211A
:1059600022EA0102C3F8D421ECE728463349334F39
:1059700003AA47F03FFE04AD0024A8B1082C03D1D0
:105980003046FCF777FF3BE7FAF722FC03AA45F81D
:10599000040B39460020013447F02CFEEDE729497D
:1059A0003046FCF712FF2BE7082CE9D1049B0F2BA4
:1059B000F5D8DDF814E0BEF1070FF0D8DDF818C017
:1059C000BCF10D0FEBD8079F07F16402C82AE6D897
:1059D000089DFF2DE3D809986428E0D80A99642926
:1059E000DDD88842DBDA0B9C032CD8D8C3EBC3028A
:1059F0000A4B134483F8391283F834E2094983F8D7
:105A000035C283F8367283F8375283F8380283F848
:105A10003A4298E753A906085CAD002028AB002065
:105A20007AA60608F1A906086FAD0608EEB30608C7
:105A300077AD0608FCAC00207CAD060880AD0608FA
:105A400082AD06083CAD0608B1AC0608B6AC060847
:105A500040FB05080B9D06083AAD0608DEB00608B7
:105A60002DE9F04F89B00C46079200211A460746EF
:105A7000FDF7C8FC0026079DDFF8A0B00690B246EF
:105A80004FF019094FF46178079B43B3294606226A
:105A9000204647F0B2FD0028069A14BF01210021DC
:105AA00038460CBF4FF0010A4FF0000AFDF7AAFC80
:105AB0006A79069019FB028205922A7919FB028203
:105AC0000492EA780392AA7802926A7801922A787C
:105AD000009233465A4651463846FBF703FF627937
:105AE00019FB02820592227919FB02820492E27864
:105AF0000392A27802926278019214F8062B009227
:105B000033465A46514638460136FBF7A3FE0A2E65
:105B100005F10605B8D109B0BDE8F08F88AD0608DB
:105B20002DE9F04F074689B00846FDF77BFD8B460F
:105B3000054638B100234C491A46012009B0BDE89A
:105B4000F04F8DE7494B084693F88CA593F88D9557
:105B500093F87686FAF73CFB092804467BDC062698
:105B600046430BF101008DF81F50F9F741FB3E4D04
:105B7000834648B1FAF72CFB0D289FBF9DF81F30D4
:105B8000A85501338DF81F305846F9F731FB83468D
:105B900060B1FAF71DFB824508D3062303FB0453CB
:105BA00058709DF81F3001338DF81F305846F9F7B3
:105BB0001FFB824660B1FAF70BFB484508D8062365
:105BC00003FB045398709DF81F3001338DF81F308C
:105BD0005046F9F70DFB814660B1FAF7F9FA8045B6
:105BE00008D3062303FB0453D8709DF81F300133FC
:105BF0008DF81F30311D0DF11F0229444846FAF778
:105C0000EBFA9DF81F30062B09D0AA190023AB51DF
:105C100038469380FCF72EFE09B0BDE8F08F634351
:105C2000EA184FF461765079192111FB0060059054
:105C3000107911FB00610491D17803919178029160
:105C400052780192EB5C00930021094A23460846F2
:105C5000FBF700FEE0E7074909232A46384609B06A
:105C6000BDE8F04FFCF7DEBEDC370020309A0020A4
:105C700088AD060857AC06082DE9F04F0F4689B0ED
:105C8000144600211A460646FDF7BCFB0546002CCB
:105C900000F0DB8022783B789A4218BF012102464F
:105CA00008BF002130460CBF4FF001084FF000083C
:105CB000FDF7A8FB23789B4A054641463046FBF793
:105CC00011FE3B78974A41463046FBF7C3FD002C56
:105CD00000F0BD8062787B789A4218BF01212A4685
:105CE00008BF002130460CBF4FF001084FF00008FC
:105CF000FDF788FB63788C4A054641463046FBF742
:105D0000F1FD7B78884A41463046FBF7A3FD07F159
:105D1000CA030493822304F1CA0B05934FF00209CE
:105D20004FF0000A3B78534500F39380002C00F0BD
:105D3000F38097F8EA3094F8EA209A4218BF0121DC
:105D40002A4608BF002130460CBF4FF001084FF033
:105D50000008FDF757FB94F8EA30744A05464146BF
:105D60003046FBF7BFFD97F8EA30704A41463046AF
:105D7000FBF770FD07F1EC09002C00F0CF8004F177
:105D8000EC034A4604F1FC014FF001089A4633F84F
:105D900002CB32F8020B844518BF4FF000088B424B
:105DA000F5D188F001012A46C9B23046FDF72AFB39
:105DB000082105465046FAF71FF85D4A034641465A
:105DC0003046FBF78FFD97F8EA104846FAF714F8CB
:105DD000574A034641463046FBF73CFD002C00F095
:105DE0009F804FF0FC094FF0010807EB090104EB1D
:105DF0000900FAF7B1F809F10409002818BF4FF0BB
:105E00000008B9F58E7FF0D188F001012A46C9B2A9
:105E10003046FDF7F7FA082104F1FC00F9F716FA0D
:105E2000444A034641463046FBF75CFD97F8EA10CA
:105E300007F1FC00F9F70AFA3E4A034641463046AC
:105E400009B0BDE8F04FFBF705BDA04639E7A04615
:105E500057E7059B3B440693002C5BD0059B0698B7
:105E6000234419460793FAF777F8049B1A789BF8AE
:105E700000309A4206BFB0FA80F84FEA58184FF047
:105E800000084B4609F11002F85AE15A02338842E1
:105E900018BF4FF000089342F6D188F001012A465E
:105EA000C9B23046FDF7AEFA627804EB0901054647
:105EB0009BF81800F9F772FF02909BF800300193ED
:105EC000079B00931C4A0AF1010341463046FBF749
:105ED00009FD049B7A78187E079307EB0901F9F70F
:105EE0005DFF079B049A02901B7801930132069B89
:105EF00004920AF1010A00930F4A53464146304684
:105F0000FBF7A8FC059B09330BF1010B09F1100904
:105F1000059307E7A046DCE7A04624E7A04652E742
:105F2000A04683E7A1AD0608B3AD0608E1AD0608BB
:105F3000F9AD060810AE0608C8AD06082DE9F04F09
:105F40008FB0044602AA0846AF4947F053FB064605
:105F500040B903460246AD494120FFF78DFE0FB020
:105F6000BDE8F08FAA49F9F7F7FF074620BBA6491D
:105F700002AA47F03FFBFAF72BF90828054606D995
:105F8000A44908233A462046FCF74CFDE7E7A24C1B
:105F900094F88C35834202DC84F88C55DFE70646A2
:105FA00004F28C573146384631F044FD94F88C3574
:105FB0000136B342F6DCEFE798493046F9F7CCFFFB
:105FC0000546E0B9904902AA47F014FBFAF700F938
:105FD0000828064603D9924908232A46D3E78E4C5F
:105FE00094F88D35834202DC84F88D65B7E7284646
:105FF000314601353FF0AEFD082DF8D1F4E789496F
:106000003046F9F7A9FF074600BB7F4902AA47F0CF
:10601000F1FA0028A3D0FAF7DBF80828054603D9DF
:10602000814908233A46AEE77B4C94F876368342A2
:1060300009DD014604F28C5031F046FD294604F298
:106040008C5031F04FFD84F8765688E7774930461A
:10605000F9F782FF054618BB6F4BDFF8AC9193F858
:10606000767606AE01461022304647F0F0FAB0468A
:10607000BD4202AA80F20E814946002047F0BAFADA
:1060800010B96B493A460EE1FAF7A2F8013528F843
:10609000020BEDE796E80F00664C84E80F005EE720
:1060A00065493046F9F758FF054600283BD15A4B61
:1060B0000DF1180893F87696464607464F45524923
:1060C00002AA4FF0000080F2F28047F093FA0146F6
:1060D00010B95A494A46E6E00322304647F008FB29
:1060E000B2464FF0000B304644F0C2FF584502D88C
:1060F00001370436E2E79AF80000F9F727FF0BF1C1
:10610000010B0AF8010BEEE74D494A46CBE0414648
:106110002046032231F076FC0135043408F10408EE
:10612000AF42F4D11BE747493046F9F715FF054662
:10613000002840F0AC80384F334997F88C8502AA8C
:1061400047F058FA00283FF40AAFFAF741F8461E24
:1061500001D4B04503DC3C494346012213E72A49F8
:1061600002AA002047F046FA014600283FF4F7AEA5
:106170004FF00008082203A8CDE903888DF81480A9
:1061800047F0B6FA0DF10C0903A844F071FF404541
:106190001CD81D4902AA002047F02CFA00283FF421
:1061A000DEAE90F800A097F88D95DFF8ACB04FF018
:1061B00000084D45144902AA4FF000007EDA47F06E
:1061C00019FA024658B921494A466CE099F800008C
:1061D000F9F7BCFE08F1010809F8010BD4E7002D1E
:1061E00040D11378303B092B3CD919490192F9F77A
:1061F000B3FE019A90B310465946F9F7ADFE019AE5
:10620000002838D013494EE080AD0608BC9F00201E
:1062100027AE06082DAE0608309A002038AE0608D4
:1062200041AE06084FAE06085BAE06086DAE060826
:106230005CAF0608A8A0002097AE06087CAF060851
:10624000A3AE0608C1AE0608C6AE06089CAF060897
:106250006B9C0608D9AE0608D2AE06084FF00108BE
:106260004FF0FF3510460192F9F7B2FF0028019A6E
:1062700003DA214917E0A846F2E70EAB03EB45032A
:10628000013523F8200C94E71C494A460BE01C49D1
:10629000324608E01B49002047F0ACF900283FF4E3
:1062A000F9AE19493A462046FCF78FFA57E647F00F
:1062B000A1F900287FF428AF144C31E747F09AF990
:1062C0000028E1D1124C06EBC6008230082203A957
:1062D000204431F097FB5046F9F738FE37446A0006
:1062E00087F8560604EB061006A9023047F04CF971
:1062F00087F86E8633E600BF0EAF060823AF0608A8
:1063000046AF060880AD060879AE0608B8A00020A2
:10631000BC9F00202DE9F04F89B00F469146002127
:10632000139A98460646FDF76DF887EA09096FEA61
:106330000903DFF8849006930446002528460BF0F5
:1063400039FE129B184230D0069BDFF870B0034034
:1063500014BF4FF0010A4FF0000A049310EA07033C
:1063600014BF4A465A462846059307920BF034FE5E
:10637000079A03900090434651463046FBF7B2FA25
:10638000049BB3FA83F1224649093046FDF73AF8F7
:10639000059A039B009304464346002A14BF5A46BD
:1063A0004A4651463046FBF755FA0135182DC5D1FE
:1063B00009B0BDE8F08F00BFABAC0608C1AF06085E
:1063C00037B504460846019144F052FE019905464E
:1063D00002462046F9F7E4FD70B9625D1046F9F710
:1063E000A5FD00B932B901352C44204601340378AB
:1063F000202BFAD003B030BD0020FBE7F0B5032915
:1064000085B005460C46164614D80B4F3970FBF77D
:106410001DFA0A492846FDF76BFD0949224601A8E5
:10642000F9F760FC01AB324608212846FDF784F8F5
:10643000FF233B7005B0F0BD94050020F1A90608CC
:10644000A7AB0608F0B5032985B005460C461646ED
:1064500014D80B4F7970FBF7F9F90A492846FDF774
:1064600077FD094922466846F9F73CFC6B463246FF
:1064700010212846FDF760F8FF237B7005B0F0BDC2
:1064800094050020F1A90608A3AB060810B586B054
:10649000104B0493104B0393104B0293104B01933A
:1064A000104B1149114A00930446114B1148FBF758
:1064B00031FAFBF7CBF910491048FBF789FA3CB1E8
:1064C0000F4A1049104806B0BDE81040FBF780BAEB
:1064D00006B010BD08B006080DB0060817B00608D3
:1064E00020B00608A59F0608D2AF0608C8AF060868
:1064F00073350020DDAF06082CB0060834B006085E
:1065000081A50608D5A5060845B006080120BDE707
:106510002DE9F04F0A4687B000210646FCF772FFCE
:106520003B4C05903B4A2378608802EB8303D3F809
:106530009CA1F8F763F983680493374BC1681A7913
:10654000002A4BD0DDF81080049100272179627970
:10655000049B07FB012213F80290B8F1000F3FD013
:1065600018F80250059A4D4514BF0121002130460C
:106570000CBF4FF0010B4FF0000BFCF743FF01374E
:1065800005907DB305F00F022D0940350292CDE94B
:106590000075224A534659463046FBF7A3F9B9F134
:1065A000000F2AD009F00F024FEA1919029209F1DF
:1065B0004002CDE900725346184A59463046FBF76F
:1065C00049F9A279012A38BF0122BA42BEDC144B34
:1065D0000834A342A6D107B0BDE8F08F9046B4E7D7
:1065E0004546BFE7B8F1000FD9D00E4A0097534691
:1065F00059463046FBF776F9D1E77306E1D4094AEC
:106600000097534659463046FBF724F9D9E700BFB7
:1066100070F6050864F30508309A002072B0060889
:1066200088F7050888B006082DE9F04F2DED028B9C
:106630000A468BB000218246FCF7E4FE6E4D81468F
:1066400005F1800B00266D4B1C79AB7AB34200F349
:1066500095801035AB45F5D140F21620F8F7CEF80D
:10666000D0E902530CB12C461D460DF1100B15223A
:106670000021584646F0EBFF00272E78002E44D02C
:1066800069780391304607F0C7FD95F9023002930F
:106690005A1C534208EE100A5341002C00F0A98006
:1066A0000399002214F802C0B44504EB020040F044
:1066B0009C8090F90280029A424540F09480427892
:1066C0008A4208BF012301220BF8072003F00103CF
:1066D0004A4683F0010150460393FCF793FE039B67
:1066E00081464CB1464A18EE101ACDE900A2304658
:1066F0004246F8F72BFE039B424A18EE101ACDE9EA
:1067000000A23046029AF8F721FE0137152F05F155
:106710000305B2D16CB33A4FDFF8E88004F13F06CD
:106720001BF8013B02930BBB2078F8B194F90220CF
:1067300001321BD0617807F06FFD4A460546012102
:106740005046FCF75FFE94F90220029B29468146E1
:106750002078CDE900A7F8F7F9FD2078029BCDE974
:1067600000A84FF0FF322946F8F7F0FD0334B44299
:10677000D6D10BB0BDEC028BBDE8F08FE888F8F7FE
:106780003DF8D0E902230CB114461A46297A6B7AF7
:1067900006FB013312F9038014B3E756B8450CBF6A
:1067A000012300234A4614BF0121002150460293D1
:1067B000FCF728FE029B814644B1114A3146CDE9DF
:1067C00000A228463A46F8F775FD029B0D4A31466D
:1067D000CDE900A228464246F8F76CFD013632E7C3
:1067E0004FF0FF37DAE700236DE703323F2A7FF4EB
:1067F00059AF4FF0FF386BE7AC050020309A00200E
:10680000E5180108551801082DE9F04F80468BB0B6
:1068100008460D4644F02CFC024678B3A5492846AC
:10682000F9F7BEFB044648BBFBF710F8A248A34D9E
:10683000A34FA44EDFF8D882FBF720F814203FF0D6
:106840009DF9E11004F0070201313846FBF762F8C8
:106850002B7F6A7F06EB8303D3F89C1152B19A48D1
:10686000FBF7B6F80134102C05F12405E9D10BB083
:10687000BDE8F08F4046FBF7ABF8F3E728469349B5
:1068800005AA46F0B7FE054620B901464120FFF7AC
:10689000CBFEECE78E49F9F75FFB20B98D49404606
:1068A000FBF793FFE3E78C4E082700243168284666
:1068B000F9F752FB002808BF3446013F06F11006E5
:1068C000F4D154B985492846F9F746FB28B18449E3
:1068D0002A464046FBF779FFC9E700207B498DF83F
:1068E000130005AA46F086FE0646002C3AD080B179
:1068F000F9F76EFC451E09D4A37A9D4206DAE268D8
:106900004AB1012303FA00F0104204D1754932461E
:10691000DFE7754EFAE7E088F7F770FF7349D0E9D3
:1069200002320979002908BF1A46217A637A05FBE9
:106930000133002712F903A0039702EB030B63490D
:1069400005AA002046F056FE8146A0BB68490123F7
:1069500044B39BF900202046CDE900312946F8F7E1
:10696000A9FC84E768B10DF11301F9F70AFC28B11D
:106970009DF81350284603F02DFB20B95D4932469F
:10698000A7E7594EFAE72846F4F7F6F88246284674
:1069900007F02EFC0390284607F068FCA346074644
:1069A0002546CCE7CDE900319DF813005246394623
:1069B000F8F7CCFC5BE74649F9F7CEFA064658BB38
:1069C000ACB14D4FEDB2207972B22946F4F7A8F878
:1069D00000283FF44CAF0288037800933146C2F39D
:1069E00003233846120BFAF7F3FF0136EBE7424C6C
:1069F0007979386872B2F4F7DBF800283FF437AFE2
:106A00000288037800933146C2F303232046120B19
:106A1000FAF7DEFF0136EBE738494846F9F79CFA0A
:106A200010B34846F9F7D4FB064642B26CB1207960
:106A3000E9B2F4F775F8C8B9CDF80090226830498A
:106A40006B1C4046FBF7C1FE11E779793868F4F713
:106A5000AFF858B99DF813302A49CDF800901A09BB
:106A6000403203F00F03ECE74FF0FF3606AF394634
:106A70003046F9F7F5F908A95046F9F7F1F9564506
:106A800048D076B24CB18BF80060009721681E4860
:106A900008AB6A1CFAF79CFFE9E69DF81320039BFC
:106AA0001A489E701109009708AB02F00F0240319E
:106AB000F0E700BF9CB00608A1B00608D002002095
:106AC000B7B0060864F305082AB2060880AD0608C8
:106AD00074A10608C8B00608AC050020DCB00608A2
:106AE000E0B00608EFB00608F1A90608309A0020C9
:106AF00055180108FFB0060811B10608A8A6060837
:106B000032B1060855B106087DB10608A0B10608E5
:106B1000EBA0060834B12168074808AB6A1CFAF7F5
:106B200057FFA4E69DF813200448110908AB02F0B2
:106B30000F024031F3E700BFC8B10608E3B1060811
:106B40002DE9F04F8BB0074640F216200391F7F77E
:106B500055FE039A044600213846FCF753FC404A90
:106B6000D4E90253147906460CB12C461D46152271
:106B7000002104A846F06BFD05F13F03039395F84F
:106B80000090B9F1000F31D095F801A0002C65D02C
:106B9000224600231178494558D128336B4492F896
:106BA0000180012203F8182CD045324614BF012180
:106BB000002138460CBF4FF0010B4FF0000BFCF7E3
:106BC00021FC064654B1B8F1000F07D0254B0093C5
:106BD0005A463B4641464846F8F7FCFB224B009399
:106BE0005A463B4651464846F8F7F4FB039B0335AB
:106BF0009D42C4D13CB3DFF86C90DFF86CA0651CFB
:106C00000DF11008403418F8013BCBB915F8013CE0
:106C1000B3B116B13046FAF737FE297815F8010CF2
:106C2000CDF800903B460022F8F7D4FB002215F87F
:106C3000010CCDF800A03B461146F8F7CBFB00262F
:106C40000335A542DFD10BB0BDE8F08F0133152B22
:106C500002F103029ED14FF00008A5E7A046A3E78A
:106C6000309A0020E5180108551801082DE9F04F69
:106C700080468DB008460D4644F0FAF9024628B920
:106C8000014601200DB0BDE8F04F59E70390B1492E
:106C90002846F9F785F9039A30B9AF4940460DB057
:106CA000BDE8F04FFBF791BDAC492846F9F778F9FC
:106CB000044600285BD1FAF7C9FDA948A94FDFF8BF
:106CC000E4B2DFF8E482FAF7D9FD17203EF056FF70
:106CD00017F9015B002D3CD029465846FAF71AFEF9
:106CE000DFF89C92DFF88CA200231A46910089B24B
:106CF00028460593049207F0F1FA039007F07CFB15
:106D0000049A0178059B561CC9B11BB90490FAF787
:106D10009DFD0498039B41789A79037802F0020262
:106D200008EB8303C1B10091D3F89C318E48002A4F
:106D300014BF4A4652463146FAF74AFE0123042E52
:106D40003246D3D113B98948FAF798FD01340E2C95
:106D5000BED10DB0BDE8F08FD3F89C318448002A35
:106D600014BF4A4652463146FAF732FEE6E700249F
:106D700080498DF81B4007AA284646F03BFC18B90D
:106D80004046FBF739FDE4E70DF11B01F9F7F9F98E
:106D900005460028F4D09DF81B60304603F01AF930
:106DA00020B975494046FBF710FDD2E7DFF8FC91AA
:106DB00023464FF0FF3403EB430212F809209642BA
:106DC0000BD0611C02D1002A08BF1C460133152BD1
:106DD000F1D1631C15D16949E4E71C46654907AA4E
:106DE000002046F007FC0646002800F09E80594926
:106DF000F9F7B2F828BB624E624FDFF8B48104465F
:106E000015E00025EAE7E97928680391F4F78CF8A2
:106E10000246A8796B79039910F0020F14BF30462F
:106E200038469B08009001334046FAF7D1FD013403
:106E30009DF81B00214607F0EFF905460028E2D136
:106E400087E7514902223046F9F7AAF80746002899
:106E500049D1B01CF9F7BCF99DF81BB00346BA46FE
:106E6000013739465846039307F0D6F9039B38B9E2
:106E70004FEA1B12454900960BF00F0340323FE0EA
:106E8000C2799A42EBD1002D40D14FF0FF36BAF1D2
:106E9000FF3F9DF81B5008BF002504EB440409EB9D
:106EA00004030AF101025A7009F80450FF220AACE7
:106EB0009A709DF81B0022465146F8F7E1FF08AA98
:106EC00031469DF81B00F8F7DBFF9DF81B20B2450B
:106ED0004FEA121120D12E4808AB02F00F024031C8
:106EE000FAF776FD35E72B493046F9F735F850B318
:106EF0009DF81B30284900961A09403203F00F0311
:106F00004046FBF762FC24E74FF0FF3A04EB4403F2
:106F10004B445E78013EBAE72048009408AB02F08B
:106F20000F024031FAF754FD13E704EB44041C4B05
:106F30000093A144024699F801109DF81B0001231B
:106F4000F8F748FA05E7002DDED14FF0FF36B246DC
:106F5000A3E700BF74A10608C8B006089CB00608E5
:106F6000FFB10608D85506081FB2060840B2060849
:106F700031B2060880AD060846B206085DB20608C2
:106F80005D9D0608F1A9060886B20608F3B2060858
:106F9000AFB20608A8A6060889B20608CDB2060850
:106FA0005518010818B2060864F3050834270020B4
:106FB00071B206082DE9F04F2DED028B85B0064623
:106FC00003AA0846924946F015FB074640B9014618
:106FD0004120FFF79DFA05B0BDEC028BBDE8F08FB4
:106FE0008C49DFF86482F8F7B7FF044600283CD1EB
:106FF00089488A4D8A4FDFF85492FAF73FFC1420F3
:107000003EF0BCFD2968AB79AA8801F13F4108EB4D
:10701000830301F57E01B2FA82F2890A4131D3F885
:107020009C31C2F11F023846FAF774FCE97911B1BC
:107030004846FAF76FFC0134FAF708FC602C05F1BA
:107040000805DFD1724903AA002046F0D3FA75493A
:10705000F8F782FF0028BED130466E49FFF706FEE2
:107060006C493046FFF7D0FBB5E7002508F54379BA
:1070700019F8353008EB8303D3F89C1101910846C9
:1070800043F0F6FF019902463846F8F789FF40B110
:107090000135232DECD164493A463046FBF795FB88
:1070A00099E75B4903AA46F0A5FA08EBC50807462D
:1070B000F9F78EF898F8123304464FEAC50A2BBB4D
:1070C000002825DC3B78002B00F09E80D144B9F8E5
:1070D0000200F7F793FBE3B2019399F8058099F862
:1070E0000430019A846802FB038804EB08013846E7
:1070F000F9F747F8002800F0878014F808A0BAF1E3
:10710000000F1CD14948FAF7B9FB64E7002805DDF8
:10711000012B1A4638BF0122A24208DA012B44494A
:1071200038BF012301223046FBF77CFC53E7384986
:1071300003AA002046F05EFA013C0746C2E750462B
:1071400002F048FF814600285ED04FEA1A13403310
:1071500008EE103A0AF00F03DFF8F48008EE903AD8
:1071600000270026B8F80200F7F748FB98F804203B
:1071700098F8053006FB02338268D15C514523D173
:10718000BD4204D101998E421ED00021D15418EE87
:10719000902A18EE101A27485FFA86FBFCB2FAF71D
:1071A000B9FB59462046FAF7F5FBBD4209D1224802
:1071B000FAF7B0FB20465946FAF7ECFB1F48FAF7FE
:1071C000A9FB1F48FAF75AFB98F80630012B06F185
:1071D000010638BF01239E42C4DB0137232F08F18B
:1071E0000808BED1D9F80010B9F80420154801F1FB
:1071F0003F4101F57E01B2FA82F2890AC2F11F0213
:107200004131FAF7E5FBE6E63046FBF7F5FAE2E650
:1072100080AD06089CB006081FB30608FC230020BA
:107220005DB3060868B306086CB3060888B30608A1
:1072300057AC06089AB30608D89C0608BEB30608E1
:107240003ECA0608C8B3060864F305080A9D060886
:1072500070F60508224BB0F5FA6F1A680346A8BF0E
:107260004FF4FA63B3F57A7FB8BF4FF47A73D20460
:1072700016D540F2DC52904215D007EE903A40F21B
:10728000DB529042F8EE677A1FD8DFED166A9FED69
:10729000167A9FED160A77EEE67AA7EE870A704710
:1072A000B0F57A7F02D89FED120A704707EE903A48
:1072B000DFED106A9FED107A9FED100AF8EE677A05
:1072C00077EEE67AA7EE870A7047DFED0D6A9FED4D
:1072D0000D7A9FED0D0A77EEE67AA7EE870A7047E2
:1072E000A835002000007A44D62000C000E0824487
:1072F0000000000000407A44661000400000404258
:1073000000A0BB44D62000400000834410B5844652
:107310004FEA810E102312F4004F14BF0E240724ED
:107320005200013BCCF8004092B2F444F3D100EBA0
:1073300081128C01035142F82130122010BD00BF90
:1073400010B584464FEA810E0424130B03EB43036C
:1073500018331201013CCCF8003092B2F444F4D15D
:1073600000EB01130A01845043F82140062010BDB0
:10737000704700BF704700BF034B00EB400003EBBA
:10738000C000407C704700BF480500100023472222
:10739000027043708370C370704700BF704700BFB6
:1073A00000207047704700BF0020704701207047E1
:1073B000704700BF704700BF704700BF704700BFF5
:1073C0009FED010A704700BF0000000000207047D9
:1073D00003681B69184730B5084B002293F9004039
:1073E0005D7801190132CD729D780555062ADC7849
:1073F0008C7503F10403F1D130BD00BF2C230608C6
:10740000002383700370C37043707047C36B33B144
:107410005B68426D9BB29A4205D3D01A7047D0E99F
:1074200007239A42F9D2C0681044C01A704700BFBF
:10743000D0E909120369914238BFC9188A1A016C50
:1074400039B14968013B12FA81F2934204D9981A82
:107450007047013B981A704700207047036C13B1C6
:1074600090F864007047D0E90903181AB0FA80F068
:1074700040097047C26B10B4034662B1426DC168E7
:107480005C69881A013A205C5DF8044B08BF0A4623
:10749000C0B25A657047006A5C69411C205CDC68B8
:1074A000A14238BF0A46C0B25DF8044B1A62704769
:1074B000836E70B504460D460BB19847B8B1636A48
:1074C000A269D554636A2169226C01338B4228BFBB
:1074D0000023636232B3EFF31183502282F31288E8
:1074E000226C1168C90703D5DBB283F3118870BD24
:1074F000516889B271B9D4E90950854218D0A6699A
:107500000644D66018D9281A80B25060A5620021BE
:1075100084F86410116841F00101DBB2116083F35B
:10752000118870BD226ED36843F08003D36070BDB4
:10753000012284F86420D7E72569281A80B25060B8
:10754000A162E4E7836E03B118477047F8B590F87D
:107550007C30012B1CD0002A164619DD0269436AD3
:1075600005460F46D41AB442A869A8BF3446394626
:107570001844224646F008F86B6A2A692344361BF1
:10758000B3FBF2F0002E02FB10336B622744E9DC00
:10759000F8BD00BF90F87C30012B0DD0036C43B3D5
:1075A000EFF31183502282F31288026C1168C9072D
:1075B00003D5DBB283F311887047516889B270B488
:1075C00071B9D0E90954A54219D086692644D6601C
:1075D0001CD92C1BA4B254608562002180F8641071
:1075E000116841F00101DBB2116083F3118870BCB6
:1075F0007047026ED36843F08003D3607047012266
:1076000080F86420DBB283F31188F0E705692C1B56
:10761000A4B254608162E0E770B5094C236873B18D
:107620000546002606E099681A681E732160904797
:10763000236823B15A68AA1A002A1846F3DA70BDE3
:10764000A0B7002070B5214C2378012B00D070BD6D
:107650001F4B1B68002BFAD01E4D2B6828465B6819
:1076600098470028F3D01C4B1C4E1A683388928828
:107670009A420ED21A4B1B4A1B7852680021217085
:1076800003F00203002AE2D0E3B9136892881A8358
:1076900070BD1549096800224968EA622A6803FB3F
:1076A00001F12846D36898470E4A3388526801335F
:1076B0003380002ACBD01368928859690A42E6D0F9
:1076C0005A8370BD13689288FAE700BFD82F002054
:1076D0002C21002030210020D02F0020D62F002088
:1076E0007C21002080210020C82F0020914B1B68A6
:1076F000D90600D47047F0B58F4C2DED028B63692D
:1077000087B00BB1201D9847A369002B70D08B4820
:1077100094ED168A9847C21C054675D0002877DA82
:10772000431C00F0F9806FF001022262844E33683E
:10773000EB1A03FB03F34FF609218B42DCBF8149AF
:10774000A1FB031394F8751004EB4100D4BF43F37D
:10775000CF034FF4C853A0F878304B1CDBB2052B95
:1077600084F8753000F0888094F882303560002B02
:1077700000F08E80B4F87A00B4F87830B4F87C1059
:1077800094F82C600344B4F87E000B44B4F88010E5
:1077900003440B441BB2B3F5FA4F1946A8BF4FF48C
:1077A000FA4121EAE171A1863EB9002A05DDB3F56F
:1077B000167F78DB012684F82C60634B18781B2831
:1077C00044D01C2837D1676A604D236B2A80002F74
:1077D0006E80AB802DDD002A2BDDB1F5167F28DA17
:1077E000002E00F0A1809342D4BF0023012321E0AA
:1077F00055494FF0FF33087823621A461B2863620D
:1078000002D1524D6A80AB8007B0BDEC028BF0BD57
:10781000E36D4F4904EB830201330968A162052B34
:107820001066E3654DD094F87430002B4ED10246BB
:107830007BE70023EB80D4ED077AB4EEE78AF1EE24
:1078400010FA0CD54FF0FF336362DDE7D4ED077A11
:107850003E4DB4EEE78AF1EE10FAE98014D4002A26
:1078600064DB07EE902AF8EEE77A67EE887AFDEEA1
:10787000E77A17EE903AC1E7002384F875300123C8
:1078800084F88230356075E74FF0FF336362B9E703
:1078900094F82C604FF6FF73A3864FF0FF31002E53
:1078A0008BD1002A89DD236B93423BDA294802EB16
:1078B0008203C3EB0313A0FB03035B0923630026CE
:1078C0007BE700220123E26584F87430224F0FCF5A
:1078D00001AE0FC6029A3B683360904202DC134649
:1078E00002461846DDE90413994202DC1E460B46A7
:1078F00031468142A8BF01469A42B8BF1A46039B4F
:107900008B4202DB0846194603468A42A8BF0A4654
:107910009A42B8BF1A4608E70D4B20621B68A36263
:10792000024603E7002648E7012383E74FF0FF33D1
:1079300064E700BF3CA20020A0B70020A4B700204D
:107940002C060020CDCCCCCCDC220020E022002074
:10795000742100201F85EB5100B800202DE9F84F5D
:107960001F4DDFF88490DFF884A006460C463A27C6
:107970004FF000082046FBF755FED5F800B048B997
:1079800021465846F8F730FB20B968682146F8F7D9
:107990002BFB80B15846F9F739FF696811B15046A1
:1079A000F9F7B8FFA96811B14846F9F7B3FFF9F73D
:1079B0004DFF4FF00108013F05F11005DAD12046D7
:1079C000FBF730FE48B9B8F1000F06D12246304629
:1079D0000449BDE8F84FFAF7F8BEBDE8F88F00BFDC
:1079E00044230608F0B30608EAB30608E4B3060821
:1079F00008B5254B1B68DB040AD5B5EE400AF1EE4D
:107A000010FA12D19FED210A45F046F880B208BD68
:107A1000DFED1F7AB4EEE70AF1EE10FA1CDA9FED03
:107A20001D0A45F039F880B208BDDFED197AB4EED1
:107A3000E70AF1EE10FAE5D49FED177AB4EEC70A23
:107A4000F1EE10FA14D870EE677A9FED147A9FED7C
:107A5000140AA7EE870AE4E770EE677A9FED117AC1
:107A60009FED110AA7EE870A45F016F880B208BD0F
:107A7000DFED0E7A9FED0E7A70EE677A9FED0D0ABC
:107A8000A7EE870ACDE700BFA83500200080BB44E1
:107A90000000404200007A4400E0824466BEFFBE1F
:107AA0000060BB4438DFFF3E00407A44000083445E
:107AB00066BEFF3E00A0BB44F8B5C64B1D6815F07E
:107AC00004072DED048B40F00081DFEDC38AC34C29
:107AD00015F0200505D094F8505115F0020540F03E
:107AE000908094F888319FEDBE8A13F0010340F036
:107AF000AC8094F88921002A7ED1D4ED637A9FED81
:107B0000B97ADFEDB96A67EE877A94ED657AE8EEC7
:107B1000A67A38EEC77AC4ED637A84ED647A65B1EB
:107B200094F89C21D4F85431C4F8983101218A4248
:107B300084F88A1118BFC4F89031AC4B1E780E2E11
:107B400000F00781DFEDA47A002794ED6B7A94EDC5
:107B50006C6A77EEC76AD4ED6A7AA6EE267A77EE7B
:107B6000676A84ED6B7AE6EE267AC4ED6A7AC4ED34
:107B7000697A0FB1C4ED647AD4ED6D6A94ED6F7AD1
:107B80009FED9B5A94ED706AC4ED6D7A77EEE66ACC
:107B9000F0EE475AD6EE855AF0EE477AE6EE257AB1
:107BA00094ED6E0AC4ED6F7A37EEC07AA6EE070A3E
:107BB00084ED6E0A44F070FF02B282EAE273A3EB36
:107BC000E2739BB2092B7ED9002AACBF0A380A3077
:107BD00005B20E2EA4F8C45160D0242E09D1DFEDD9
:107BE000857A94ED640A20EE270A44F055FF824B13
:107BF0005880BDEC048BF8BD84F88A3184F8893153
:107C00007BE7D4ED587AB4F86431F8EEE77AC4ED46
:107C1000557A002B00F08A8007EE903ADFED746A07
:107C20009FED767AF8EEE77A86EEA78AB4EEC78AF9
:107C3000F1EE10FA88BFB0EE478A94F8883113F05D
:107C400001034FF001053FF454AF94F88931002B44
:107C500056D094ED659A78EEC99A002D3AD094F8F2
:107C60008A31002B54D0D4ED557A94ED660A5F4BDF
:107C70001E7877EEC07A0E2EC4ED697A5FD094F844
:107C80009C31002B75D0022B02D00FB1012B31D0CB
:107C9000D4ED697AF0EE698A012756E7DFED547A70
:107CA000554C9FED540A28EE278A28EE800ABDEE37
:107CB000C88A18EE103A238044F0EEFEBDEC048B27
:107CC0006080E580F8BD002583E7444C0127D4EDB2
:107CD000518AFDE6454B1E780E2E2AD094F88A5123
:107CE0009FED3D8A002DCAD1002FD1D094F89C3150
:107CF000002BCBD1F0EE697A0127F0EE698A24E7F8
:107D000094ED639A012384ED659A84F88931A2E7A2
:107D1000002F56D0D4ED557A37EEE80A012330EE25
:107D2000090A84F88A3184ED660AA0E79FED2C8A5F
:107D300083E7D4ED697A94F88A519FED278A9FED05
:107D40002D0A27EE800A44F0A7FE2B4B0E269880C2
:107D5000C8E7DFED2B7A94ED557A274B27EE277A8B
:107D60000027BDEEC77ADFED1C7A17EE102A9A8045
:107D7000EBE6002F8CD094ED696A94F89D31DFED2D
:107D8000216A07EE903A76EE688AB8EEE77A78EEE6
:107D9000897AF0EE698AF0EEE77A67EE877AF4EE98
:107DA000E67AF1EE10FAC4BF68EE266A86EEA78A7C
:107DB000F7EE007A77EEC87A67EEA97AE6EE087AEF
:107DC000C3E60A4B1E780E2E7FF462AFD4ED697ABB
:107DD0003D46B4E73CA2002000000000A0B7002010
:107DE0009A99993ECDCC4C3FCDCC4C3EDC22002024
:107DF0000000C842CDCCCC3DE02200206666663F44
:107E00000AD7233C00401C46F2F72ABA10B50446B4
:107E100044F042FE81B22046BDE81040F2F720BA9D
:107E200070B50468236A1B69054643B1236AD0F81C
:107E300094001B69984701282AD002280DD0236A94
:107E4000DA699AB9586958B399692162BDE87040F6
:107E5000C3E90522F2F7BEBB2362236ADA69143351
:107E6000002AF9D1236ADA69002AEBD0216A94F852
:107E700024200E7B1433F6B22362D2B996B9284679
:107E8000F2F72CFB28460121BDE87040F2F7ECBA6E
:107E9000236A143B014623622846F2F7E5FACEE74F
:107EA000206270BDAB68002BE9D01A689B885383B1
:107EB000E5E700212846F2F7D7FA002384F82430BA
:107EC000002EDCD0EEE700BF8069002834D00368C4
:107ED0001A6A127B1ABBD3E904125B6849686AB15B
:107EE00010B4546800220A6022609A885DF8044B3E
:107EF00022F003021204120C9A8091E71A891206EA
:107F0000FCD41A89D20708D400220A609A8822F089
:107F100002021204120C9A8082E79A89F1E78268C1
:107F2000002AD8D0116892880A83D3E904125B68CA
:107F30004968002AD4D1E1E7704700BF806900B9E1
:107F40007047016830B4D1E904424B68646872B18B
:107F50005568002222602A609A8822F003021204E7
:107F6000120C9A800B6A1B7B9BB930BC58E71A89AC
:107F70001506FCD41A89D20713D4002222609A88ED
:107F800022F002021204120C9A800B6A1B7B002B57
:107F9000EBD08368002BE8D01A689B88138330BC31
:107FA0003EE79A89E6E700BF30B50446006E838954
:107FB000A16023F400531B041B0C838195B06379EB
:107FC000009113F0040F21794FEA03324FEA0323A3
:107FD00003F48063ADF8083001F0010302F40052AD
:107FE00014BF4FF480550025002B4FF00003ADF86F
:107FF0000620ADF80C3007BF002208230C23042212
:10800000ADF804508D07694654BFADF80A20ADF8AD
:108010000A303CF003FC6279236ED00700F18A80BD
:1080200012F0080F9A8A7FD092B242F008029A8228
:108030009A8992B242F400529A812279D10732D5BC
:10804000E06B002800F088800023E26D0793CDE903
:108050000B33CDE90F33CDE911334FF4807509931C
:108060006369E1680D9505920693626C04924FF482
:1080700080634FF480350A9308910E953CF084F9A3
:1080800004A9E06B3CF016FAE16B236E0A6842F03B
:1080900001020A609A8A92B242F040029A824968CA
:1080A000227989B26165920737D5206C00285FD0AC
:1080B0002369A26D0893A36CCDE90432002240230A
:1080C0000025CDE906234FF480314FF480630A93F5
:1080D0000E91CDE90B55CDE90F55CDE91155099517
:1080E0000D953CF051F9206C04A93CF0E3F9226CA9
:1080F000236E506940F080005061106840F0160017
:10810000106055609A8A92B242F0800203F10C012D
:108110009A820A6842F040020A609A8992B242F456
:1081200000529A8115B030BD22F008021204120CE0
:108130009A827DE71D498B4223D0A1F54C418B42A9
:108140001DD001F580618B421DD102200121F2F783
:1081500019F86279236E63E74FF6DF711980D968E9
:1081600041F02001D960D96841F01001D9609AE747
:10817000DA6842F0800203F10C01DA60C9E70120FD
:10818000E4E70020E2E701F580618B420AD001F5C7
:1081900080618B4208D001F544418B427FF440AFAF
:1081A0000520D3E70320D1E70420CFE700100140EA
:1081B00030B50446006E21718389A26823F4005310
:1081C0001B041B0C8381637995B013F0040F00929C
:1081D00014BF4FF480520022ADF804201A031B0292
:1081E00003F48063ADF8083001F0010302F400529B
:1081F000002B4FF00003ADF80620ADF80C3007BFA0
:10820000002208230C2304228D07694654BFADF8D1
:108210000A20ADF80A303CF001FB6279236ED007EA
:1082200000F18A8012F0080F9A8A7FD092B242F051
:1082300008029A829A8992B242F400529A81227973
:10824000D10732D5E06B002800F088800023E26D72
:108250000793CDE90B33CDE90F33CDE911334FF45B
:10826000807509936369E1680D9505920693626CC8
:1082700004924FF480634FF480350A9308910E9571
:108280003CF082F804A9E06B3CF014F9E16B236E3A
:108290000A6842F001020A609A8A92B242F04002F1
:1082A0009A824968227989B26165920737D5206C34
:1082B00000285FD02369A26D0893A36CCDE9043236
:1082C000002240230025CDE906234FF480314FF4EE
:1082D00080630A930E91CDE90B55CDE90F55CDE999
:1082E000115509950D953CF04FF8206C04A93CF010
:1082F000E1F8226C236E506940F0800050611068F4
:1083000040F01600106055609A8A92B242F08002E6
:1083100003F10C019A820A6842F040020A609A89CD
:1083200092B242F400529A8115B030BD22F0080298
:108330001204120C9A827DE71D498B4223D0A1F5CD
:108340004C418B421DD001F580618B421DD1022032
:108350000121F1F717FF6279236E63E74FF6DF71B2
:108360001980D96841F02001D960D96841F0100125
:10837000D9609AE7DA6842F0800203F10C01DA6012
:10838000C9E70120E4E70020E2E701F580618B42C4
:108390000AD001F580618B4208D001F544418B423F
:1083A0007FF440AF0520D3E70320D1E70420CFE7D7
:1083B000001001402DE9F84FB44C94F88831DB07E8
:1083C0002DED028B804679D5B14B94F8C6511F88AC
:1083D000B04E012D5FD0022D38D0002D44D094ED49
:1083E000768AF37B33B1B38923B1AB4B1B78002B77
:1083F00040F0E88094F8C721AA4238BF2A46317A73
:10840000632907D8022D00F0FD8094F8D031002BAD
:1084100040F00E81A14BDFEDA26A1A70D4E97A30E8
:10842000C4F8EC311B1A07FB03F307EE903AF8EEA1
:10843000E77AB0EE487AA7EEA67AB17B84ED767A39
:10844000002970D1BDEC028BBDE8F88FB4F8CA31B9
:10845000BB42C4D2934B94ED768A1B68C4F8DC31DE
:10846000012584F8C651BCE7B4F8CC31BB421ED319
:108470008C4BD4F8DC111A68F37D03EB830303EB18
:108480008303521AB2EB830FA9DB012594ED768AA0
:1084900084F8C651A5E7B4F8CE31BB4280F09E8087
:1084A000B4F8C831BB423CBF002584F8C6517D4BAF
:1084B00094ED768A1B68C4F8DC3192E794F8C651D3
:1084C000DFF8CC91EB1E012B39D9B9F80800C0F3C5
:1084D0000B0043F0F9FA092840F3C1806D4EB9F85A
:1084E0000070F3889F4203D33288BA42BFF471AF61
:1084F000B7EB430F3FF76DAF0323DFED6B7A664AAF
:1085000084F8C63184F8C7310023B0EE678AC4ED21
:10851000767A1370A4F8C831A4F8CA31A4F8CC3123
:10852000A4F8CE3192E0012A00F09280022A89D18B
:10853000BDEC028B0720BDE8F84F0AF0A9B9554EF3
:10854000B9F80070F3889F4202D33288BA4202D24F
:10855000B7EB430F76DDB9F80800C0F30B0043F02A
:10856000B3FA092840F38F80337D002584F8C65183
:1085700084F8C751002B00F09D80474A137099B2D0
:10858000B288738812FB01F213FB01F3717C92B283
:108590008A429BB2A4F8C82186BF521A92B2002226
:1085A0008B42A4F8CA3186BF5B1A9BB20023A4F8A1
:1085B000CE31642384F8D1310023A4F8CC21C4F84F
:1085C000D43106E712F054F900284CD102239D4221
:1085D0002A4684F8C73138BF1A4610E7314BD4F821
:1085E000DC111A68337E03EB830303EB8303521A17
:1085F000B2EB830FFFF6F3AE022594ED768A84F892
:10860000C651EEE694F8D00190B90123C4F8D481A4
:1086100084F8D031254BC1F1640100FB01F183FBEB
:108620000103C917A1EBA351643184F8D111F1E61C
:10863000D4F8D4011E4BA8EB00009842EADB84F882
:10864000D111E7E6032D7BD194ED768A0325C8E6A8
:10865000BDEC028B0820BDE8F84F0AF019B9B9F853
:1086600000700C4EB5E6337C834207D301239D4254
:108670002A4684F8C73138BF1A46C0E6002384F87A
:10868000C7312A46BBE6032DDED0A8E6A0B70020FE
:1086900004AA0020E89E002003AA002002AA0020CD
:1086A000ACC5273774210020000000006BCA5F6B47
:1086B00080969800274A284D126892F96C103288EB
:1086C000B7FBF2F20132082A28BF08225FFA82FCC7
:1086D000914285F800C02BD051B3204991F800E0B9
:1086E0000EF1010101F00301714521D0DFF870B0F6
:1086F0004FF0FF304FF0A40A0AE0B0F1FF3F02D183
:10870000002B08BF0846013101F00301714512D06A
:108710000AFB01B393F96C309A42EED10846C0B21D
:10872000F8F7CCFC2B78B9F8007094F8C65126E71E
:108730001D46634623E7431CF1D1634600251EE72F
:10874000B9F80800C0F30B0043F0BEF909283FF761
:10875000C6AE44E65437002003AA00206C35002042
:10876000589B00202DE9F843CE4CA368204698473B
:10877000002800F08F80B4F90E30A17D06EE903A0B
:10878000B4F9103007EE903AB4F9123007EE103A0F
:10879000F8EEE66AF8EEE77AB8EEC77A012309291F
:1087A00084F85430C4ED126AC4ED137A84ED147A5F
:1087B00072D004F1480027F045F9BB4DAA8DAB6A91
:1087C000002A40F0F980B94A1268520700F1C180CE
:1087D000B3F9002094ED125A94ED136A94ED147AD3
:1087E00005EE902AB3F90220B3F9043006EE902A80
:1087F00007EE903AF8EEE55AF8EEE66AF8EEE77A18
:1088000075EE655A76EE666A77EE677A2B88C4ED68
:10881000125AC4ED136AC4ED147ADBB395ED025A13
:1088200095ED056A95ED087AD5ED033A95ED064A82
:10883000D5ED094A75EEC55A76EEC66A77EEC77A67
:10884000A5EEA35AA6EE846AA4EEA77AD5ED015A46
:10885000D5ED046AD5ED077A85ED025A35EE652A25
:1088600076EE662A37EE673AE3EE825AE2EE846AE3
:10887000E4EE837AC5ED015AC4ED125A85ED056A1E
:10888000C5ED046AC4ED136A85ED087AC5ED077A73
:10889000C4ED147ABDE8F883D4ED0B5A94ED0C6A5C
:1088A00094ED0D5AD4ED094A94ED084A804B67EED9
:1088B000A55A27EE866A67EE857A94ED0A5A1B78E8
:1088C000A6EEA46AE6EE845AE6EE857AD4ED0E6A48
:1088D000D4ED0F4A94ED105AE6EE875AF0EE466A50
:1088E000E4EE876AE5EE077AC4ED125AC4ED136A26
:1088F000C4ED147A002B7FF460AF6E4B93ED055AF4
:1089000093ED036A93ED047AD3ED014A93ED004AA7
:1089100026EE866A26EE877A66EE856A93ED025A1F
:10892000A5EEA47AE5EE856AA5EE846AD3ED064A43
:1089300093ED075AD3ED085AA7EEA46AA7EE857AFD
:10894000E7EEA56A84ED126A84ED137AC4ED146A29
:1089500033E7594EB6F8FC21322A63D0002A40F0A2
:10896000CF8096F81A22002A3FF432AF06F5037042
:1089700007C8524F4FF0000C87FB028E86F81AC2D0
:10898000D217A689C2EB2E12921B9A8087FB006237
:10899000C017C0EB221087FB0127C917C1EB2711B5
:1089A00018805980464B0122A3F80EC0C3F80A2054
:1089B000F8F79CFDAB6A0BE7B2F5C87F00F0848046
:1089C0003D4994ED127AD1ED7C6AD4ED137A94EDA1
:1089D000146AF8EEE66A002676EE876A91ED7D7AF3
:1089E000A664B8EEC77AFDEEE66A37EE277AD1EDD7
:1089F0007E7AC1ED7C6AF8EEE77ABDEEC77A77EE53
:108A0000867A0020FDEEE77A012A188081ED7D7AD2
:108A1000E6645880C1ED7E7A2665988075D0013A6B
:108A2000AA85D0E61A68C6F80022B3F90420A6F891
:108A30000422234ADFED237AD268C6F8082294ED97
:108A4000127A0020002177EE877AA0641980B6F8A8
:108A5000FC21FDEEE77A322AC6ED837A00F08280AF
:108A600096ED847AD4ED137AD4ED146AE064B8EE0E
:108A7000C77A012A37EE277AD6ED857A5980F8EE43
:108A8000E77ABDEEC77A77EEA67A2065FDEEE77A43
:108A9000998086ED847AC6ED857A74D0013AA6F87D
:108AA000FC215EE7E4140010AC140010A83500208F
:108AB0005905002028370020A0B700201F85EB5162
:108AC0001C9F002000000000D4ED126A94ED137A80
:108AD000D4ED147A364EFDEEE66ABDEEC77AFDEEB1
:108AE000E77A00200021A064C6ED7C6A198086ED3B
:108AF0007D7AE0645980C6ED7E7A206599808EE7A4
:108B0000D6ED837AF8EEE77A99E717EE906ADFF808
:108B1000A8E0B4F80C80C8368EFB061916EE90CA91
:108B2000F11717EE107AC1EBE9110CF1C80CA1EBAB
:108B300008019980C8378EFB0C614FEAEC7CCCEBC6
:108B4000E11C8EFB071EFF17C7EBEE17A3F800C052
:108B50005F80184BC3F80A20D881F8F7C7FCAA8DAC
:108B6000AB6A5CE794ED137AD4ED147AE064BDEE61
:108B7000C77AFDEEE77A598086ED847A2065C6EDE6
:108B8000857A99808AE70B2086F8192286F81812D0
:108B900009F07EFEAB6AD6F800221A60B6F904220C
:108BA0009A80044AD6F80812D160B6F8FC2175E71D
:108BB000A0B700201C9F00201F85EB5138B5074C43
:108BC000074DAC4203D3074B01221A7038BDD4E9DC
:108BD0000210A28844F0D8FC1C34F2E79CE406089A
:108BE00094ED0608349A00202DE9F04F0C4695B01C
:108BF0003449054620461746FDF7E2FB06460028A5
:108C00004FD131492046FDF7DBFB064600284AD10B
:108C10002E492046FDF7D4FB0646002845D12C49B5
:108C20002046FDF7CDFB0646002840D120462949C5
:108C3000FDF7C6FB0028064612BF0824264601247D
:108C40000FB144F0100424493046FDF7B9FB80B35E
:108C500044F02004214B1B780BB9FFF7AFFFF6F768
:108C600025FC14F0090F00F048831D48F8F70CFEAE
:108C70000020FDF70BFC14F4807306933CD11948D7
:108C8000F8F702FE1848F8F7F9FD04F01803182B5E
:108C900005D11648F8F7F8FD1548F8F7EFFD012360
:108CA0002BE00124CCE70224CAE70424C8E781248E
:108CB000C6E710493046FDF783FB0028CAD044F4CC
:108CC0008074C7E723B406082AB4060832B406083D
:108CD00038B4060868B30608ECA80608349A0020E1
:108CE00046B406084EB4060866B4060872B4060810
:108CF0009AB4060841B4060800230593F8F7A6FDC8
:108D0000AA49AB48F8F764FEAA49AB48F8F760FEF9
:108D100004F48473082B04F0100807D1A7492846EF
:108D2000F8F72AFFA5492846F9F720FF14F0800339
:108D300008930ED1A24B93F81C22002AA14A03F5F6
:108D4000077306BF0121134600219F4A2046F8F70A
:108D500081FD9E492046FDF7DBFB9D492046FDF73E
:108D6000EFFE9C492046FDF75FFC9B4BD3F800B01B
:108D70009A4B1B680493B8F1000F40F0FC819848AF
:108D8000F8F782FD4646974B07930393049BDFF861
:108D900014A36BEA03034FF000090A93039B53F8F3
:108DA000047B0393002F40F0E881049BDFF8F8A2D6
:108DB00063EA0B030993079B53F8042B0392079371
:108DC000002A40F00482884B884A89492046FBF7F4
:108DD00065FC089B002B40F0A282DFF8D0A2DFF8F0
:108DE000D0B29AF800209BF80030DFF8C8929A427F
:108DF00014BF012100217F4A20460CBF0127002714
:108E0000FAF700FB9BF800307B4A013B394659F8E2
:108E1000233006462046F8F765FD9AF80030764A7A
:108E2000013B3946754F59F823302046F8F712FDBB
:108E3000D7ED007A724AF5EE407AF1EE10FA0CBFE7
:108E4000012100212046F8F705FD6E4933463A46D8
:108E50002046FBF79FFE6C4B6C4A6D492046FCF7A1
:108E6000DFFAB8F1000F05D06A4B93F90230002BFE
:108E700000F0DD816848F8F707FD6848F8F7FEFC68
:108E80000023644A6649674F674E2046FCF708FC9A
:108E9000664B01936FF07F4200923A68316820463A
:108EA000FDF738FA40F20222614B01930092BA6852
:108EB000B1682046FDF72EFAB8F1000F40F0B981F5
:108EC0005C48F8F7E1FC42465B485C49DFF8E8C1E2
:108ED0000826012710F8013B11F8019B03F1500E01
:108EE000EE440EF8209C1CF801EB0EF1500AEA4407
:108EF0000AF8109C2FB1A3EB0E0EDEF1000747EB32
:108F00000E07013EE6D187F0010120468DF838605A
:108F1000FAF778FA4A4A8DF8486010AB394620468D
:108F2000F8F7E0FC464A0CAB39462046F8F792FCCD
:108F3000444B454A45492046FCF760F8444B454AB6
:108F400045492046FCF7E8F8444B3F4A3F49204654
:108F5000FCF776F9424B434A43492046FBF74CFA6B
:108F6000424B434A43492046FBF7CCFC424B434A21
:108F700043492046FBF780FF424B434A4349204682
:108F8000FCF77AFE424B434A43492046FCF768FD12
:108F9000B8F1000F40F04F814048F8F775FC404FA2
:108FA000DFF818814FF0000B8AE000BF81A50608AA
:108FB000C7A50608D5A50608EAA50608F1A906086A
:108FC000A0B700200DCB0608AAB40608B7B406085F
:108FD000C1B406084E9F0608983E0020F43B0020CE
:108FE00004B40608C4FA0508DEB40608249E00206E
:108FF00060B5002012B40608E5B406082836002043
:10900000EEB40608D83C002082AD0608FCAC002077
:1090100044AE00205CAD00200CB40608FDB4060888
:10902000D0AD00205C370020203F00200AB50608A4
:1090300011B5060818B4060828B70020FC68060811
:109040000FA5060898A606080CAC0020A8AE0020C4
:109050001DB506088CAC002028AF002018B5060806
:1090600023B50608389F00209CB1002027B50608CC
:10907000D0AA0020B0AF002030B50608FCAB00201D
:109080009CAF002038B50608BC9F0020D4B5002056
:1090900041B50608DC370020983D00201CB40608C6
:1090A000E0B00020C7B40608D3B40608C43F0020CF
:1090B0002136002040FB0508EC9D002088AA0020F6
:1090C00041460222384644F098FA002814BF012194
:1090D0000021039A97F800A020460CBF4FF0010929
:1090E0004FF00009FAF78EF9BAF1020F039040F041
:1090F000A58098F801204FF0190A40F2EE231AFBE0
:109100000232019298F80020884B9A5C00925B46EC
:10911000874A49462046F8F7E5FB7A78834B40F2C8
:10912000EE211AFB021201923A789A5C00925B4699
:109130007F4A49462046F8F78DFB0BF1010BBBF146
:10914000120F07F1020708F10208B9D1794B224644
:1091500000212846FAF7F0F9230700F18580764EC2
:10916000224631782846FDF749F97178224628468B
:10917000FDF768F9B7E0714E05E63B7823B30A9A2C
:10918000012303FA09F31A400CBF012100210992BF
:10919000204632460B93FAF735F9049B63EA0B023B
:1091A0000B9B1A4214BF012100213B465246064642
:1091B0002046F8F797FB099900393B46524618BFFD
:1091C00001212046F8F746FB09F10109E6E5039B7A
:1091D0001B7853B3049B4FF0010909FA07F913EA0E
:1091E000090F0BD06BEA030313EA090F5246039BE6
:1091F00014BF012100212046F8F774FB1BEA090F78
:1092000013D0099B13EA090932460CBF0121002142
:109210002046FAF7F7F8B9F100010646039B5246DB
:1092200018BF01212046F8F715FB0137C3E5444B71
:1092300027E6444A48E6444B0393B0E698F80020FA
:109240003A4B9A5C00925B464946404A2046F8F702
:1092500049FB3A78354B9A5C00925B463B4A49465B
:109260002046F8F7F7FA68E70027F9B222462846C1
:109270000137FDF7C3F8042FF7D12F4FDFF8F08047
:109280003B7888F80030069B33B93148F8F7FCFA90
:1092900030492846FAF72CFEFF2388F80030F1B257
:1092A000224628460136FDF7CDF8042EF7D12A4C88
:1092B0007B782370069BA3B92848F8F7E5FA25497F
:1092C0002846FAF745FE2648F8F7DEFA2548F8F76B
:1092D0009DFAFF232370002015B0BDE8F04FFAF788
:1092E0009CB8FF232370059B002BF4D01E48F8F791
:1092F000CBFA1E48F8F7C2FAEDE7A10706D50E4BE8
:10930000224619782846FDF779F8E4E76207E2D5A6
:10931000094B224659782846FDF794F8DBE7054BC0
:10932000224618212846FAF707F9DCE7F86A06080A
:1093300016A9060823B406080C40002004B4060849
:109340000CB4060818B406081CB4060826A90608BA
:1093500045B50608F1A906089505002068B5060878
:109360008FB50608A5B40608A2B50608B8B5060864
:1093700094050020002237E4012235E4302821D072
:10938000312826D0322828D0332828D0342828D095
:10939000352828D0202828D0212828D0102828D0C7
:1093A000112828D0122828D0132828D0142812D009
:1093B000152826D0162826D0172808BF0F2202D03D
:1093C000002070470022114B03EBC20393F8BC034B
:1093D00070470122F7E70C22F5E70222F3E70322A8
:1093E000F1E70422EFE70522EDE70622EBE707228B
:1093F000E9E70822E7E70922E5E70A22E3E70B228B
:10940000E1E70D22DFE70E22DDE700BF2C2306088F
:109410000123302803FA01F129D031281ED0322847
:109420001CD033281AD0342813D0352811D0202846
:109430000FD021280DD0102810D011280ED01228BE
:109440000CD013280AD0142803D0152801D01628D0
:1094500009D111F0030018BF0120704711F0070077
:1094600018BF012070471728F3D00020704711F073
:10947000070018BF18467047244B82B09A790190B4
:109480008AB393F82630DFED226A224A07EE903A3B
:10949000F8EEE77A204B127886EEA77A83ED107A01
:1094A000FAB11E499FED1E6AB1F84A12DDED017A4C
:1094B00007EE101AB8EE477AF8EE677A27EE067ACA
:1094C000F7EE006A27EE277A002177EE266A03EB93
:1094D000C202C7EE267A1960083343ED017A9A4238
:1094E000F9D102B070470F4A12681201F9D593F80A
:1094F0002630DFED076A07EE903AF8EEE77A064B82
:1095000086EEA77A83ED107AEBE700BFD027002024
:1095100055555540C00D001018160010A0B700207A
:1095200027D4D236A835002010B5437B8268044684
:10953000581C6073D154627B237B934206D82AB1B6
:109540002368D4E9010198470023637310BD00BF6D
:10955000427B42B110B503680446D0E90101984747
:109560000023637310BD704730B5056895F800E0BF
:10957000BEF1010F95B004468C4608D0BEF1020F33
:1095800002D119462B6AB3B1002015B030BD95F950
:109590000450691CF8D0022DF6DC017900922846AF
:1095A0006246F2F74FFA0028EED0284615B0BDE823
:1095B0003040F2F7BFB9CDE90A210DF10F02049254
:1095C0000122CDE90532CDE908336CF07F018DF839
:1095D0001C308DF830208DF844200D931093129399
:1095E00000220023CDE90E238DF80F10EFF3118C2C
:1095F000102383F3128803681B6A0BB3069B04A82D
:1096000002461BB1D3691432002BFBD12B6A6BB11C
:10961000996839B99A4209D0196829B15B68996883
:109620000029F7D01433F3E7C3E900405FFA8CFC5C
:109630008CF311882268136A002BFCD10120A4E767
:1096400004AB2B625FFA8CFC8CF31188F0F7C2FF3D
:10965000F0E700BF30B593B00DF107050892002286
:10966000CDE90252CDE906228DF807108DF81420BD
:10967000012109930B920E92109200230022049173
:109680008DF828108DF83C10CDE90C2301680446B4
:10969000EFF3118C102383F3128803681B6A0BB35A
:1096A000049B02A802461BB1D3691432002BFBD1E4
:1096B0000B6A6BB1996839B9934209D0196829B11D
:1096C0005B6899680029F7D01433F3E7C3E90040D9
:1096D0005FFA8CFC8CF311882268136A002BFCD192
:1096E00013B030BD02AB0B625FFA8CFC8CF31188B7
:1096F000F0F770FFF0E700BF30B40568EFF3118CAE
:10970000102383F3128803681B6AEBB18B6804464D
:109710000A461BB1D3691432002BFBD12B6A6BB103
:10972000986838B9934209D0186828B15B6898687E
:109730000028F7D01433F3E7C3E900415FFA8CFC4B
:109740008CF3118830BC704729625FFA8CFC8CF373
:10975000118830BCF0F73EBF30B5056895F800E0E1
:10976000BEF1010F95B004468C4608D0BEF1020F41
:1097700002D119462B6A7BB1002015B030BD95F996
:109780000400411CF8D00228F6DC217900926246E0
:10979000F2F758F915B030BDCDE90A210DF10F02ED
:1097A00004920122CDE90532CDE908336CF07F0146
:1097B0008DF81C308DF830208DF844200D931093D7
:1097C000129300220023CDE90E238DF80F10EFF342
:1097D000118C102383F3128803681B6A0BB3069B5A
:1097E00004A802461BB1D3691432002BFBD12B6AAB
:1097F0006BB1996839B99A4209D0196829B15B6887
:1098000099680029F7D01433F3E7C3E900405FFA01
:109810008CFC8CF311882268136A002BFCD1012088
:10982000ABE704AB2B625FFA8CFC8CF31188F0F78A
:10983000D1FEF0E730B58BB04FF0010C0091002164
:10984000CDE90123CDE90411CDE9061105688DF8B4
:109850000CC004468DF820C00991EFF3118C102341
:1098600083F3128803681B6A0BB3029B68460246A7
:109870001BB1D3691432002BFBD12B6A6BB19968F1
:1098800039B9934209D0196829B15B6899680029F0
:10989000F7D01433F3E7C3E900405FFA8CFC8CF394
:1098A00011882268136A002BFCD10BB030BDC5F8BB
:1098B00020D05FFA8CFC8CF31188F0F78BFEF0E778
:1098C00030B593B000238DF807108DF806200DF108
:1098D00006010122CDE90332CDE90631CDE9083296
:1098E0000DF107058DF814308DF828208DF83C20F7
:1098F0000B930E93109300220023CDE90C230168F3
:1099000002950446EFF3118C102383F31288036849
:109910001B6A0BB3049B02A802461BB1D369143225
:10992000002BFBD10B6A6BB1996839B9934209D00E
:10993000196829B15B6899680029F7D01433F3E7F7
:10994000C3E900405FFA8CFC8CF311882268136A2B
:10995000002BFCD113B030BD02AB0B625FFA8CFC64
:109960008CF31188F0F736FEF0E700BF30B50568DC
:109970002C78012C83B006D0022C01D12B6ACBB1FC
:10998000002003B030BD95F904408DF80720631C1A
:109990008E460179F4D0022CF2DC0DF107037246F9
:1099A00020463FF085FA0028EAD02046F1F7C2FFB2
:1099B00003B030BDFFF784FF0120E2E730B595B07A
:1099C00000230122CDE90532CDE908338DF81C30A2
:1099D0000D93109312930DF10F030DF107050B92E8
:1099E0008DF830208DF844200A93002200238DF852
:1099F0000710CDE90E23016804950446EFF3118C9E
:109A0000102383F3128803681B6A1BB3069B04A808
:109A100002461BB1D3691432002BFBD10B6A6BB128
:109A2000996839B9934209D0196829B15B68996876
:109A30000029F7D01433F3E7C3E900405FFA8CFC48
:109A40008CF311882268136A002BFCD19DF80F005B
:109A500015B030BD04AB0B625FFA8CFC8CF311883F
:109A6000F0F7B8FDEEE700BF134B1B68B0EB930FA8
:109A700014D2B0EBD30F13D2B0EB131F12D2B0EB52
